:020000040800F2
:1000000000060020E1020008E3020008E302000805
:10001000E3020008E3020008E3020008E30200082C
:10002000E3020008E3020008E3020008F17600089A
:10003000E3020008E3020008E3020008E30200080C
:10004000E3020008E3020008E3020008E3020008FC
:10005000E3020008E3020008FD8500082986000885
:100060005586000881860008AD860008094600080C
:10007000314600085D46000889460008B54600087C
:10008000DD46000809470008E3020008E302000813
:10009000E3020008E3020008E3020008D986000832
:1000A000E3020008E3020008E3020008E30200089C
:1000B000E3020008E3020008E3020008E30200088C
:1000C000E3020008E3020008E3020008E30200087C
:1000D000E3020008E3020008C5870008D98700088A
:1000E0003D870008E3020008E3020008E30200087D
:1000F000E3020008E3020008E302000835470008B5
:10010000E3020008B187000801880008E302000844
:10011000E3020008E3020008E3020008E30200082B
:100120006147000889470008B5470008E147000813
:100130000D480008E3020008E3020008E30200089B
:10014000E3020008E3020008E3020008E3020008FB
:1001500035480008614800088D480008E30200089F
:10016000E3020008E3020008E3020008E3020008DB
:10017000E3020008DD820008E3020008E302000851
:10018000E3020008E3020008ED870008E30200082C
:10019000E3020008E3020008E3020008E3020008AB
:1001A000E3020008E3020008E3020008E30200089B
:1001B000E3020008E3020008E3020008E30200088B
:1001C000E3020008E3020008E3020008E30200087B
:1001D000E3020008C9820008E3020008E302000805
:1001E000E3020008E3020008E3020008E30200085B
:1001F000E3020008E3020008E3020008E30200084B
:10020000E3020008E3020008E3020008E30200083A
:10021000E3020008E3020008E3020008E30200082A
:10022000E3020008E3020008E3020008E30200081A
:10023000E3020008E3020008E3020008E30200080A
:10024000E3020008E3020008E3020008E3020008FA
:10025000E3020008E3020008E3020008E3020008EA
:10026000E3020008E3020008E3020008E3020008DA
:10027000E3020008E3020008E3020008E3020008CA
:10028000E3020008E3020008E3020008E3020008BA
:10029000E3020008E3020008E3020008E3020008AA
:1002A000E3020008E3020008E3020008E30200089A
:1002B000E3020008E3020008E3020008E30200088A
:1002C000E3020008E3020008E3020008E30200087A
:1002D000E3020008E3020008E3020008E30200086A
:1002E00002E000F000F8FEE772B6374880F30888B5
:1002F000364880F3098836483649086040F20000E5
:10030000CCF200004EF63471CEF200010860BFF36B
:100310004F8FBFF36F8F40F20000C0F2F0004EF637
:100320008851CEF200010860BFF34F8FBFF36F8F8B
:100330004FF00000E1EE100A4EF63C71CEF20001E3
:100340000860062080F31488BFF36F8F07F032FA3D
:1003500006F0A4FB4FF055301F491B4A91423CBFA9
:1003600041F8040BFAE71D49184A91423CBF41F895
:10037000040BFAE71A491B4A1B4B9A423EBF51F83D
:10038000040B42F8040BF8E700201849184A914280
:100390003CBF41F8040BFAE707F04AFA06F002FC0A
:1003A000144C154DAC4203DA54F8041B8847F9E7A6
:1003B00000F0C4F9114C124DAC4203DA54F8041B9E
:1003C0008847F9E707F032BA000600200022002033
:1003D0000000000808ED00E00000002000060020FA
:1003E000989C00080022002074220020782200201F
:1003F00034670020E0020008E0020008E002000884
:10040000E00200082DE9F04F2DED108AC1F80CD064
:10041000D0F80CD0BDEC108ABDE8F08F002383F338
:1004200011882846A047002006F01AF9FEE706F0DA
:1004300073F800DFFEE7000053B94AB9002908BF8E
:1004400000281CBF4FF0FF314FF0FF3000F074B9AF
:10045000ADF1080C6DE904CE00F006F8DDF804E01B
:10046000DDE9022304B070472DE9F047089D0446FA
:100470008E46002B4DD18A42944669D9B2FA82F257
:1004800052B101FA02F3C2F1200120FA01F10CFA93
:1004900002FC41EA030E94404FEA1C48210CBEFBCB
:1004A000F8F61FFA8CF708FB16E341EA034306FB54
:1004B00007F199420AD91CEB030306F1FF3080F0E3
:1004C0001F81994240F21C81023E63445B1AA4B230
:1004D000B3FBF8F008FB103344EA034400FB07F7D2
:1004E000A7420AD91CEB040400F1FF3380F00A8113
:1004F000A74240F207816444023840EA0640E41B08
:1005000000261DB1D4400023C5E900433146BDE8B3
:10051000F0878B4209D9002D00F0EF800026C5E955
:10052000000130463146BDE8F087B3FA83F6002E6D
:100530004AD18B4202D3824200F2F980841A61EBE5
:10054000030301209E46002DE0D0C5E9004EDDE703
:1005500002B9FFDEB2FA82F2002A40F09280A1EBEB
:100560000C014FEA1C471FFA8CFE0126200CB1FB40
:10057000F7F307FB131140EA01410EFB03F0884239
:1005800008D91CEB010103F1FF3802D2884200F2C6
:10059000CB804346091AA4B2B1FBF7F007FB101158
:1005A00044EA01440EFB00FEA64508D91CEB0404F6
:1005B00000F1FF3102D2A64500F2BB800846A4EB51
:1005C0000E0440EA03409CE7C6F12007B34022FA3C
:1005D00007FC4CEA030C20FA07F401FA06F31C436B
:1005E000F9404FEA1C4900FA06F3B1FBF9F8200C78
:1005F0001FFA8CFE09FB181140EA014108FB0EF0BE
:10060000884202FA06F20BD91CEB010108F1FF3A0D
:1006100080F08880884240F28580A8F10208614419
:10062000091AA4B2B1FBF9F009FB101144EA014127
:1006300000FB0EFE8E4508D91CEB010100F1FF34D2
:100640006CD28E456AD90238614440EA0840A0FB6A
:100650000294A1EB0E01A142C846A64656D353D040
:100660005DB1B3EB080261EB0E0101FA07F722FA64
:1006700006F3F1401F43C5E9007100263146BDE88D
:10068000F087C2F12003D8400CFA02FC21FA03F3F0
:10069000914001434FEA1C471FFA8CFEB3FBF7F071
:1006A00007FB10360B0C43EA064300FB0EF69E4296
:1006B00004FA02F408D91CEB030300F1FF382FD22F
:1006C0009E422DD9023863449B1B89B2B3FBF7F6D7
:1006D00007FB163341EA034106FB0EF38B4208D9B0
:1006E0001CEB010106F1FF3816D28B4214D9023EF1
:1006F0006144C91A46EA004638E72E46284605E70F
:100700000646E3E61846F8E64B45A9D2B9EB0208DF
:1007100064EB0C0E0138A3E74646EAE7204694E76F
:100720004046D1E7D0467BE7023B614432E73046A2
:1007300009E76444023842E7704700BF38B501F06A
:10074000FFF901F0AFFB06F0C1FE054606F0C6FF5B
:100750000446D0B90F4B9D4219D001339D4241F25E
:10076000883504BF01240025002006F0B9FE0CB135
:1007700000F078F801F036FB00F026FD08B100F03B
:1007800071F8284600F01CF9F9E70025ECE705466A
:10079000EAE700BF010007B008B501F09DF9A0F13C
:1007A00020035842584108BD07B541F21203022107
:1007B00001A8ADF8043001F0ADF903B05DF804FB19
:1007C00038B5302383F31188174803680BB106F05E
:1007D0002BF80023154A4FF47A71134806F01AF8E3
:1007E000002383F31188124C236813B12368013B63
:1007F0002360636813B16368013B63600D4D2B7820
:1008000033B963687BB9022001F056FA3223636082
:100810002B78032B07D163682BB9022001F04CFA27
:100820004FF47A73636038BD78220020C107000856
:100830009823002090220020084B187003280CD821
:10084000DFE800F008050208022001F02BBA0220C0
:1008500001F01EBA024B00225A607047902200201D
:1008600098230020F8B5504B504A1C4619680131B6
:1008700000F0998004339342F8D162684C4B9A425D
:1008800040F291804B4B9B6803F1006303F500330A
:100890009A4280F08880002001F06CF90220FFF776
:1008A000CBFF454B0021D3F8E820C3F8E810D3F87C
:1008B0001021C3F81011D3F81021D3F8EC20C3F89D
:1008C000EC10D3F81421C3F81411D3F81421D3F881
:1008D000F020C3F8F010D3F81821C3F81811D3F89A
:1008E0001821D3F8802042F00062C3F88020D3F8AA
:1008F000802022F00062C3F88020D3F88020D3F853
:10090000802042F00072C3F88020D3F8802022F0CB
:100910000072C3F88020D3F8803072B64FF0E02325
:10092000C3F8084DD4E90004BFF34F8FBFF36F8FB6
:10093000224AC2F88410BFF34F8F536923F48033E7
:100940005361BFF34F8FD2F8803043F6E076C3F3A4
:10095000C905C3F34E335B0103EA060C29464CEA92
:1009600081770139C2F87472F9D2203B13F1200F5C
:10097000F2D1BFF34F8FBFF36F8FBFF34F8FBFF332
:100980006F8F536923F4003353610023C2F8503250
:10099000BFF34F8FBFF36F8F302383F311888546EA
:1009A00080F308882047F8BD0000020820000208F4
:1009B000FFFF0108002200200044025800ED00E083
:1009C0002DE9F04F93B0B44B2022FF2100900AA8EC
:1009D0009D6801F0B1F9B14A1378A3B90121B0487B
:1009E00011700360302383F3118803680BB105F0A5
:1009F0001BFF0023AB4A4FF47A71A94805F00AFFA8
:100A0000002383F31188009B13B1A74B009A1A604F
:100A1000A64A1378032B03D000231370A24A536015
:100A20004FF0000A009CD3465646D146012001F003
:100A300039F924B19C4B1B68002B00F02682002062
:100A400001F04AF80390039B002BF2DB012001F038
:100A50001FF9039B213B1F2BE8D801A252F823F07A
:100A6000E10A0008090B00089D0B00082D0A000888
:100A70002D0A00082D0A00082F0C0008FF0D0008A1
:100A8000190D00087B0D0008A30D0008C90D000812
:100A90002D0A0008DB0D00082D0A00084D0E000885
:100AA000810B00082D0A0008910E0008ED0A0008CD
:100AB000810B00082D0A00087B0D00082D0A000894
:100AC0002D0A00082D0A00082D0A00082D0A00082A
:100AD0002D0A00082D0A00082D0A00089D0B0008A9
:100AE0000220FFF759FE002840F0F981009B022107
:100AF00005A8BAF1000F08BF1C4641F21233ADF849
:100B0000143001F007F891E74FF47A7000F0E4FF39
:100B1000071EEBDB0220FFF73FFE0028E6D0013F77
:100B2000052F00F2DE81DFE807F0030A0D1013360F
:100B30000523042105A8059300F0ECFF17E004212C
:100B40005548F9E704215A48F6E704215948F3E7E4
:100B50004FF01C08404608F1040801F00DF804218C
:100B6000059005A800F0D6FFB8F12C0FF2D10120B6
:100B70004FF0000900FA07F747EA0B0B5FFA8BFB0F
:100B800001F026F926B10BF00B030B2B08BF002454
:100B9000FFF70AFE4AE704214748CDE7002EA5D01B
:100BA0000BF00B030B2BA1D10220FFF7F5FD07463D
:100BB00000289BD00120002600F0DCFF0220FFF778
:100BC0003BFE1FFA86F8404600F0E4FF0446B0B151
:100BD000039940460136A1F140025142514100F0D3
:100BE000E9FF0028EDD1BA46044641F21213022172
:100BF00005A83E46ADF8143000F08CFF16E72546F8
:100C00000120FFF719FE244B9B68AB4207D9284609
:100C100000F0B2FF013040F067810435F3E70025B2
:100C2000224BBA463E461D701F4B5D60A8E7002E62
:100C30003FF45CAF0BF00B030B2B7FF457AF02209C
:100C4000FFF7FAFD322000F047FFB0F10008FFF691
:100C50004DAF18F003077FF449AF0F4A08EB0503C7
:100C6000926893423FF642AFB8F5807F3FF73EAFC0
:100C7000124BB845019323DD4FF47A7000F02CFF3E
:100C80000390039A002AFFF631AF039A0137019BC4
:100C900003F8012BEDE700BF002200209423002081
:100CA00078220020C107000898230020902200200D
:100CB00004220020082200200C2200209422002080
:100CC000C820FFF769FD074600283FF40FAF1F2D2E
:100CD00011D8C5F120020AAB25F003008449424532
:100CE000184428BF4246019201F000F8019AFF2102
:100CF0007F4801F021F84FEAA803C8F387027C4936
:100D00002846019301F020F8064600283FF46DAF15
:100D1000019B05EB830533E70220FFF73DFD00282B
:100D20003FF4E4AE00F064FF00283FF4DFAE00279C
:100D3000B846704B9B68BB4218D91F2F11D80A9B2D
:100D400001330ED027F0030312AA134453F8203CBA
:100D500005934046042205A9043701F003F98046B3
:100D6000E7E7384600F008FF0590F2E7CDF8148079
:100D7000042105A800F0CEFE02E70023642104A8A8
:100D8000049300F0BDFE00287FF4B0AE0220FFF710
:100D900003FD00283FF4AAAE049800F01FFF059061
:100DA000E6E70023642104A8049300F0A9FE0028CC
:100DB0007FF49CAE0220FFF7EFFC00283FF496AED4
:100DC000049800F00DFFEAE70220FFF7E5FC002899
:100DD0003FF48CAE00F01CFFE1E70220FFF7DCFCE3
:100DE00000283FF483AE05A9142000F017FF074642
:100DF0000421049004A800F08DFE3946B9E73220A2
:100E000000F06AFE071EFFF671AEBB077FF46EAE00
:100E1000384A07EB0903926893423FF667AE022017
:100E2000FFF7BAFC00283FF461AE27F003074F44F8
:100E3000B9453FF4A5AE484609F1040900F09CFE0F
:100E40000421059005A800F065FEF1E74FF47A70E3
:100E5000FFF7A2FC00283FF449AE00F0C9FE0028CD
:100E600044D00A9B01330BD008220AA9002000F0CD
:100E70006BFF00283AD02022FF210AA800F05CFF77
:100E8000FFF792FC1C4805F0F1FB13B0BDE8F08FB2
:100E9000002E3FF42BAE0BF00B030B2B7FF426AE92
:100EA0000023642105A8059300F02AFE07460028C8
:100EB0007FF41CAE0220FFF76FFC804600283FF451
:100EC00015AEFFF771FC41F2883005F0CFFB0598B5
:100ED00000F0C6FF46463C4600F07AFFA6E506460F
:100EE0004EE64FF0000901E6BA467EE637467CE65C
:100EF0009422002000220020A086010070470000FC
:100F000070470000704700002DE9F04100F5803780
:100F1000044616463B7C5BB9C0681030204400F0A4
:100F2000E5FEE5683544B5F5004FE56002D816B139
:100F3000BDE8F081DEB905F07F0605F11000002163
:100F4000C6F180062044F6B232462E4400F0F4FE8C
:100F5000A06804F11008324600F10060414600F537
:100F6000003006F05FF830B901233B74E0E74FF43E
:100F700000463546ECE7A26805F1100140463244D0
:100F80002144A260E268521BE26000F0AFFE022042
:100F9000BDE8F04100F090BE183000F0E9BC000060
:100FA00010B5044600F0FAFF204610BD10B5044607
:100FB00000F0F4FF204610BDC3B280B2A3F141029D
:100FC000052A02D8373800B27047613B052B94BF21
:100FD00057383038F7E70000F8B50446154608469C
:100FE00003220C4900F08CFE014688B908346F1CBE
:100FF00015F91100FFF7E0FF064617F9110001315E
:10100000FFF7DAFF102940EA061004F8010BEFD1D0
:10101000F8BD00BF549200082DE9F04FADF53F7DBB
:101020000746416801222AA802F09AFE002840F0F3
:1010300087800646824681461125DFF80C81DFF85D
:101040000CB101AB4FF4805241462AA802F0E8FFF0
:10105000002875D1019AB2F5805F71D8002A65D059
:101060000446019A9442ECD2282D0FD008DC132DAF
:101070002DD01E2D39D0112D13D00134A4B2F0E79C
:10108000322D2DD0372D2FD02D2DF6D13B68121BB0
:1010900008EB040138461B692D259847BDF804402C
:1010A000EBE7121B022A09D9594608EB040000F0AD
:1010B00027FE18B902342825A4B2DEE718F8043058
:1010C0003A2B3DD00A2B1CBFA1461325D5E718F8B3
:1010D00004300A2B34D03A2B04BFA2463225CCE789
:1010E00018F80430202BC8D0264618F804300A2BF4
:1010F0001AD1AAEB090208EB090102A811254F2A0F
:1011000028BF4F2208F092F8A21B08EB060116A890
:101110004F2A28BF4F2208F089F83B6816AA02A977
:10112000DB6838469847A8E71E25A6E73B6838469F
:1011300004491B69984701200DF53F7DBDE8F08FFC
:101140000020F9E756930008A023002058920008D9
:1011500000F1180110B5044686B00846019100F070
:10116000F1FB2046FFF758FF60B1019902A800F09B
:1011700049FC102204F1080102A808F017F8B0FA9F
:1011800080F0400906B010BD70B504460025EEB2EF
:10119000304600F0FFFC58B100213046013500F028
:1011A00009FD08B9002070BD022000F085FDEEE7C2
:1011B0002046FFF731FF0028F4D004F58034207C6E
:1011C00080F00100EFE70000F0B5C9B006F096F935
:1011D00000F000FF18B90025284649B0F0BD694667
:1011E0002A4802F0DFFF00284BD1294C204603F0AB
:1011F00009F8284803F006F8274803F003F82146C9
:10120000224803F07BF80028E5D1702000F0C0FEF2
:10121000064610B1214B44600360336830469B683A
:101220009847054600282ED01A4F1948394603F032
:1012300065F805460028CED1194800F0A9FE0446FD
:1012400038B1184B4760036000F58033C0E90255A0
:101250001D74236820469B689847054628B10E49AF
:101260000C4803F04BF80028B5D1336830465B6872
:1012700098471CB1236820465B68984700F092FEAF
:10128000AAE70025FAE70446EFE700BF5C920008F2
:101290006C9200088392000899920008BC920008A2
:1012A00014000100D89200082DE9F04FD44A8DB007
:1012B0000B68D0F804A001931A440368D14E1A4475
:1012C000D1F81C90DFF8B4C3DFF8B4B3D0E902342E
:1012D000634003EA0A03634013444A6802920AEB3C
:1012E0007363029CC84A2244C468224484688AEA20
:1012F00004051D40654015448A68039203EB35558B
:10130000039CC24A2244846822448AEA03042C4093
:1013100084EA0A041444CA6805EBF43404921644BF
:1013200083EA0502224056445A4032440E6905962B
:1013300004EBB222059FB64E3E441E4485EA0403E8
:1013400013406B4033444E69069602EB7363069F6D
:10135000B04E3E442E4484EA02051D4065403544AB
:101360008E69079603EB3555079FAB4E3E442644E6
:1013700082EA03042C4054403444A84E4E4405EB0A
:10138000F434164483EA050222405A4032440E6A7D
:10139000089604EBB222089FA14E3E441E4485EA03
:1013A000040313406B4033444E6A099602EB7363A7
:1013B000099F9C4ED1F830E03E44D1F83880F34488
:1013C0002E4484EA02051D40654035448E6AA6F528
:1013D000244703EB35550A964F3F274482EA03041E
:1013E0002C4054403C44CF6A0B9705EBF4340B9EE1
:1013F0008D4F3744029E174483EA050222405A402B
:101400003A448A4F774404EBB2221F4485EA04032E
:1014100013406B403B444F6BBC4402EB7363654429
:1014200084EA020C0CEA030C8CEA040C6544DFF835
:1014300054C2C44403EB3555A44482EA03042C404F
:1014400054406444D1F83CC0794905EBF43461441C
:10145000114483EA050222405A400A44754904EBCC
:10146000B2223144079E194484EA02032B406340B0
:101470000B44714902EBF36331440B9E0D4482EA45
:1014800003012140514029446C4D03EBF151354497
:10149000019E254483EA010414405C402C44684DBD
:1014A00001EBB4443544069E154481EA04021A4017
:1014B0004A402A44634D04EB323235440A9E1D44AF
:1014C00084EA02030B4063402B445F4D02EBF3635D
:1014D0003544059E0D4482EA0301214051402944D0
:1014E0005A4D03EBF1516544254483EA010414404D
:1014F0005C402C44564D01EBB4443544099E1544E0
:1015000081EA04021A404A402A44524D04EB323226
:101510003544049E1D4484EA02030B4063402B447F
:101520004D4D02EBF36345440D4482EA0301214033
:1015300051402944494D03EBF1513544089E2C4458
:1015400083EA010515405D402C44454D01EBB44450
:101550003544039E2A4481EA04051D404D402A4437
:10156000404D04EB32323D442B4484EA020593445F
:101570000D4065402B443C4D02EBF3633544069E21
:10158000294482EA0305254055402944374D03EBA1
:10159000F1514D442C4483EA010515405D4025443A
:1015A00001EBB54581EA050404EA03024A405A44C6
:1015B000A6F5B82B089E05EB3232ABF2BE6B544059
:1015C0005B4423442A4C344402EB33730B9E0C449B
:1015D00085EA020159402144264C344403EB715101
:1015E000029E254482EA03044C402544224C444494
:1015F00001EB3545144483EA01026A40224443E08A
:1016000078A46AD7EECEBDC156B7C7E8DB702024F8
:10161000AF0F7CF52AC68747134630A8019546FDD3
:10162000D8988069AFF7448BBED75C892211906B44
:101630002108B44962251EF640B340C0515A5E26C7
:10164000AAC7B6E95D102FD65314440281E6A1D88B
:10165000C8FBD3E7E6CDE121D60737C3870DD5F424
:10166000ED145A4505E9E3A9F8A3EFFCD9026F6729
:1016700081F6718722619D6D0C38E5FD937198FDAF
:101680008A4C2A8D8E4379A6934C344405EB722202
:10169000059E1C4481EA0503534023448F4C344487
:1016A00002EB33730A9E0C4485EA0201594021443F
:1016B0008B4C4C4403EB7151254482EA03044C40AB
:1016C0002C44884D354401EB3444019E154483EA93
:1016D000010262402A44844D3D4404EB72221D44C1
:1016E00081EA040353402B44804D354402EB3373AD
:1016F000049E294484EA02055D4029447C4D35441A
:1017000003EB7151079E254482EA03044C402C44AC
:10171000784D354401EB3444099E2A4483EA01059F
:1017200065401544744A324404EB7525039E134406
:1017300081EA04026A401A44704B734405EB32722A
:101740000B4484EA0501514019446D4B634402EB9C
:1017500071511C4485EA02034B401C44694B3344DD
:1017600001EB3444019E1D4482EA010363402B4493
:10177000654D04EB73233544069E154463EA01026C
:1017800062402A44614D03EBB2624D4462EA0409AF
:1017900029445F4D89EA0309454449442C445D4D81
:1017A00002EBB1513544049E61EA03081D4488EA06
:1017B0000208444401EB744464EA02034B402B44A6
:1017C000554D04EBF323754463EA010E15448EEA8C
:1017D000040E0EEB0502514D03EBB262354462EA92
:1017E000040E29440A9D8EEA030EA5F580164C4D81
:1017F0007144A6F6833602EBB151264461EA030434
:1018000054403444029E01EB7444354464EA0206B9
:101810001D444E407319089E424D04EBF32335449A
:1018200063EA01061544664072193F4D03EBB2624C
:10183000654462EA040629443C4D5E403144079EFB
:1018400002EBB151354461EA03062C44384D564051
:101850003D443444059E1D4401EB744464EA020394
:101860004B402B44334D04EBF32335440B9E15447E
:1018700063EA010262402A442F4D03EBB262354411
:10188000039E0D4462EA0401594029442B4D02EBAA
:10189000B15135442A4E254461EA030454402C4496
:1018A000099D01EB74442E4464EA02051E4485EA56
:1018B00001039D1903681A440AEB040303EBF523A3
:1018C0000260436083681C44C36819448460C1603B
:1018D0000DB0BDE8F08F00BF44EABEA4A9CFDE4B37
:1018E000604BBBF670BCBFBEC67E9B28FA27A1EA40
:1018F0008530EFD4051D880439D0D4D9E599DBE6CD
:10190000F87CA21F6556ACC4442229F497FF2A43F1
:10191000A72394AB39A093FCC3595B6592CC0C8F81
:10192000D15D84854F7EA86FE0E62CFE144301A3B1
:10193000A111084E827E53F735F23ABDBBD2D72AA9
:1019400091D386EB094B036003F18833436003F1C5
:101950002943A3F59613A3F68B638360A3F1883321
:10196000C3600023C0E90433704700BF012345670B
:101970002DE9F8431446026905460E46E300C2F31A
:10198000C50800F118079B18036122BF43690133A2
:10199000436112F4FC7F436903EB5473436114D039
:1019A000C8F1400907EB08004C4504D22246BDE8C7
:1019B000F84307F00BBC403C4A464E4407F006FC97
:1019C000444439462846FFF76FFCA04606EB04095D
:1019D000B8F13F0FA9EB08010AD94022384607F0B9
:1019E000F5FB39462846A8F14008FFF75DFCEFE714
:1019F000A1096FF03F02384602FB014206EB81115C
:101A0000D5E7000070B50B6901F1180506460C46D4
:101A1000C3F3C503EA18501C8022EA54C3F13F0205
:101A2000072A1FD8002100F087F929462046FFF732
:101A30003BFC38220021284600F07EF92369294624
:101A40002046236563696365FFF72EFC214610225B
:101A5000304607F0BBFB204658220021BDE870400D
:101A600000F06AB9C3F137020021E5E72DE9F84F2C
:101A70004FF47A7306460D46002402FB03F7DFF8A5
:101A80005080DFF8509098F900305FFA84FA5A1CC1
:101A900001D0A34210D159F824002A4631460368E8
:101AA000D3F820B03B46D847854205D1074B0120EB
:101AB00083F800A0BDE8F88F0134042CE3D14FF483
:101AC000FA7004F0D3FD0020F4E700BFE4330020F7
:101AD0001022002014220020002307B50246012115
:101AE0000DF107008DF80730FFF7C0FF20B19DF81A
:101AF000070003B05DF804FB4FF0FF30F9E700008A
:101B00000A46042108B5FFF7B1FF80F00100C0B21A
:101B1000404208BD074B0A4630B41978064B53F8CB
:101B20002140014623682046DD69044BAC4630BCA9
:101B3000604700BFE433002014220020A08601008B
:101B400070B50A4E00240A4D05F010FA308028685E
:101B50003388834208D905F005FA2B680444013321
:101B6000B4F5003F2B60F2D370BD00BFE633002018
:101B7000A033002005F0C8BA00F1006000F5003085
:101B80000068704700F10060920000F5003005F039
:101B900049BA0000054B1A68054B1B889B1A834203
:101BA00002D9104405F0DEB900207047A0330020B0
:101BB000E633002038B50446074D29B12868204493
:101BC000BDE8384005F0E6B92868204405F0D0F9B2
:101BD0000028F3D038BD00BFA0330020002070479C
:101BE00000F1FF5000F58F10D0F80008704700009A
:101BF000064991F8243033B100230822086A81F89D
:101C00002430FFF7BFBF0120704700BFA43300207E
:101C1000014B1868704700BF0010005C194B013879
:101C20000322084470B51D68174BC5F30B042D0C37
:101C30001E88A6420BD15C680A46013C82421346CC
:101C40000FD214F9016F4EB102F8016BF6E7013AB9
:101C500003F10803ECD181420B4602D22C2203F897
:101C6000012B0424094A1688AE4204D1984284BF4D
:101C7000967803F8016B013C02F10402F3D1581A83
:101C800070BD00BF0010005C2422002018930008E3
:101C9000022803D1024B4FF080529A61704700BF77
:101CA00000100258022803D1024B4FF480529A616F
:101CB000704700BF00100258022804D1024A53693D
:101CC00083F48053536170470010025870B5044686
:101CD0004FF47A764CB1412C254628BF412506FBAE
:101CE00005F0641B04F0C2FCF4E770BD002310B5DE
:101CF000934203D0CC5CC4540133F9E710BD00001B
:101D0000013810B510F9013F3BB191F900409C42F8
:101D100003D11AB10131013AF4E71AB191F9002067
:101D2000981A10BD1046FCE703460246D01A12F975
:101D3000011B0029FAD1704702440346934202D0A6
:101D400003F8011BFAE770472DE9F8431F4D1446CD
:101D50000746884695F8242052BBDFF870909CB364
:101D600095F824302BB92022FF2148462F62FFF737
:101D7000E3FF95F824004146C0F1080205EB80001E
:101D8000A24228BF2246D6B29200FFF7AFFF95F8D5
:101D90002430A41B17441E449044E4B2F6B2082E2B
:101DA00085F82460DBD1FFF723FF0028D7D108E0B6
:101DB0002B6A03EB82038342CFD0FFF719FF002881
:101DC000CBD10020BDE8F8830120FBE7A43300203D
:101DD000024B1A78024B1A70704700BFE4330020A0
:101DE00010220020F8B5194C194803F047FF21468E
:101DF000174803F06FFF24684FF47A70154ED4F83B
:101E00009020154DD2F80438114F43F00203C2F868
:101E10000438FFF75BFF2046104904F069F8D4F856
:101E200090200424D2F8043823F00203C2F80438C6
:101E30004FF4E133336055F8040BB84202D0314619
:101E400003F07AFE013CF6D1F8BD00BF189B0008F4
:101E500018490020CC33002014220020209B0008C9
:101E60000C4B70B50C4D04461E780C4B55F82620D3
:101E70009A420DD00A4B002118221846FFF75CFF4A
:101E80000460014655F82600BDE8704003F054BEDA
:101E900070BD00BFE4330020142200201849002048
:101EA000CC330020F8B571B6002301201A4619463C
:101EB00002F094FD0446802005F0C6F9002849D0C0
:101EC0000025254A80274FF4D06C3D26136913F076
:101ED000C06F26D1D2F8103113F0C06F21D1236822
:101EE00005F1006199602368D86023685F6023680A
:101EF000C3F800C021680B6843F001030B60216840
:101F00000B6823F01E030B6021680B68DB07FCD411
:101F1000237B8035616806FA03F3B5F5001F0B607B
:101F2000D4D1204602F09AFDB5F5001F11D000244F
:101F30000A4E0B4D012005F0E7F83388A34205D97E
:101F400028682044013405F025F8F6E7002005F064
:101F5000DBF861B6F8BD00BF00200052E633002078
:101F6000A033002030B50A44084D91420DD011F83D
:101F7000013B5840082340F30004013B2C4013F080
:101F8000FF0384EA5000F6D1EFE730BD2083B8EDBF
:101F90000121884238BF084605F08EB908B105F026
:101FA0008FB9704710B5084C01220849002001F094
:101FB000B3FE23783BB1064803F036FD044803F036
:101FC00069FD0023237010BDE8330020289300082A
:101FD000C83600201D482DE9F041036D2BB90122C0
:101FE0004FF48051503005F0CBFA194E33780BB1D5
:101FF000FFF7D8FF0324174F4FF00008134D154982
:102000002846C7F8048003F037FD284603F070FB2C
:1020100048B1013C284603F03DFD14F0FF04EED129
:10202000204634700FE00C4901220C4801F074FE88
:10203000014618B1284603F0F7FCEAE7084800F02B
:1020400011F801203070BDE8F08100BFC8360020D3
:10205000E83300203C22002028930008EC330020C5
:102060002C9300080FB4002004B07047006870473C
:1020700003460068596870470B0A017043700B0CE7
:10208000090E8370C1707047110A027003714170AC
:10209000110C120E8170C2701A0A42711A0C1B0EBA
:1020A0008271C37170470000C36A0239023B8B42E0
:1020B00083BF4389006C01FB0300002070470000D0
:1020C000C2F307238A76CB760378032B01BF120C69
:1020D0000A75120A4A75704700F10B010022D301FC
:1020E00043EA520310F8012B52FA83F38842DAB222
:1020F000F5D110467047000010B541780446002025
:10210000013102464901022A16BFA35C032203EBF8
:10211000C03302F101021EBF9BB203EB500398B221
:102120009142F0D810BD000002684AB1134613F87E
:10213000011B1F290DD93A29F9D1911C8B4202D0DC
:102140004FF0FF3070471278302AF9D10360002039
:102150007047014B187870473836002038B50D4667
:10216000044618B9092000232B6038BD0368002BF2
:10217000F8D01A78002AF5D08188DA889142F1D116
:10218000587804F00FFC10F00100EBD12368EBE766
:1021900038B50D4640F25231144602F0B9F9FF2825
:1021A00007D9012C0BD9030A022468702B70204632
:1021B00038BD30B1002CFAD001242870F7E7002494
:1021C000F5E70446F3E700002DE9F8430026D0F8D0
:1021D000008005460C468E76836B002B4AD098F81B
:1021E0000030042B4BD133463546402720E0B7F56D
:1021F000187F80F0C480F90606F1010608BF023797
:10220000D05B02372BB900F5205292B2B2F5006FC5
:102210000DD305F11A01C5F1FF0240EA0340214444
:10222000FFF7B6FF002800F0AA800544002003460F
:10223000D8F8102092F82310B142D8D8002B40F0E3
:102240009E80002D00F09B8000232544AB766373B5
:10225000D8F81020137903F03701DB0621730BD473
:1022600002F13800FFF704FFC4E90001938963819C
:10227000D3892381BDE8F88300200146F4E7C36CCD
:1022800001335ED1EA6B00232E26551E184615F841
:10229000011F013020290CD0052908BFE52109289C
:1022A00004D10B2B9EBFE71801337E73E71801336F
:1022B00079730B28EBD1E11800204873A17E002927
:1022C0004BD1002B40D06FF00C0604F10D00082517
:1022D000361B331810F8011B002938D02E298BB279
:1022E0004AD0A3F14101192903D8117B0D4200D036
:1022F00020330373EDE7B9F1000F05D100F520534A
:102300009BB2B3F5006F0BD307F11A01C7F1FF02BF
:1023100040EA09402144FFF73BFF48B10744002051
:1023200002368146D8F80C30985B0028E3D1384655
:10233000B9F1000F4FF0000218BF002023189A7661
:10234000A0E7B1463746EDE73F23A37601232344B8
:1023500000219976137B03B96373D37A02F11C00D1
:1023600003F03F0323730023FFF780FE20606360C8
:10237000D38A6381138B7CE710250B46B9E73F2393
:102380000125A37660E7000038B50546002435F83E
:10239000020B08B9204638BD02F0EEF86308C2B25D
:1023A00003EBC43312FA83F39AB2C0F3072303EBAF
:1023B000520303EBC2339CB2E9E7000037B5C378A0
:1023C00004461BB90025284603B030BD00F14C017E
:1023D000826C01234078019104F00AFB054680B924
:1023E000A36BE070A06C226BC31A9342EAD2A3786D
:1023F0000199022BE6D102440123607804F0F8FA37
:10240000E1E70125DFE7000038B5836C05460C469F
:102410008B4210D0FFF7D2FF60B92246012305F1AD
:102420004C01687804F0C0FA00281CBF4FF0FF345C
:102430000120AC6438BD0020FCE7000038B5002363
:102440000446C3704FF0FF338364FFF7DDFF0028BD
:102450004BD1B4F84A524AF655239D4207D10B227C
:10246000254904F14C0006F0A1FE00283FD094F865
:102470004C30EB2B03D01833DBB2012B2ED84AF6AD
:1024800055239D4206D108221C4904F19E0006F006
:102490008DFE48B3B4F85730B3F5007F1ED194F8E1
:1024A0005930DBB15A1E1A4218D1B4F85A30ABB1C8
:1024B00094F85C30013B012B10D8B4F85D306BB15F
:1024C000B4F85F307F2B06D804F16C00FFF7CEFD27
:1024D000B0F5803F02D3B4F8623053B94AF65520C4
:1024E00085420CBF0220032038BD0420FCE70120F8
:1024F000FAE70020F8E700BF58930008649300084B
:1025000002392DE9F04701F007044FF0010A466C4B
:1025100005460AFA04F41746984606EB1136C1F34D
:10252000C809E4B2314628460136FFF76DFF18B1FD
:102530000120BDE8F087994605EB090292F84C307E
:10254000234214BF01210021414513D06340013FC4
:1025500082F84C3085F803A0EBD0640014F0FF043F
:10256000EAD109F1010301244FF00009B3F5007F1E
:10257000E1D1D7E70220DCE701290246F8B50C4695
:1025800040F28C800668F36A8B4240F28780337891
:10259000013B032B00F28280DFE803F00229384B75
:1025A00004EB5405B16B304601EB5521FFF72CFFCE
:1025B00010B14FF0FF30F8BD6F1CC5F30805B16BCB
:1025C0003046354401EB572195F84C50FFF71CFF7E
:1025D0000028EED1C7F30807E3073E4496F84C0005
:1025E00045EA00204CBF0009C0F30B00E3E7B16BE4
:1025F000304601EB1421FFF707FF0028D9D1640012
:1026000004F4FF742644B6F84C00D4E7B16B3046AE
:1026100001EBD411FFF7F8FE0028CAD1A40006F19F
:102620004C0004F4FE742044FFF720FD20F07040BD
:10263000C1E7D0E90430D57953EA000101D09168AF
:1026400001B95DBB9168022DA4EB01010DD1013BE5
:10265000728940F1FF305B0A43EAC053B3FBF2F3E7
:1026600099421BD81CD0601CA5E7032D02D19369A9
:102670008B42F8D8D3699BB9B16B304601EBD411CA
:10268000FFF7C2FE002894D1A0004C3600F4FE7083
:102690003044FFF7EBFC20F000408CE701208AE794
:1026A0006FF0004087E70000F8B5066804460D4665
:1026B0003378042B0CBF4FF080524FF400128A4243
:1026C00001D80220F8BDCA06FBD182680163D2B9E5
:1026D000022B13D83389B3EB551FF2D9F36BA363E5
:1026E000A36B6263002BECD003EB55234C36C5F390
:1026F00008050020A3633544E563E3E7F36BC2718B
:10270000002BE7D01A4677897F02BD42114604D2DA
:102710003046FFF7C9FCA063E2E72046FFF72CFF35
:10272000431C024606D00128CBD9F36A8342C8D99C
:10273000ED1BEAE70120C5E701292DE9F047064630
:102740000C46174608D9C36A8B4205D90378022B79
:1027500062D003D8012B22D0022552E0033B012B8B
:10276000FAD8816B01EBD411FFF74EFE0546002825
:1027700047D1A40006F14C0304F4FE741C443378E2
:10278000042B07D0204627F07047FFF76FFC00F0BE
:102790007040074339462046FFF76EFC2FE001EBFF
:1027A0005108816B01EB5821FFF72EFE054640BB17
:1027B00014F0010406F14C0908F1010AC8F30808F5
:1027C00008BFFBB230461FBF19F8083003F00F02F4
:1027D0003B0103F0F00318BF134309F8083001234D
:1027E000B16BF37001EB5A21FFF70EFE054640B9BD
:1027F000CAF3080A44B1C7F3071709F80A7001239E
:10280000F3702846BDE8F08719F80A30C7F30327AC
:1028100023F00F031F43F0E7816B01EB1421FFF757
:10282000F3FD05460028ECD1640006F14C0304F4E6
:10283000FF741F551919C7F307274F70DFE7000012
:10284000F8B504460E461746E3690BB91846F8BDBD
:10285000012BA6EB0305206814BFAA1C3A46691C8D
:10286000FFF76AFF0028F2D1E369013BE361EBE780
:1028700001292DE9F84306460C461746056802D89B
:102880000220BDE8F883EB6A8B42F9D97AB9A146F8
:1028900021463046A046FFF76FFE0446B0B92B78BC
:1028A000042B02D1002F43D1F7710020E9E72B78E8
:1028B000042B02D1C379022BE9D04FF0FF32394605
:1028C0002846FFF739FF0028E1D0DAE70128D7D002
:1028D000421C01D10120D4E72B78042B19D1EA6ADC
:1028E000AB69023A93421CD308F10102A2420CD018
:1028F0002B78042B08D10023A2EB09024946284675
:10290000FFF7FEFD0028BCD1A146EB6AA342BFD869
:10291000C5E7002241462846FFF70EFF0028DED01B
:10292000AFE70133AB612B7943F001032B71DBE798
:10293000F3798BB9B468BC4202D10223F371B4E7D6
:1029400021463046FFF718FE012899D9431CC1D013
:1029500001348442EFD0A8E7032BA6D1B368BB4271
:10296000A3D8B2691344BB429FD3E6E770B5C379DD
:102970000446032B06D181688369CD18A94203D18F
:102980000023E371002070BD4E1C20683246FFF723
:10299000D3FE0028F7D13146F0E700002DE9F743D8
:1029A00005460191FFF70AFD0446002849D105F1CB
:1029B0004C09019928464FF40072FFF775FB214638
:1029C000A86407464846FFF7B7F96C896402B4F576
:1029D000004F28BF4FF40044B4F5007F2FD92046A4
:1029E00004F072FC804630B122460021640A0026C1
:1029F000FFF7A2F909E06408EEE72346BA19414659
:102A0000687803F0F5FF18B926446B899E42F4D329
:102A1000404604F069FC6889801B18BF012003B0A0
:102A2000BDE8F08301366B899E42F4D20123BA19C6
:102A30004946687803F0DCFF0028F3D0EBE7002676
:102A4000F1E70120EBE70000F8B50446FFF7B6FC1C
:102A50000546002842D12378032B37D12779012F4F
:102A600034D104F14C0601464FF400723046FFF7B2
:102A700063F955234122722184F84A32AA2304F5CE
:102A80000D7084F84F2084F84B32522384F83012B2
:102A900084F84C3084F84D30612384F8311284F886
:102AA0004E3084F83332A16984F83222FFF7E4FA19
:102AB000616904F50E70FFF7DFFA626B3B46314641
:102AC00001326078A26403F093FF257100226078E0
:102AD000114603F0B1FF003818BF0120F8BD000017
:102AE00000232DE9F0430B6085B00F461546FFF734
:102AF0001BFB061EC0F2B281804B53F82640002C0F
:102B000000F0AE813C6005F0FE0523786BB1607883
:102B100003F048FFC70708D41DB110F0040500D02A
:102B20000A25284605B0BDE8F0830023F0B22370E3
:102B3000607003F023FFC10700F194810DB14207DB
:102B4000EED400212046FFF779FC022840F099805E
:102B50006E4604F2122304F2522132461846103314
:102B6000FFF784FA42F8040B8B42F7D1002556F8A0
:102B7000041B00297DD02046FFF760FC012879D88E
:102B80000128A26C40F0C08004F1570304F18C01CD
:102B900013F8015B002D7BD18B42F9D1B4F8B4302E
:102BA000B3F5807F74D194F8B830092B70D104F15B
:102BB0009400FFF75DFA4FF0FF33171841F1000161
:102BC000BB4275EB010363D304F1A000FFF74EFA9B
:102BD00094F8BA302063012BA37059D194F8B990BE
:102BE00003FA09F91FFA89F36381002B50D0444B93
:102BF00004F1A800FFF73AFA0646984248D8831C29
:102C0000626304F1A400E362FFF730FA00EB02080C
:102C100004F19C00C4F84080FFF728FA10441FFA22
:102C200089F2A06306FB02F313EB080345EB0502F0
:102C30009F4271EB02032BD32E4604F1AC00FFF749
:102C400015FAE06365B96389B34221D9E16B204687
:102C5000FFF72AFA81192046FFF7D6FB98B901360B
:102C6000631993F84C30812B14D02035C5F3080537
:102C7000E8E703200135042D7FF479AF042807D15C
:102C800001E0042801D101254BE701287FF678AF48
:102C90000D2546E705F1140004F14C063044FFF71A
:102CA000E5F901280546F3D9E36A8342F0D9618941
:102CB000821E236C02FB01336364A16B204601EB8F
:102CC000D511FFF7A1FB0028DDD105F07F0006EB51
:102CD0008000FFF7CBF9431C03D00135A842ECD0AC
:102CE000D6E70425C4E90500064A257000251388A7
:102CF000E56101339BB21380E38012E73C3600208C
:102D0000FDFFFF7F40360020B4F85730B3F5007F59
:102D1000BED1B4F8626026B904F17000FFF7A6F9DD
:102D2000064694F85C302663591EA3700129AFD87B
:102D300094F859506581002DAAD0691E2942A7D167
:102D4000B4F85D8018F00F0FA4F80880A0D1B4F893
:102D50005F0018B904F16C00FFF788F9B4F85A1055
:102D6000002995D006FB03FE01EB181CF4446045D6
:102D70008ED3A0EB0C00A842B0FBF5F388D33E48FD
:102D8000834285D84FF6F57083426DD903259F1C89
:102D9000114402EB0C03032DE7626263A163236419
:102DA0004CD1B4F8763053EA08037FF471AFBB001E
:102DB00004F17800FFF75AF9E06303F2FF13B6EB72
:102DC000532FFFF465AF4FF0FF33032DC4E90533F4
:102DD0004FF08003237187D1B4F87C30012B83D16D
:102DE000511C2046FFF710FB00287FF47DAFB4F89C
:102DF0004A224AF6552320719A427FF475AF1F4B41
:102E000004F14C00FFF732F998427FF46DAF03F103
:102E1000FF5304F50C70FFF729F903F50053203335
:102E200098427FF461AF04F50D70FFF71FF9A061C0
:102E300004F50E70FFF71AF9606155E7B8F1000F5D
:102E40003FF426AF7144022D4FEA4703E1631EBFF2
:102E5000D91907F0010303EB5103AEE70B2560E638
:102E60000C255EE603255CE640F6F575AB428CBFAB
:102E7000022501258BE700BFF5FFFF0F525261418C
:102E80002DE9F84F07460568884649B96E69C6B10D
:102E9000EB6AB34298BF0126AB69A3B9002405E0F1
:102EA000FFF76AFB0128044603D801242046BDE849
:102EB000F88F421C00F0D280EB6A8342F6D8464677
:102EC000EAE70126E8E72A78EB6A042A40F08380E3
:102ED000A6F1020A023B4FF0010B9A4528BF4FF0C2
:102EE000000AD146696C284601EB1931FFF78CFACC
:102EF00000283BD109F00703EA6AC9F3C8010BFABD
:102F000003F3901EDBB26A184C4609F1010992F8EE
:102F10004C20814502EA030233BF5B0000234FF4DB
:102F20000071DBB228BF9946B2B90234631E033385
:102F3000BCD80123214628461A46FFF7E1FA0228A9
:102F4000B3D0012800F08A80B8F1000F13D102231A
:102F5000FB710028A9D130E0CA450AD0002BD2D19C
:102F60000131B1F5007FBDD20123CCE74FF0FF3432
:102F7000DCE70024DAE7FB79022B07D1731CA342BC
:102F8000E7D0BB68F31ABB610323FB7108F10102B0
:102F9000FB69A24205D113B10133FB61D9E70223DA
:102FA000FBE70BB90123FB61224641463846FFF798
:102FB00047FC00284FD10123FB61EA6AAB69023A62
:102FC0006C6193429CBF03F1FF33AB612B7943F0FB
:102FD00001032B716AE7464514D1741C3846A3429D
:102FE00098BF02242146FFF7C7FA01283FF45DAFDE
:102FF000431C33D0E0B16B69012B03D9EA6A9342D9
:1030000038BF1E4634460134EB6AA34203D8012E72
:103010007FF644AF022421463846FFF7ADFA48B1A7
:1030200001283FF442AF013018D0B442EBD135E76C
:10303000002CE7D04FF0FF3221462846FFF77CFBFB
:1030400048B9B8F1000FB8D0224641462846FFF7EC
:1030500073FB0028B1D001287FF427AF4FF0FF3475
:1030600024E700002DE9F84306680446076B89460B
:1030700033782037042B0CBF4FF080534FF40013EC
:10308000BB429CBF00238363836B73B1C7F3080803
:10309000B8F1000F3CD10133416B836339B93389F7
:1030A000B3EB571F34D80023A36304200AE07389CD
:1030B000013B13EA57232BD1FFF75EFA012805469F
:1030C00002D80220BDE8F883421C01D10120F9E7B3
:1030D000F36A834216D8B9F1000FE4D0616B204641
:1030E000FFF7CEFE0546C8B10128EAD0431CEDD05B
:1030F00001463046FFF752FC0028E7D1E37943F060
:103100000403E371294630466563FEF7CDFFA063F3
:103110004C36002027634644E663D3E70720D1E717
:10312000F8B50E46002104460768FFF7BDFA98B9C6
:103130000546A16B3846FFF767F968B93A78E36B43
:10314000042A1B780CD11B060ED50546012120460A
:10315000FFF788FF0028ECD0042808BF072006E00E
:10316000E52B01D0002BF0D10135B542EED1F8BDF1
:10317000C16C4B1C2DE9F04104460568066B1FD15C
:10318000E5274FF00108A16B2846FFF73DF998B9F4
:103190002A78E36B042A09BF1A781F7002F07F02B5
:1031A0001A7085F80380236BB3420DD200212046AC
:1031B000FFF758FF0028E6D0042808BF022003E0EC
:1031C000FFF772FA0028DBD0BDE8F0812DE9F0416D
:1031D00005460068A96B0669FFF716F9044620B991
:1031E000EB6B1A78852A03D002242046BDE8F081D3
:1031F000324603F1200153F8040B8B4242F8040BD2
:10320000F9D1777801377F01A7F16003B3F5007F2B
:10321000EAD800212846FFF725FF04280446E3D01A
:103220000028E2D1A96B2868FFF7EEF804460028D1
:10323000DBD1EB6B1A78C02AD6D106F1200203F15C
:10324000200153F8040B8B4242F8040BF9D196F895
:1032500023300F222C33B3FBF2F3B7EB431FC3D35E
:103260004FF0400800212846FFF7FCFE04280446E2
:10327000BAD00028B9D1A96B2868FFF7C5F8044671
:103280000028B2D1EB6B1A78C12AADD1B8F5187FFE
:1032900009D206EB080203F1200153F8040B8B421C
:1032A00042F8040BF9D108F120084745DAD8B8F5FF
:1032B000187F9AD83046FEF71FFF7388834294D058
:1032C00092E700000B68002210B5036004460B6A09
:1032D00083604B6AC261C37123F0FF03896AC0E94E
:1032E0000432C164FFF7E0F920B92046BDE8104080
:1032F000FFF76CBF10BD0000F8B503680546012755
:103300001C692046FEF7F8FEA070000A6678E0709F
:103310002846E96CFFF7C8F920B1022828BF02202F
:10332000C0B2F8BDA96B2868FFF76EF80028F4D189
:10333000EB6B04F1200254F8041B944243F8041B85
:10334000F9D12B68DF70002EE7D000212846013E1E
:10335000FFF788FEE0E700002DE9F8434FF0FF0893
:1033600006460768042445464FF6FF79B16B11B94C
:10337000002C73D063E03846FFF746F80446002877
:103380005DD1F06B0378002B6ED03A78042A11D10E
:10339000852B4DD1336B3046F364FFF717FF04469E
:1033A00000284CD13B691B7903F03F03B3712046E1
:1033B000BDE8F883C27AE52B02F03F02B27143D038
:1033C0002E2B41D022F0200108293DD00F2A40D1D8
:1033D000590637D503F0BF05336B90F80D80F364C1
:1033E000437B434530D1428B72BB03780D21FC688F
:1033F00023F04003DFF874E0013B4B4301211EF84A
:1034000001CB30F80CC009B3FF2B1DD824F813C032
:103410006146013301320D2AF1D10278520605D5F9
:1034200021B1FF2B10D8002224F81320013DEDB26A
:1034300000213046FFF716FE0446002896D00023F0
:10344000B363B4E7AB42CBD0FF25F1E7CC45E1D085
:10345000FAE72DB9FEF740FE404501D10024A6E76A
:103460004FF0FF33F364A2E70424E8E70094000878
:103470002DE9F04F002187B00446D0F80090FFF707
:1034800013F9804670B999F80030042B33D1D9F87C
:103490000C00FEF779FF07462046FFF75DFF054663
:1034A00020B18046404607B0BDE8F08FD9F8103013
:1034B0009A8CBA42F0D193F823B040265D4506D1EC
:1034C000D9F80C3033F81530002BE5D1EAE7F106D6
:1034D000D9F8103008BF0236985B01F04DF8D9F8E2
:1034E0000C30824633F8150001F046F88245D3D1FE
:1034F00002360135E2E74FF0FF0A4FF0FF3B554639
:10350000C4F84CB0A16B4846FEF77EFF00285CD1A2
:10351000E66B3778002F77D0F27AE52F02F03F0381
:10352000A37103D0120704D50F2B04D0C4F84CB0FC
:103530004FE00F2B54D194F84B3058063FD4790606
:1035400045D5236B07F0BF0796F80DA0E364737BA6
:1035500053453ED1738B002B3BD135780121D9F8EF
:103560000C3005F03F0501930D23013D5D43284BD1
:1035700013F8012BB25A71B3FF2D059329D81046C9
:10358000049200F0F9FF6B1C03900293019B33F847
:10359000150000F0F1FF039981421AD1049A029DAF
:1035A0001146059B1B4A9342E2D133785A0604D553
:1035B00019B1019B33F815305BB97D1EEDB20021C6
:1035C0002046FFF74FFD00289CD080466AE7BD42A9
:1035D000BDD0FF25F3E74FF6FF708242E2D0F8E757
:1035E0002DB93046FEF778FD50453FF45BAF94F8B7
:1035F0004B30DB079AD40B2204F14001304605F032
:10360000D5FD002892D14DE74FF004084AE700BFEE
:10361000009400080D9400082DE9F04F90F84BB08D
:1036200099B004461BF0A00540F068810668F26876
:1036300032F81530002B4AD13378042B40F08780C4
:103640000F230E352046B5FBF3F5A91CFFF768FDE7
:103650008146002877D1236B0135A3EB4515E3792B
:103660005A07E56435D523F004032046E371FFF7DC
:103670007DF950BB4FF0FF32616B2046FFF7E0F859
:1036800018BBA3682BB3214604A8FFF71BFEE0B9C3
:1036900070894FF40071D4E90423E0FB0123306901
:1036A000C4E904233830FEF7EFFC3069D4E9042381
:1036B0002830FEF7E9FCE379326904A843F00103FE
:1036C00082F82130FFF718FE18B181463BE0013542
:1036D000AEE7D6E90354402200212046FEF72CFB3A
:1036E0008523012140222370C0234FF0C10C04EB3D
:1036F000010884F8203000231E469E46571C04F81B
:1037000002C0F0B2023204F807E021B135F813101C
:1037100009B10133DBB20F0AA15408F8027002327A
:10372000D706F2D135F813700136002FE6D184F8B0
:103730002330831C28466370FEF726FE84F824009D
:10374000000A84F82500484619B0BDE8F08F04F15E
:1037500040070DF1100A1BF0010F97E807008AE8F7
:10376000070000F0D38040234FF0010884F84B306D
:10377000BC46F368B8F1050F9AE80700ACE803000F
:103780002CF8022B4FEA12428CF8002059D9981ECF
:10379000424630F8021F002942D10DF10F0C0721DB
:1037A00002F00F0E914612090EF13000392888BF41
:1037B0000EF1370001390CF8010902D0B9F10F0FF1
:1037C000EED818AB7E205A1802F8580C3846002262
:1037D000914206D010F801CB02F1010EBCF1200F8E
:1037E00031D104F13F0C072902F1010297BF18AB58
:1037F00020205818013198BF10F8580C072A0CF8EF
:103800000200F0D92046FFF733FE8146002878D128
:1038100008F10108B8F1640FAAD14FF0070992E747
:103820004FF0100C01F0010E49080EEB4202D303D9
:1038300044BF82F4883282F02102BCF1010CF1D144
:10384000A7E74246A9E77246C2E7216B2046A1EBF3
:103850004511FEF729FF814600287FF474AF4FF62B
:10386000FF783846FEF738FC0190A16B3046FEF732
:10387000CBFD814600287FF466AFE36BE9B2019A85
:103880004FF00D0CD6F80CE05A734FF00F02DFF832
:10389000E0A0DA724A1E18730CFB02F28446987696
:1038A000D87640451AF8019B0CF1010C18BF3EF880
:1038B000120003EB090B18BF013203F809004FEAAD
:1038C0001029002808BF4046BCF10D0F8BF801906D
:1038D000E7D1404502D03EF812200AB941F040013C
:1038E0001970012300212046F370FFF7BBFB8146CE
:1038F00000287FF428AF013DB7D11BE04FF0060947
:1039000021E704287FF41FAF84F84BB01BF0020FAF
:1039100020461BBF0C350D210125B5FBF1F518BF65
:1039200001352946FFF7FCFB814600287FF40BAFE9
:10393000013D8AD1A16B3046FEF766FD8146002825
:103940007FF401AF01462022E06BFEF7F5F9E36B4F
:1039500003CF18605960BA7839889A72198194F83F
:103960004B30E26B03F0180313730123F370EAE6A4
:103970000094000810B504460A463430FEF776FB82
:10398000886004F13800FEF773FBC2E9040194F883
:10399000213003F00203D3710023D36110BD000076
:1039A00003284B8B04BF8A8A43EA024318467047B8
:1039B0002DE9F04F0B7899B0044689462F2BD0F8AB
:1039C00000B001D05C2B09D14A46137891460132F0
:1039D0002F2BFAD05C2BF8D0002301E0DBF81C3051
:1039E000A3600023E3619BF80030042B1ED1A36881
:1039F000E3B1DBF82030214604A82362DBF8243051
:103A00006362DBF82830A362FFF75CFC0346002802
:103A100054D1DBF8102002F13800FEF727FBC4E98F
:103A2000040392F8213003F00203E37199F80030A7
:103A30001F2B00F2358180230021204684F84B3073
:103A400019B0BDE8F04FFEF72FBE49460B78894606
:103A500001312F2BFAD05C2BF8D01F2B8CBF002507
:103A60000425012F2FD113882E2B31D1002322F8CA
:103A7000173004F140029F428CBF2E2120210133D8
:103A80000B2B02F8011BF6D145F02005204684F8E7
:103A90004B50FFF7EDFC94F84B30002800F0E78026
:103AA00004280BD1990603F0040240F1DC80002ABF
:103AB00000F0F6808023002084F84B3019B0BDE878
:103AC000F08F0425CDE7022F02D153882E2BCAD0C8
:103AD000911E87BB002322F81730002F00F01181C0
:103AE00032F81300194601332028F9D009B92E28DD
:103AF00001D145F00305901E30F817302E2B01D070
:103B0000013FF9D14FF020334FF0000A6364D046F3
:103B10002364C4F847300823481C32F81160009031
:103B2000F6B1202E03D02E2E0DD1B84210D045F084
:103B300003050099F0E731F81730202B01D02E2B28
:103B4000C8D1013FC5E79A4505D20099B9423BD19A
:103B50000B2B30D101E00B2B27D145F003050B23B4
:103B600094F84020E52A04BF052284F84020082B61
:103B700004BF4FEA88085FFA88F808F00C030C2BA2
:103B800003D008F00303032B01D145F00205A80779
:103B90003FF57CAF18F0010F18BF45F0100518F085
:103BA000040F18BF45F0080570E70099B94202D02C
:103BB00045F00305D4D84FEA88080B234FF0080AD4
:103BC00000975FFA88F8B4E77F2E15D9304640F2A7
:103BD0005231CDE9022345F00203019300F098FC35
:103BE00010F0800F0646DDE9022316D000F07F06B4
:103BF00046498E5D019D46B331464548CDE90123D6
:103C000005F0FEFADDE90123F8B9A6F1410189B218
:103C100019291ED848F0020810E0FF28EAD9591ED9
:103C20008A4503D345F003059A4682E704EB0A016F
:103C3000000A0AF1010A019D81F8400004EB0A0123
:103C40000AF1010A81F8406073E745F003055F2639
:103C5000F4E7A6F1610189B219299EBF203E48F020
:103C60000108B6B2EAE7002A08BF052026E75A078E
:103C70003FF524AFA379DB0645D59BF80000042867
:103C800035D1A3682146E27923622369DBF810006D
:103C900023F0FF0313436362E36CA362FFF76AFE42
:103CA00023680027DA6819F8010B00283FF409AFF0
:103CB00040F25231009200F04BFC054608B31F2839
:103CC000009A7FF6FEAE2F283FF4BFAE5C283FF48B
:103CD000BCAE7F2805D801460E4805F091FA009A3F
:103CE00078B9FF2F0DD022F817500137DBE7216B91
:103CF0000BF14C03C1F308011944FFF751FEA0601A
:103D0000CEE70620DAE60520D8E600BF809300085B
:103D100079930008709300081FB5CDE9001003A83F
:103D200014460391FEF700FA002815DB0B4A52F8FF
:103D300020300BB100211970019B0BB100211970CB
:103D400042F820302CB1002201A96846FEF7C8FED7
:103D50000446204604B010BD0B24FAE73C36002090
:103D60002DE9F04798B0904605460191002800F0F3
:103D7000528102F03F0603A901A83246FEF7B0FEC9
:103D8000002840F04681039B4FF48C60049303F0BD
:103D90009BFA0746002800F04081039B00F5007263
:103DA0000199D86004A81A61FFF702FE044620B901
:103DB0009DF95B30002BB8BF062418F01C0F00F0F3
:103DC000CD80002C4CD0042C40D104A8FFF724FC5B
:103DD000044600283AD146F00806039B1A78042AC4
:103DE00040F08380186929462B60FFF7C3FD039BD1
:103DF0001E22002118690230FDF79EFF039C00215E
:103E00001A2220692630FDF797FF236920221A71B4
:103E1000246903F093FA0146012208342046FEF794
:103E20002BF9039B04A81B6983F82120FFF764FA90
:103E3000044658B9A96801B302462846FEF718FDA2
:103E4000AB68039A0446013B5361B4B1384603F0B2
:103E50004BFA0CB100232B60204618B0BDE8F08768
:103E60009DF8163013F0110F40F0848018F0040F05
:103E700040F0C98018F0080FAFD1039A31071399A9
:103E8000936C48BF46F04006E964AB6410780428A0
:103E900072D1069B9DF817102B62089B106923F0C6
:103EA000FF030B4329466B62179BAB62FFF762FD72
:103EB000DDF80CA00024002205F15008BAF8063005
:103EC00021464046C5F800A0AB80002385F830604D
:103ED00085F831406C64C5E90E234FF40072FDF79C
:103EE0002BFFB20653D40024B0E703F027FA0146B3
:103EF000009013980E30FEF7BFF813980099163013
:103F0000FEF7BAF8039C13992078FFF749FD2023A8
:103F100000228046CB7220461399FEF7D1F8139BFE
:103F2000002201211A775A779A77DA77039BD970A2
:103F3000B8F1000FA1D0414604A8D3F84890FEF78D
:103F400097FC0446002881D149460398FEF75CFAA5
:103F5000039B044608F1FF30586176E7002C7FF49C
:103F600075AF9DF81630DC064FD418F0020F84D0E0
:103F7000D80782D5072469E7FFF712FD0023A86060
:103F800001F11C00FEF772F86B61286190E7D5E93A
:103F9000046956EA0903A6D0BAF80AA0A9684FEA4C
:103FA0004A2AC5E90E69B24574EB09031BD3002404
:103FB0002964002C7FF44AAFC6F30803002B92D08B
:103FC000039C2046FEF770F808B3760A01234146A9
:103FD00046EAC95682196A64607802F0E5FC041E5C
:103FE00018BF012432E72846FEF7C6FAB6EB0A06E8
:103FF000014669F10009012803D9431CD3D10124EA
:10400000D6E70224D4E7082420E704241EE702248C
:104010001CE704461EE709241EE711241CE70000E4
:104020002DE9F04F994685B00023884603A9044640
:10403000C9F800301646FEF791F8054680BB94F8A3
:1040400031506DBB94F8303013F00103009300F051
:10405000A68004F1500AD4E90432D4E90E011B1AF7
:1040600062EB0102B34272F1000238BF1E46BEB1DC
:10407000D4E90E10C1F30803002B40F08280039BAB
:104080005A894B0A013A43EAC0531A401BD151EAFC
:10409000000309D1A06801280DD8022584F8315009
:1040A000284605B0BDE8F08F216C20460192FEF74E
:1040B00063FA019AEFE7431C04D10123009D84F8C1
:1040C0003130EDE72064DDF80CB0216C5846FDF787
:1040D000EBFF0028E1D0B6F5007F02EB000731D3FB
:1040E000BBF80A1002EB5620730A88429BF80100C5
:1040F00088BF8B1A3A464146019302F055FC0028CE
:10410000DBD194F93020019B002A0BDA606CC01BD4
:10411000984207D24FF40072514608EB4020FDF759
:10412000E5FD019B5F02D9F80030F61BB8443B4423
:10413000C9F80030D4E90E32DB1942F10002C4E9BB
:104140000E3294E7626CBA421AD094F93030002BE8
:104150000DDA012351469BF8010002F049FC0028CA
:10416000ABD194F8303003F07F0384F830300398FB
:1041700001233A465146407802F016FC00289CD1B3
:104180006764A16B4046C1F30801C1F50077514453
:10419000B74228BF37463A46FDF7A8FDC3E70725D3
:1041A0007EE7000070B596B00E460022019002A98D
:1041B00001A8FEF795FC0446E0B94FF48C6003F0CB
:1041C00083F80546D8B1029B00F500720199D860CA
:1041D00002A81A61FFF7ECFB044640B99DF9533081
:1041E000002B0ADB1EB1314602A8FDF7EDFF284681
:1041F00003F07AF8204616B070BD0624F7E71124C4
:10420000F8E7000070B5B8B00222019003A901A838
:10421000FEF766FC044608BB039B4FF48C601093CA
:1042200003F052F80546002866D0039B00F50072A3
:104230000199D86010A81A61FFF7BAFB044650B97B
:104240009DF88B30980655D4190653D49DF8463006
:10425000DA0706D50724284603F046F8204638B08A
:1042600070BD039B04931878042814D104A918691D
:10427000FFF780FB069E9DF84630DB0610D410A8A1
:10428000FEF776FF04460028E5D156BB0398FEF7FB
:10429000DBFB0446DFE71F99FFF782FB0646EAE7F0
:1042A000039BDA69B242D5D024930021269624A834
:1042B0001B78042B01BFDDE90823CDE928239DF8F5
:1042C00017308DF89730FEF7EFF904460028C2D179
:1042D00024A8FFF741F804460028BBD00428BAD12F
:1042E000CDE70246314604A8FEF7C2FA044600288C
:1042F000B1D1CBE70624AEE71124AFE7F0B5BDB0EE
:10430000CDE900106846FDF70FFF022203A901A8BE
:10431000FEF7E6FB0446002841D1039B4FF48C6076
:10432000149302F0D1FF0546002800F0EE80039BB5
:1043300000F5007214AE0199D8601A613046FFF79B
:1043400037FB044640BB9DF89B3013F0A00F40F0B4
:10435000D880039B009F1A78042A68D11B6904AC9B
:1043600003F1400C1868083353F8041C22466345D7
:1043700003C21446F6D15022314628A8FDF7B6FCF8
:10438000394628A8FFF714FB044600284CD12A9A86
:10439000169B9A4206D00824284602F0A5FF204624
:1043A0003DB0F0BD349A209B9A42F4D128A8FFF783
:1043B00033F904460028EFD1039B04AF1B6993F83F
:1043C00001E093F823C09C8C3A46083303CAB242FA
:1043D00043F8080C43F8041C1746F5D1039B28A8A2
:1043E0001B6983F801E0039B1A6982F823C01A69EC
:1043F00082F82440240A82F825401A691379D906E4
:104400005CBF43F020031371FEF776FF04460028DB
:10441000C2D13046FEF7ACFE04460028BCD103985A
:10442000FEF712FB0446B7E70428B5D1BEE7239A8E
:1044300004AB02F1200C1068083252F8041C1C4630
:10444000624503C42346F6D15022314628A8FDF721
:104450004DFC394628A8FFF7ABFA044600284CD19A
:104460002A9A169B9A4296D1349A209B9A4292D1CC
:1044700028A8FFF7D1F8044600288DD137990DF10F
:104480001D030DF12D0001F10D0253F8044B834281
:1044900042F8044BF9D11888012710809B7893705B
:1044A0009DF81B30039CDA0658BF43F02003CB7203
:1044B000E770CB7ADB06ACD5169A2A9B9A42A8D035
:1044C0002078FFF76DFA01462046FDF7EDFD014625
:1044D000C8B12046FDF798FF044600287FF45CAF82
:1044E000039890F86D302E2B93D12A9A00F16C012D
:1044F000FDF7E6FD039BDF708BE704287FF44CAFEC
:10450000B6E7062448E7022446E7112447E70000FF
:104510007F2810B501D880B210BDB0F5803F13D20E
:1045200040F2523399420FD10849002231F8024B30
:1045300093B2844203D103F18000C0B2ECE70132B0
:10454000802AF3D11346F6E70020E5E7C09600087D
:104550007F280DD940F25233994208D1FF2806D85E
:1045600000F10040034B803833F810007047002002
:10457000704700BFC0960008B0F5803FF0B522D26A
:104580001F4A83B21F49B0F5805F28BF0A46141D39
:1045900034F8042C2146AAB1934213D334F8025CB8
:1045A0002E0AEFB252FA85F5A84222DA082E09D86F
:1045B000DFE806F0050A10121416181A1C00801AFB
:1045C00034F810301846F0BD981A00F001001B1A9C
:1045D0009BB2F7E7103BFBE7203BF9E7303BF7E7FF
:1045E0001A3BF5E70833F3E7503BF1E7A3F5E35354
:1045F000EEE70434002ECBD101EB4702C7E700BF42
:10460000109400080496000808B5074B074A19687B
:1046100001F03D01996053680BB190689847BDE87F
:10462000084003F09DB800BF00000240443600205F
:1046300008B5084B1968890901F03D018A019A60A3
:10464000054AD3680BB110699847BDE8084003F0EC
:1046500087B800BF000002404436002008B5084B70
:104660001968090C01F03D010A049A60054A536972
:104670000BB190699847BDE8084003F071B800BFDE
:10468000000002404436002008B5084B1968890D27
:1046900001F03D018A059A60054AD3690BB1106AA1
:1046A0009847BDE8084003F05BB800BF0000024037
:1046B0004436002008B5074B074A596801F03D0110
:1046C000D960536A0BB1906A9847BDE8084003F07F
:1046D00047B800BF000002404436002008B5084B30
:1046E0005968890901F03D018A01DA60054AD36AF7
:1046F0000BB1106B9847BDE8084003F031B800BF1C
:10470000000002404436002008B5084B5968090CE7
:1047100001F03D010A04DA60054A536B0BB1906B5E
:104720009847BDE8084003F01BB800BF00000240F6
:104730004436002008B5084B5968890D01F03D0149
:104740008A05DA60054AD36B0BB1106C9847BDE857
:10475000084003F005B800BF0000024044360020C6
:1047600008B5074B074A196801F03D019960536C81
:104770000BB1906C9847BDE8084002F0F1BF00BF54
:10478000000402404436002008B5084B1968890926
:1047900001F03D018A019A60054AD36C0BB1106D9E
:1047A0009847BDE8084002F0DBBF00BF00040240AC
:1047B0004436002008B5084B1968090C01F03D018A
:1047C0000A049A60054A536D0BB1906D9847BDE895
:1047D000084002F0C5BF00BF00040240443600207C
:1047E00008B5084B1968890D01F03D018A059A60EA
:1047F000054AD36D0BB1106E9847BDE8084002F032
:10480000AFBF00BF000402404436002008B5074B8C
:10481000074A596801F03D01D960536E0BB1906EA3
:104820009847BDE8084002F09BBF00BF000402406B
:104830004436002008B5084B5968890901F03D014C
:104840008A01DA60054AD36E0BB1106F9847BDE854
:10485000084002F085BF00BF00040240443600203B
:1048600008B5084B5968090C01F03D010A04DA60EB
:10487000054A536F0BB1906F9847BDE8084002F0AE
:104880006FBF00BF000402404436002008B5084B4B
:104890005968890D01F03D018A05DA60054AD36F38
:1048A00013B1D2F880009847BDE8084002F058BF25
:1048B000000402404436002000230C4910B51A467B
:1048C0000B4C0B6054F82300026001EB43000433EF
:1048D0004260402BF6D1074A4FF0FF339360D3601C
:1048E000C2F80834C2F80C3410BD00BF44360020B2
:1048F000C0970008000002400F28F8B510D9102812
:1049000010D0112811D0122808D10F240720DFF869
:10491000C8E00126DEF80050A04208D9002653E086
:104920000446F4E70F240020F1E70724FBE706FA2A
:1049300000F73D424AD1264C4FEA001C3D4304EBB0
:1049400000160EEBC000CEF80050C0E90123FBB208
:1049500073B12048D0F8D83043F00103C0F8D83004
:10496000D0F8003143F00103C0F80031D0F8003135
:1049700017F47F4F0ED01748D0F8D83043F0020319
:10498000C0F8D830D0F8003143F00203C0F800314D
:10499000D0F8003154F80C00036823F01F030360C3
:1049A000056815F00105FBD104EB0C033D2493F8D9
:1049B0000CC05F6804FA0CF43C602124056044617B
:1049C00012B1987B00F0CAFC3046F8BD0130A3E775
:1049D000C0970008004402584436002010B5302427
:1049E00084F31188FFF788FF002383F3118810BD3B
:1049F00010B50446807B00F0C7FC01231549627B9B
:104A000003FA02F20B6823EA0203DAB20B6072B90E
:104A1000114AD2F8D81021F00101C2F8D810D2F80A
:104A2000001121F00101C2F80011D2F8002113F4A5
:104A30007F4F0ED1084BD3F8D82022F00202C3F8E2
:104A4000D820D3F8002122F00202C3F80021D3F8C5
:104A5000003110BD443600200044025808B5302310
:104A600083F31188FFF7C4FF002383F3118808BD87
:104A7000836CC26A8B42506810B506D95A1E4C002E
:104A800002EB4103B3FBF4F3184410BD01F0010342
:104A90008A0748BF43F002034A0748BF43F00803B0
:104AA0000A0748BF43F00403CA0648BF43F0100397
:104AB0008A06426B48BF43F02003134343637047A9
:104AC00010B5074C204600F0CBFF064B0022C4E98E
:104AD0001023054BA364054BE363054BE36410BD52
:104AE000C83600200070005200B4C4041C370020F7
:104AF0001C390020C36A0BB9104BC3620379012B28
:104B000011D10F4B98420ED10E4BD3F8D42042F462
:104B10008032C3F8D420D3F8FC2042F48032C3F8AA
:104B2000FC20D3F8FC30436C00221A65DA621A606C
:104B30005A605A624FF0FF329A637047C09800087B
:104B4000C8360020004402580379012B1BD0436C67
:104B500000221A65DA621A605A605A624FF0FF3218
:104B60009A63094B98420ED1084BD3F8D42022F413
:104B70008032C3F8D420D3F8FC2022F48032C3F86A
:104B8000FC20D3F8FC307047C8360020004402589F
:104B900010B5446C0649FFF76BFF6060236842F272
:104BA000107043F003032360BDE8104001F05EBDC8
:104BB000801A06000129F8B5466C0B4F09D17568BB
:104BC0000A493D40FFF754FF054345F480557560A1
:104BD000F8BD746806493C40FFF74AFF044344F4BB
:104BE00080547460F4E700BF00ECFFFF80F0FA022D
:104BF00040787D01436C00225A601A6070470000C3
:104C0000426C0129536823F4404304D0022905D0A3
:104C100001B95360704743F48043FAE743F400431B
:104C2000F7E70000436C41F480519A60D9605A6BF9
:104C30001206FCD580229A637047000010B541F43B
:104C40008851446CA260E160616B11F04502FBD0B9
:104C5000A26311F0040203D0FFF718FF012010BD7A
:104C6000616910461960FAE710B541F48851446C47
:104C7000A260E160616B11F04502FBD0A26311F00C
:104C8000050203D0FFF702FF012010BD6169104645
:104C90001960FAE773B5134604460E46302282F3D4
:104CA0001188426CD26B32B14FF0FF31403001932A
:104CB00001F0E8FC019B606C00220265C263C262E5
:104CC000456B15F4807504D185F31188012002B07D
:104CD00070BD4FF0FF31816382F31188012E06D938
:104CE0000C21204602B0BDE87040FFF7BDBF104662
:104CF000EDE7000073B5446C0E4600250192616B30
:104D0000A1632565E562FFF7C1FE012E07D9019B6E
:104D10002A460C2102B0BDE87040FFF7A5BF02B0E3
:104D200070BD000010B541F49851446CA260E16080
:104D3000616B11F04502FBD0A26311F03F0203D07A
:104D4000FFF7A4FE012010BD216A10461960E16939
:104D50005960A16999606169D960F4E72DE9F74369
:104D600004460191006D01A91746984602F020FC07
:104D7000064600284AD0626C2046DDF8049055684B
:104D8000C5F3090501356B00A56CB5FBF3F54FF4D0
:104D90007A73B5FBF3F55D43556200F027FE50BB17
:104DA000636C4FF0FF3201254146C3F8589020460E
:104DB0001D659A634FF49572DA6342F207029F62AF
:104DC000DA62E36C0A9AFFF74FFFA0B9E26C104B6E
:104DD00011680B407BB929462046FFF75BFF05466B
:104DE00048B92E463A460199206D02F019FC30462A
:104DF00003B0BDE8F0833A460199206D02F010FC43
:104E0000E26C01212046FFF775FFF0E70126EEE78F
:104E100008E0FFFD2DE9F7431F46436C01924FF474
:104E20007A725D6804468846C5F3090501356E004F
:104E3000856CB5FBF6F5B5FBF2F555435D6200F008
:104E4000D5FD20B10125284603B0BDE8F0837E02E0
:104E500001A9206D324602F0ABFB05460028F1D0D7
:104E6000636C019AD4F84C909A6501221A654FF050
:104E7000FF329A634FF49572DA639E62236BDB060E
:104E80004B4658BF4FEA4828012F42461BD91221F2
:104E90002046FFF7E9FEC0B9D9F80020104B1340B7
:104EA0009BB9636C42F2930239462046DA62E26CA7
:104EB000FFF7F0FE804640B932460199206D454625
:104EC00002F0AEFBBFE71121E2E732460199206D07
:104ED00002F0A6FBE26C39462046FFF70BFFB2E773
:104EE00008E0FFFD2DE9F3411F46436C01924FF4AA
:104EF0007A725D6804468846C5F3090501356E007F
:104F0000856CB5FBF6F5B5FBF2F555435D6200F037
:104F10006DFD20B10125284602B0BDE8F0817E027A
:104F200001A9206D324602F089FB05460028F1D028
:104F3000636C019A9A6501221A654FF0FF329A63F9
:104F40004FF48D72DA639E62236BE66CDB063346A8
:104F500058BF4FEA4828012F424619D91921204647
:104F6000FFF782FEB0B932680F4B134093B9636C00
:104F700042F2910239462046DA62E26CFFF78AFE7D
:104F8000064638B901993546206D02F093FBC2E719
:104F90001821E4E70199206D02F08CFBE26C3946A0
:104FA0002046FFF7A7FEB6E708E0FFFD12F0030F6B
:104FB0002DE9F04107460C4615461E4617D00E4413
:104FC000B44202D10020BDE8F0810123FA6B2146F2
:104FD0003846FFF71FFF0028F5D128464FF400722E
:104FE000F96B05F500750134FCF780FEE8E7BDE8D4
:104FF000F041FFF70FBF000012F0030F2DE9F04161
:1050000007460C4615461E4617D00E44B44202D140
:105010000020BDE8F08129464FF40072F86B05F5D9
:105020000075FCF763FE0123FA6B21463846FFF753
:1050300059FF0028EDD10134E8E7BDE8F041FFF762
:1050400051BF000000207047302310B583F3118852
:105050000024436C40302146DC6301F021FB84F3E3
:10506000118810BD026843681143016003B11847FD
:1050700070470000024A136843F0C0031360704792
:1050800000440040024A136843F0C00313607047B5
:1050900000480040024A136843F0C00313607047A1
:1050A00000780040064BD3F8E8200243C3F8E8201C
:1050B000D3F810211043C3F81001D3F81031704712
:1050C0000044025837B5274C274D204600F028FDF4
:1050D00004F11400009400234FF40072234900F0FF
:1050E000C3F94FF40072224904F138000094214BB7
:1050F00000F03CFA204BC4E91735204C204600F064
:105100000FFD04F11400009400234FF400721C49B9
:1051100000F0AAF94FF400721A4904F13800009423
:10512000194B00F023FA194BC4E91735184C2046E7
:1051300000F0F6FC04F1140000234FF4007215494E
:10514000009400F091F9144B4FF40072134904F1EC
:105150003800009400F00AFA114BC4E9173503B087
:1051600030BD00BF2039002000E1F505643A002081
:105170006440002075500008004400408C39002035
:10518000643C002064420020855000080048004034
:10519000F8390020643E0020955000086444002047
:1051A0000078004038B5264D0446037C002918BF1E
:1051B0000D46012B06D1234B984230D14FF40030DD
:1051C000FFF770FF2A68236EE16D03EB5203A566BB
:1051D000B3FBF2F36A68100442BF23F0070003F048
:1051E000070343EA4003CB60AB6843F040034B60E6
:1051F000EB6843F001038B6042F4967343F00103C4
:105200000B604FF0FF330B62510505D512F01022F1
:1052100011D0B2F1805F10D084F8643038BD0A4BF1
:10522000984205D0094B9842CCD14FF08040C7E757
:105230004FF48020C4E77F23EEE73F23ECE700BF75
:10524000C8980008203900208C390020F839002047
:105250002DE9F047C66D05463768F46921073462C9
:105260001AD014F0080118BF4FF48071E20748BF4C
:1052700041F02001A3074FF0300348BF41F0400147
:10528000600748BF41F0800183F31188281DFFF7B4
:10529000E9FE002383F31188E2050AD5302383F366
:1052A00011884FF48061281DFFF7DCFE002383F393
:1052B00011884FF030094FF0000A14F0200838D15F
:1052C0003B0616D54FF0300905F1380A200610D5F7
:1052D00089F31188504600F07DF9002836DA08215C
:1052E000281DFFF7BFFE27F080033360002383F300
:1052F0001188790614D5620612D5302383F31188FC
:10530000D5E913239A4208D12B6C33B127F040071B
:105310001021281DFFF7A6FE3760002383F31188B4
:10532000E30618D5AA6E1369ABB15069BDE8F04722
:10533000184789F31188736A284695F86410194054
:1053400000F008FC8AF31188F469B6E7B06288F3CC
:105350001188F469BAE7BDE8F0870000090100F19F
:105360006043012203F56143C9B283F8001300F0E2
:105370001F039A4043099B0003F1604303F5614317
:10538000C3F880211A60704700F01F0301229A4081
:10539000430900F160409B0000F5614003F1604368
:1053A00003F56143C3F88020C3F88021002380F80F
:1053B00000337047F8B51546826804460B46AA428A
:1053C00000D28568A1692669761AB5420BD21846C3
:1053D0002A46FCF78BFCA3692B44A3612846A368EB
:1053E0005B1BA360F8BD0CD9AF1B18463246FCF717
:1053F0007DFC3A46E1683044FCF778FCE3683B44C6
:10540000EBE718462A46FCF771FCE368E5E7000085
:1054100083689342F7B50446154600D28568D4E9FF
:105420000460361AB5420BD22A46FCF75FFC63696A
:105430002B4463612846A3685B1BA36003B0F0BDE7
:105440000DD93246AF1B0191FCF750FC01993A4649
:10545000E0683144FCF74AFCE3683B44E9E72A464C
:10546000FCF744FCE368E4E710B50A440024C36198
:10547000029B8460C16002610362C0E90000C0E970
:10548000051110BD08B5D0E90532934201D18268FB
:1054900082B98268013282605A1C4261197000210F
:1054A000D0E904329A4224BFC368436101F012F983
:1054B000002008BD4FF0FF30FBE7000070B530233F
:1054C00004460E4683F31188A568A5B1A368A269B6
:1054D000013BA360531CA36115782269934224BF4A
:1054E000E368A361E3690BB120469847002383F387
:1054F0001188284607E03146204601F0DBF80028F5
:10550000E2DA85F3118870BD2DE9F74F04460E46A7
:1055100017469846D0F81C904FF0300A8AF311884D
:105520004FF0000B154665B12A4631462046FFF77D
:1055300041FF034660B94146204601F0BBF8002810
:10554000F1D0002383F31188781B03B0BDE8F08FFE
:10555000B9F1000F03D001902046C847019B8BF39F
:105560001188ED1A1E448AF31188DCE7C160C3611B
:10557000009B82600362C0E905111144C0E900008C
:1055800001617047F8B504460D461646302383F393
:105590001188A768A7B1A368013BA36063695A1C7F
:1055A00062611D70D4E904329A4224BFE3686361EA
:1055B000E3690BB120469847002080F3118807E08B
:1055C0003146204601F076F80028E2DA87F31188A8
:1055D000F8BD0000D0E9052310B59A4201D18268D8
:1055E0007AB982680021013282605A1C82611C787B
:1055F00003699A4224BFC368836101F06BF82046B7
:1056000010BD4FF0FF30FBE72DE9F74F04460E4683
:1056100017469846D0F81C904FF0300A8AF311884C
:105620004FF0000B154665B12A4631462046FFF77C
:10563000EFFE034660B94146204601F03BF80028E2
:10564000F1D0002383F31188781B03B0BDE8F08FFD
:10565000B9F1000F03D001902046C847019B8BF39E
:105660001188ED1A1E448AF31188DCE70379052BB3
:1056700005BF836A002001204B6004BF4FF4007314
:105680000B60704770B55D1E866A04460D44B542D6
:1056900005D9436B43F080034363012070BD0625A9
:1056A0000571FFF783FC05232371F7E770B55D1ED5
:1056B000866A04460D44B54205D9436B43F0800326
:1056C0004363012070BD07250571FFF795FC052395
:1056D0002371F7E738B505790446052D05D1082370
:1056E0000371FFF7AFFC257138BD0120FCE7000016
:1056F0000323F0B5037185B00446FFF749FA002291
:1057000020461146FFF78EFA4FF4D57203AB0821FD
:105710002046FFF7A9FA0246B8B901232363039B89
:10572000C3F30323012B09D103AB37212046FFF735
:105730009BFA18B9A44B039A1340ABB1204601253C
:10574000FFF758FA0223237137E103AB0022372118
:105750002046FFF789FA28B99B4A039B1A40002A82
:1057600000F0A78002232363236B03F00F03022BB7
:1057700040F0A9806425954E42F2107000F076FF4B
:1057800003AB324601212046FFF758FA0028D5D155
:10579000039B002B80F293805A0003D5236B43F0C8
:1057A00010032363002204F1080302212046FFF7BF
:1057B000B9FA02460028C1D104F13803032120467A
:1057C000FFF752FA0028B9D104F11805A26B09219C
:1057D00020462B46FFF7A6FA0028AFD102ABA26BFA
:1057E00007212046FFF740FA06460028A6D1236B82
:1057F00003F00F03022B40F08F807E227F2128468A
:1058000003F01CFA012840F28780E76B42F2107027
:1058100000F02CFF08234FF4007239462046009612
:10582000FFF79CFA002889D1384603F055FA236B1C
:10583000A06203F00F03022B72D103AB644A06216E
:105840002046FFF711FA002871D15F49039B1940E8
:10585000B1FA81F149092046FFF7ACF902AB4FF4E8
:10586000007210212046FFF7FFF9054600287FF45B
:1058700065AF554E029B33427FF460AF236B13F04C
:105880000E0F03F00F0273D0022A7FF457AFE36AC2
:105890001978012900F09480022900F093800029F2
:1058A00000F089804B4F2046FFF7AAF903AB3A4638
:1058B00076E0114620462263FFF7B4F954E7013D34
:1058C0007FF45AAF3AE7444D6426444A3E4F012BD9
:1058D00018BF154603AB002237212046FFF7C4F955
:1058E00000287FF42BAF039B3B427FF427AF03AB31
:1058F0002A4629212046FFF7A1F900287FF41EAF90
:10590000039B002BFFF648AF013E3FF417AF42F276
:10591000107000F0ABFEDDE7284603F0B1F986E732
:105920007E227F212846E66B03F088F908B9002122
:1059300091E7002340223146204600930623FFF7DB
:105940000DFA0028F3D1B3895BBA9B07EFD5244B3E
:1059500040223146204600930623FFF7FFF9002836
:10596000E5D1317C01F00F010F3918BF012172E739
:10597000E36A1978F9B101297FF4E0AE2046FFF718
:105980003FF903ABA26B37212046FFF76DF90028E2
:105990007FF4D4AE039B33427FF4D0AE03AB02223C
:1059A00006212046FFF760F900287FF4C7AE039B6D
:1059B00033427FF4C3AE05232371284605B0F0BD02
:1059C000084F70E7084F6EE708E0FFFD0080FFC05A
:1059D0000001B9030000B7030080FF5000001080F1
:1059E000F1FFFF800001B7030002B70337B504469B
:1059F0000C4D01ABA26B0D212046FFF735F978B9AC
:105A0000019B2B420BD1C3F34323042B08D0053B4E
:105A1000022B04D84FF47A7000F028FEE9E7012049
:105A200003B030BD08E0FFFD70B53023054683F3B9
:105A3000118803790024022B03D184F311882046B6
:105A400070BD0423037184F311880226FFF7CEFF93
:105A500004462846FFF7CEF82E71F0E7FFF730B87E
:105A6000044B03600123037100234363C0E90A333D
:105A7000704700BFE098000810B53023044683F358
:105A80001188C162FFF736F802230020237180F3EA
:105A9000118810BD10B53023044683F31188FFF739
:105AA00053F800230122E362227183F3118810BDB1
:105AB000026843681143016003B118477047000052
:105AC0001430FFF721BD00004FF0FF331430FFF713
:105AD0001BBD00003830FFF797BD00004FF0FF33CB
:105AE0003830FFF791BD00001430FFF7E7BC00002D
:105AF0004FF0FF311430FFF7E1BC00003830FFF702
:105B000041BD00004FF0FF323830FFF73BBD0000D1
:105B1000012914BF6FF0130000207047FFF7D2BABD
:105B2000044B036000234360C0E902330123037484
:105B3000704700BF0499000810B53023044683F372
:105B40001188FFF72FFB02230020237480F31188B4
:105B500010BD000038B5C36904460D461BB90421C9
:105B60000844FFF7A5FF294604F11400FFF78AFC5B
:105B7000002806DA201D4FF40061BDE83840FFF729
:105B800097BF38BD026843681143016003B11847ED
:105B90007047000013B5406B00F58054D4F8A4386A
:105BA0001A681178042914D1017C022911D11979BC
:105BB000012312898B4013420BD101A94C3002F012
:105BC0006BFFD4F8A4480246019B2179206800F0BD
:105BD000DFF902B010BD0000143002F0EDBE00008D
:105BE0004FF0FF33143002F0E7BE00004C3002F0FB
:105BF000BFBF00004FF0FF334C3002F0B9BF0000D0
:105C0000143002F0BBBE00004FF0FF31143002F040
:105C1000B5BE00004C3002F08BBF00004FF0FF32E9
:105C20004C3002F085BF00000020704710B500F531
:105C30008054D4F8A4381A681178042917D1017C4B
:105C4000022914D15979012352898B4013420ED174
:105C5000143002F04DFE024648B1D4F8A4484FF487
:105C6000407361792068BDE8104000F07FB910BD35
:105C7000406BFFF7DBBF0000704700007FB5124BA1
:105C800001250426044603600023057400F1840204
:105C900043602946C0E902330C4B02901430019353
:105CA0004FF44073009602F0FFFD094B04F6944256
:105CB000294604F14C000294CDE900634FF440738F
:105CC00002F0C6FE04B070BD2C990008715C00089B
:105CD000955B00080A68302383F311880B790B3336
:105CE00042F823004B79133342F823008B7913B128
:105CF0000B3342F8230000F58053C3F8A4180223A5
:105D00000374002080F311887047000038B5037FCA
:105D1000044613B190F85430ABB90125201D02217F
:105D2000FFF730FF04F114006FF00101257700F058
:105D3000DDFC04F14C0084F854506FF00101BDE823
:105D4000384000F0D3BC38BD10B501210446043002
:105D5000FFF718FF0023237784F8543010BD0000AC
:105D600038B504460025143002F0B6FD04F14C00AD
:105D7000257702F085FE201D84F854500121FFF79D
:105D800001FF2046BDE83840FFF750BF90F8803053
:105D900003F06003202B06D190F881200023212AF4
:105DA00003D81F2A06D800207047222AFBD1C0E959
:105DB0001D3303E0034A426707228267C36701205D
:105DC000704700BF4422002037B500F58055D5F854
:105DD000A4381A68117804291AD1017C022917D134
:105DE0001979012312898B40134211D100F14C041F
:105DF000204602F005FF58B101A9204602F04CFEF2
:105E0000D5F8A4480246019B2179206800F0C0F82B
:105E100003B030BD01F10B03F0B550F8236085B03D
:105E200004460D46FEB1302383F3118804EB850749
:105E3000301D0821FFF7A6FEFB6806F14C005B69E8
:105E40001B681BB1019002F035FE019803A902F016
:105E500023FE024648B1039B2946204600F098F8ED
:105E6000002383F3118805B0F0BDFB685A691268FE
:105E7000002AF5D01B8A013B1340F1D104F18002C6
:105E8000EAE70000133138B550F82140ECB1302377
:105E900083F3118804F58053D3F8A428136852794A
:105EA00003EB8203DB689B695D6845B104216018E0
:105EB000FFF768FE294604F1140002F023FD204696
:105EC000FFF7B4FE002383F3118838BD704700004C
:105ED00001F044BD01234022002110B5044600F822
:105EE000303BFBF729FF0023C4E9013310BD00005C
:105EF00010B53023044683F3118824224160002129
:105F00000C30FBF719FF204601F04AFD0223002068
:105F1000237080F3118810BD70B500EB8103054636
:105F200050690E461446DA6018B110220021FBF7C2
:105F300003FFA06918B110220021FBF7FDFE3146D6
:105F40002846BDE8704001F031BE00008368202281
:105F5000002103F0011310B5044683601030FBF7F5
:105F6000EBFE2046BDE8104001F0ACBEF0B40125C8
:105F700000EB810447898D40E4683D43A469458175
:105F800023600023A2606360F0BC01F0C9BE000082
:105F9000F0B4012500EB810407898D40E4683D439E
:105FA0006469058123600023A2606360F0BC01F096
:105FB0003FBF000070B50223002504462422037071
:105FC0002946C0F888500C3040F8045CFBF7B4FE5A
:105FD000204684F8705001F07DFD63681B6823B192
:105FE00029462046BDE87040184770BD0378052B50
:105FF00010B504460AD080F88C300523037043683E
:106000001B680BB1042198470023A36010BD00005A
:106010000178052906D190F88C20436802701B682E
:1060200003B118477047000070B590F8703004460F
:1060300013B1002380F8703004F18002204601F093
:1060400065FE63689B68B3B994F8803013F060050F
:1060500035D00021204602F057F90021204602F0F9
:1060600047F963681B6813B1062120469847062349
:1060700084F8703070BD204698470028E4D0B4F80A
:106080008630A26F9A4288BFA36794F98030A56FCB
:10609000002B4FF0300380F20381002D00F0F280DE
:1060A000092284F8702083F3118800212046D4E966
:1060B0001D23FFF76DFF002383F31188DAE794F8BF
:1060C000812003F07F0343EA022340F2023293422D
:1060D00000F0C58021D8B3F5807F48D00DD8012BC2
:1060E0003FD0022B00F09380002BB2D104F1880244
:1060F00062670222A267E367C1E7B3F5817F00F020
:106100009B80B3F5407FA4D194F88230012BA0D1BD
:10611000B4F8883043F0020332E0B3F5006F4DD09D
:1061200017D8B3F5A06F31D0A3F5C063012B90D879
:106130006368204694F882205E6894F88310B4F86F
:106140008430B047002884D0436863670368A3673E
:106150001AE0B3F5106F36D040F6024293427FF456
:1061600078AF5C4B63670223A3670023C3E794F80F
:106170008230012B7FF46DAFB4F8883023F0020336
:10618000A4F88830C4E91D55E56778E7B4F8803095
:10619000B3F5A06F0ED194F88230204684F88A308F
:1061A00001F0F6FC63681B6813B101212046984793
:1061B000032323700023C4E91D339CE704F18B0300
:1061C00063670123C3E72378042B10D1302383F3C3
:1061D00011882046FFF7BAFE85F311880321636812
:1061E00084F88B5021701B680BB12046984794F8B7
:1061F0008230002BDED084F88B3004232370636858
:106200001B68002BD6D0022120469847D2E794F88D
:10621000843020461D0603F00F010AD501F068FD09
:10622000012804D002287FF414AF2B4B9AE72B4BA4
:1062300098E701F04FFDF3E794F88230002B7FF4EC
:1062400008AF94F8843013F00F01B3D01A0620463B
:1062500002D502F071F8ADE702F062F8AAE794F80F
:106260008230002B7FF4F5AE94F8843013F00F01E8
:10627000A0D01B06204602D502F046F89AE702F0AD
:1062800037F897E7142284F8702083F311882B469F
:106290002A4629462046FFF769FE85F31188E9E67C
:1062A0005DB1152284F8702083F311880021204607
:1062B000D4E91D23FFF75AFEFDE60B2284F8702077
:1062C00083F311882B462A4629462046FFF760FEB5
:1062D000E3E700BF5C99000854990008589900084A
:1062E00038B590F870300446002B3ED0063BDAB249
:1062F0000F2A34D80F2B32D8DFE803F037313108BA
:10630000223231313131313131313737856FB0F8A7
:1063100086309D4214D2C3681B8AB5FBF3F203FB9F
:1063200012556DB9302383F311882B462A4629462E
:10633000FFF72EFE85F311880A2384F870300EE0F3
:10634000142384F87030302383F31188002320460F
:106350001A461946FFF70AFE002383F3118838BD59
:10636000C36F03B198470023E7E70021204601F0FF
:10637000CBFF0021204601F0BBFF63681B6813B10F
:106380000621204698470623D7E7000010B590F86D
:1063900070300446142B29D017D8062B05D001D80D
:1063A0001BB110BD093B022BFBD80021204601F098
:1063B000ABFF0021204601F09BFF63681B6813B10F
:1063C000062120469847062319E0152BE9D10B2317
:1063D00080F87030302383F3118800231A46194661
:1063E000FFF7D6FD002383F31188DAE7C3689B69C2
:1063F0005B68002BD5D1C36F03B19847002384F8A5
:106400007030CEE70023826880F8243083691B68EF
:1064100099689142FBD25A680360426010605860EC
:10642000704700000023826880F8243083691B686D
:1064300099689142FBD85A680360426010605860C6
:106440007047000008B50846302383F3118891F89F
:106450002430032B05D0042B0DD02BB983F31188E6
:1064600008BD8B6A00221A604FF0FF338362FFF78A
:10647000C9FF0023F2E7D1E9003213605A60F3E765
:10648000034610B51B68984203D09C688A68944202
:10649000F8D25A680B604A601160596010BD000064
:1064A000FFF7B0BF064BD96881F82400186802686E
:1064B00053601A600122D86080F82420F9F7A2BF47
:1064C000684600200C4B30B5DD684B1C87B0044695
:1064D0000FD02B46094A684600F09CF92046FFF78A
:1064E000E1FF009B13B1684600F09EF9A86A07B06F
:1064F00030BDFFF7D7FFF9E7684600204564000884
:10650000044B1A68DB6890689B68984294BF00202F
:106510000120704768460020094B10B51C68D868F8
:10652000226853601A600122DC6084F82420FFF79F
:1065300079FF01462046BDE81040F9F763BF00BF70
:1065400068460020044B1A68DB6892689B689A4290
:1065500001D9FFF7E1BF70476846002038B5012335
:10656000084C00252370656002F0E4FB02F00AFC91
:106570000549064802F0E0FC0223237085F31188E8
:1065800038BD00BF1049002064990008684600200B
:1065900000F080B9034A516853685B1A9842FBD8EF
:1065A000704700BF001000E08B604B630023CA619E
:1065B00000F128020B6302230A618B8401238861A6
:1065C00081F8263001F11003C26A4A611360C36288
:1065D00001F12C030846CB6270470000D0E901317D
:1065E000026841F8183CA1F19C033839CB6003697B
:1065F00041F8243C436941F8203C034B41F8043CFA
:10660000C3680248FFF7D0BF1D0400086846002099
:1066100008B5FFF7E3FFBDE80840FFF741BF000002
:1066200038B50E4BDC6804F12C05A062E06AA84284
:106630000FD194F826303BB994F825309B0702BF60
:10664000D4E9043213605A600F20BDE83840FFF7E8
:1066500029BF0368E362FFF723FFE7E768460020EE
:10666000302383F31188FFF7DBBF000008B5014634
:10667000302383F311880820FFF724FF002383F3DE
:10668000118808BD054BDB6821B1036098620320C7
:10669000FFF718BF4FF0FF30704700BF684600207B
:1066A00003682BB10022026018469962FFF7F8BE1A
:1066B00070470000064BDB6839B1426818605A60C9
:1066C000136043600420FFF7FDBE4FF0FF307047BA
:1066D000684600200368984206D01A68026050603D
:1066E00018469962FFF7DCBE7047000038B50446D3
:1066F0000D462068844200D138BD036823605C6089
:106700008562FFF7CDFEF4E7036810B59C68A242EE
:106710000CD85C688A600B604C6021605960996895
:106720008A1A9A604FF0FF33836010BD121B1B68FA
:10673000ECE700000A2938BF0A2170B504460D466F
:106740000A26601902F0F0FA02F0D8FA041BA542FA
:1067500003D8751C04462E46F3E70A2E04D90120FF
:10676000BDE8704002F0B0BC70BD0000F8B5144B3D
:106770000D460A2A4FF00A07D96103F11001826021
:1067800038BF0A22416019691446016048601861E7
:10679000A81802F0B9FA02F0B1FA431B0646A34268
:1067A00006D37C1C28192746354602F0BDFAF2E7CD
:1067B0000A2F04D90120BDE8F84002F085BCF8BDDD
:1067C00068460020F8B506460D4602F097FA0F4AD3
:1067D000134653F8107F9F4206D12A4601463046A1
:1067E000BDE8F840FFF7C2BFD169BB68441A2C1955
:1067F00028BF2C46A34202D92946FFF79BFF224619
:1068000031460348BDE8F840FFF77EBF68460020E8
:1068100078460020C0E90323002310B45DF8044B40
:106820004361FFF7CFBF000010B5194C23699842B0
:106830000DD08168D0E9003213605A609A680A442A
:106840009A60002303604FF0FF33A36110BD02681C
:10685000234643F8102F53600022026022699A42B7
:1068600003D1BDE8104002F059BA936881680B4427
:10687000936002F043FA2269E1699268441AA242E5
:10688000E4D91144BDE81040091AFFF753BF00BF17
:10689000684600202DE9F047DFF8BC8008F11007BA
:1068A0002C4ED8F8105002F029FAD8F81C40AA68EB
:1068B000031B9A423ED814444FF00009D5E9003238
:1068C000C8F81C4013605A60C5F80090D8F8103022
:1068D000B34201D102F022FA89F31188D5E90331DC
:1068E00028469847302383F311886B69002BD8D052
:1068F00002F004FA6A69A0EB040982464A450DD207
:10690000022002F0E1FB0022D8F81030B34208D197
:1069100051462846BDE8F047FFF728BF121A224427
:10692000F2E712EB09092946384638BF4A46FFF715
:10693000EBFEB5E7D8F81030B34208D01444C8F8DD
:106940001C00211AA960BDE8F047FFF7F3BEBDE8BF
:10695000F08700BF784600206846002038B502F076
:10696000CDF9054AD2E90845031B181945F1000184
:10697000C2E9080138BD00BF6846002010B560B903
:10698000074804790368053C9B6818BF01249847B1
:1069900008B144F00404204610BD0124FBE700BF09
:1069A000C8360020FFF7EABF2DE9F04788461746B2
:1069B0009A460446B0B90D4E3579052D05D003240D
:1069C0000DE0013D15F0FF050ED032685346394603
:1069D0003046D2F814904246C8470028F1D12046EC
:1069E000BDE8F0870424FAE70124F8E7C836002060
:1069F0002DE9F047884617469A460446B0B90D4E31
:106A00003579052D05D003240DE0013D15F0FF0576
:106A10000ED03268534639463046D2F81890424676
:106A2000C8470028F1D12046BDE8F0870424FAE7E2
:106A30000124F8E7C836002037B50C46154670B972
:106A400051B101290BD10748694603681B6A984771
:106A500010B9019B04462B60204603B030BD0424CE
:106A6000FAE700BFC836002000207047FEE70000AC
:106A7000704700004FF0FF30704700004B684360E4
:106A80008B688360CB68C3600B6943614B690362A9
:106A90008B6943620B6803607047000008B53C4B8C
:106AA00040F2FF713B48D3F888200A43C3F888209E
:106AB000D3F8882022F4FF6222F00702C3F888206E
:106AC000D3F88820D3F8E0200A43C3F8E020D3F8B5
:106AD00008210A43C3F808212F4AD3F80831114688
:106AE000FFF7CCFF00F5806002F11C01FFF7C6FF45
:106AF00000F5806002F13801FFF7C0FF00F580600B
:106B000002F15401FFF7BAFF00F5806002F1700155
:106B1000FFF7B4FF00F5806002F18C01FFF7AEFFD4
:106B200000F5806002F1A801FFF7A8FF00F5806082
:106B300002F1C401FFF7A2FF00F5806002F1E0015D
:106B4000FFF79CFF00F5806002F1FC01FFF796FF64
:106B500002F58C7100F58060FFF790FF01F084FC76
:106B60000E4BD3F8902242F00102C3F89022D3F8E2
:106B7000942242F00102C3F894220522C3F898201F
:106B80004FF06052C3F89C20054AC3F8A02008BD0E
:106B900000440258000002587899000800ED00E017
:106BA0001F00080308B501F06BFEFFF7D7FC104B80
:106BB000D3F8DC2042F04002C3F8DC20D3F80421F3
:106BC00022F04002C3F80421D3F80431094B1A68BB
:106BD00042F008021A601A6842F004021A6000F0DB
:106BE00071FD00F035FBBDE8084000F0B5B800BF0E
:106BF00000440258001802480120704700207047E6
:106C00007047000002290CD0032904D0012907484D
:106C100018BF00207047032A05D8054800EBC200C2
:106C20007047044870470020704700BF7C9B0008F5
:106C300054220020309B000870B59AB005460846E3
:106C4000144601A900F0C2F801A8FBF76DF8431C37
:106C50000022C6B25B001046C5E90034237003234E
:106C6000023404F8013C01ABD1B202348E4201D8A7
:106C70001AB070BD13F8011B013204F8010C04F8BE
:106C8000021CF1E708B5302383F311880348FFF7AE
:106C90009BF8002383F3118808BD00BF184900202A
:106CA00090F8803003F01F02012A07D190F881206C
:106CB0000B2A03D10023C0E91D3315E003F0600364
:106CC000202B08D1B0F884302BB990F88120212AEC
:106CD00003D81F2A04D8FFF759B8222AEBD0FAE7C5
:106CE000034A426707228267C3670120704700BFDB
:106CF0004B22002007B5052917D8DFE801F0191647
:106D000003191920302383F31188104A01210190BF
:106D1000FFF702F9019802210D4AFFF7FDF80D482F
:106D2000FFF71EF8002383F3118803B05DF804FB1E
:106D3000302383F311880748FEF7E8FFF2E730239A
:106D400083F311880348FEF7FFFFEBE7D09A0008B2
:106D5000F49A00081849002038B50C4D0C4C2A460E
:106D60000C4904F10800FFF767FF05F1CA0204F1BE
:106D700010000949FFF760FF05F5CA7204F1180019
:106D80000649BDE83840FFF757BF00BFF06100205B
:106D900054220020AC9A0008B99A0008C49A00084E
:106DA00070B5044608460D46FAF7BEFFC6B2204647
:106DB000013403780BB9184670BD32462946FAF7FC
:106DC0009FFF0028F3D10120F6E700002DE9F84FDE
:106DD00005460C46FAF7A8FF2C49C6B22846FFF72D
:106DE000DFFF08B10336F6B229492846FFF7D8FF7E
:106DF00008B11036F6B2632E0DD8DFF89080DFF8B8
:106E00009090244FDFF894A0DFF894B02E7846B924
:106E10002670BDE8F88F29462046BDE8F84F02F0FD
:106E2000FDB9252E2ED1072241462846FAF768FFE4
:106E300070B9DBF8003007350A3444F80A3CDBF857
:106E4000043044F8063CBBF8083024F8023CDDE787
:106E5000082249462846FAF753FF98B9A21C0E4B60
:106E6000197802320909C95D02F8041C13F8011BE4
:106E700001F00F015345C95D02F8031CF0D118342D
:106E80000835C3E7013504F8016BBFE79C9B000898
:106E9000C49A0008AF9B000800E8F11F0CE8F11F3E
:106EA000A49B0008BFF34F8F044B1A695107FCD114
:106EB000D3F810215207F8D1704700BF00200052CC
:106EC00008B50D4B1B78ABB9FFF7ECFF0B4BDA683D
:106ED000D10704D50A4A5A6002F188325A60D3F8C1
:106EE0000C21D20706D5064AC3F8042102F18832E4
:106EF000C3F8042108BD00BF4E64002000200052EA
:106F00002301674508B5114B1B78F3B9104B1A697B
:106F1000510703D5DA6842F04002DA60D3F8102155
:106F2000520705D5D3F80C2142F04002C3F80C21DA
:106F3000FFF7B8FF064BDA6842F00102DA60D3F8D7
:106F40000C2142F00102C3F80C2108BD4E64002060
:106F5000002000520F289ABF00F5806040040020F6
:106F6000704700004FF40030704700001020704759
:106F70000F2808B50BD8FFF7EDFF00F500330268C6
:106F8000013204D104308342F9D1012008BD002030
:106F9000FCE700000F2838B505463FD8FFF782FF11
:106FA0001F4CFFF78DFF4FF0FF3307286361C4F8D4
:106FB00014311DD82361FFF775FF030243F024034A
:106FC000E360E36843F08003E36023695A07FCD47D
:106FD0002846FFF767FFFFF7BDFF4FF4003100F0D1
:106FE000ABFA2846FFF78EFFBDE83840FFF7C0BF79
:106FF000C4F81031FFF756FFA0F108031B0243F05D
:107000002403C4F80C31D4F80C3143F08003C4F8E5
:107010000C31D4F810315B07FBD4D9E7002038BD20
:10702000002000522DE9F84F05460C46104645EA6F
:107030000203DE0602D00020BDE8F88F20F01F001A
:10704000DFF8BCB0DFF8BCA0FFF73AFF04EB0008A4
:10705000444503D10120FFF755FFEDE720222946E3
:10706000204602F0A3F810B920352034F0E72B4673
:1070700005F120021F68791CDDD104339A42F9D151
:1070800005F178431B481C4EB3F5801F1B4B38BFDE
:10709000184603F1F80332BFD946D1461E46FFF722
:1070A00001FF0760A5EB040C336804F11C0143F0F9
:1070B00002033360231FD9F8007017F00507FAD1D7
:1070C00053F8042F8B424CF80320F4D1BFF34F8FB9
:1070D000FFF7E8FE4FF0FF332022214603602846E9
:1070E000336823F00203336002F060F80028BBD05D
:1070F0003846B0E7142100520C20005214200052F0
:10710000102000521021005210B5084C237828B1ED
:107110001BB9FFF7D5FE0123237010BD002BFCD057
:107120002070BDE81040FFF7EDBE00BF4E640020A8
:107130002DE9F04F0D4685B0814658B111F00D068E
:1071400014BF2022082211F00803019304D0431E2B
:10715000034269D0002435E0002E37D009F11F0129
:1071600021F01F094FF00108314F05F00403DFF84B
:10717000CCA005EA080BBBF1000F32D07869C0073C
:107180002FD408F101080C37B8F1060FF3D19EB9DE
:10719000284D4946A819019201F016FE0446002820
:1071A00039D12036019AA02EF3D1494601F00CFEC8
:1071B000044600282FD1019A49461F4801F004FED9
:1071C000044660BB204605B0BDE8F08F0029C9D158
:1071D00001462846029201F0F7FD0446D8B9029A0A
:1071E000C0E713B178694107CBD5AC0702D5786900
:1071F0008007C6D5019911B178690107C1D5494603
:107200000AEB4810CDE9022301F0DEFD0446DDE97A
:1072100002230028B5D04A460021204601E04A4614
:107220000021FAF789FDCDE70246002E96D199E7B5
:10723000C09B00089064002050640020706400200F
:107240000021FFF775BF00000121FFF771BF0000AB
:1072500070B5144D0124144E40F2FF32002101207C
:10726000FAF76AFD06EB441001342A6955F80C1F41
:1072700001F096FD062CF5D137254FF4C054204679
:10728000FFF7E2FF014628B122460848BDE87040FA
:1072900001F086BDC4EBC404013D4FEAD404EED135
:1072A00070BD00BFC09B00087064002050640020C7
:1072B0000421FFF73DBF00004843FFF7C1BF0000B6
:1072C00008B101F0F3BD7047B0F5805F10B504461A
:1072D00007D8FFF7EDFF28B92046BDE81040FFF7BB
:1072E000AFBF002010BD0000FFF7EABF70B5AAB124
:1072F00040EA010313F01F030FD1094C0144A568B4
:107300006D0706D52568A84203D366683544A942AF
:1073100004D903330C34122BF1D10022104670BD76
:10732000C09B000808B501F0D7FE034AD2E900323D
:10733000C01842EB010108BD30650020434BD3E982
:1073400000232DE9F34113437CD0FFF7EBFF404AC4
:1073500000230027F9F770F806460D463D4A002342
:10736000F9F76AF80023144630462946394AF9F7F6
:1073700063F84FF461613C23ADF80170B4FBF1F5A3
:10738000B4FBF3F601FB154103FB16464624B1FBA3
:10739000F3F1314BF6B28DF8004098423CD84FF0F3
:1073A000640C4FF4C87EA30704F26C7225D1B2FBC3
:1073B000FCF30CFB132313BBB2FBFEF30EFB1322F7
:1073C000B2FA82F35B0903F26D18621C8045D2B2F7
:1073D00017D90FB18DF800400022204C4FF00C0C53
:1073E00017460CFB0343D4B2013213F804C08445A2
:1073F0000CD8A0EB0C000127F5E70023E3E70123FD
:10740000E1E7A0EB080014460127CCE70FB18DF8A7
:107410000140431C8DF802309DF80100431C9DF88B
:1074200000005038400640EA43509DF8023040EAE0
:10743000034040EA560040EAC52040EA411002B04D
:10744000BDE8F0814FF40410F9E700BF306500207B
:1074500040420F008051010090230B00089C00085F
:107460000244074BD2B210B5904200D110BD441C6B
:1074700000B253F8200041F8040BE0B2F4E700BF7B
:10748000504000580E4B30B51C6F240405D41C6FBF
:107490001C671C6F44F400441C670A4C02442368B8
:1074A000D2B243F480732360074B904200D130BDC9
:1074B000441C51F8045B00B243F82050E0B2F4E7FA
:1074C00000440258004802585040005807B50122B5
:1074D00001A90020FFF7C4FF019803B05DF804FB89
:1074E00013B50446FFF7F2FFA04205D0012201A91F
:1074F00000200194FFF7C6FF02B010BD10B5642450
:10750000013C4FF47A70FFF7B1F814F0FF04F7D1A3
:10751000084B4FF0807214249A6103F580530822BF
:107520009A61013C4FF47A70FFF7A0F814F0FF0461
:10753000F7D110BD000002580144BFF34F8F064B36
:10754000884204D3BFF34F8FBFF36F8F7047C3F8E8
:107550005C022030F4E700BF00ED00E00144BFF31F
:107560004F8F064B884204D3BFF34F8FBFF36F8F0B
:107570007047C3F870022030F4E700BF00ED00E070
:1075800070B5054616460C4601201021FFF794FE03
:10759000286046733CB1204636B1FFF789FE2B6860
:1075A000186000B19C6070BDFFF74EFEF7E7000069
:1075B000F8B50F461546044648B905F11F010126E6
:1075C000386821F01F01FFF7B7FF3046F8BD427B56
:1075D00029463868FFF78AFE06460028EDD13B6849
:1075E0006360A368AB4210D213B12068FFF768FE56
:1075F000637B28462BB1FFF75BFE206020B9A060BB
:10760000E3E7FFF721FEF8E7A560206805F11F0119
:10761000012621F01F013860FFF78EFF2673D4E7A3
:1076200010B5044640B10068884205D1606808B1D1
:10763000FAF75CFB0023237310BD0000F8B50F467A
:107640001446054648B904F11F010126386821F0A7
:107650001F01FFF783FF3046F8BD427B21463868A3
:10766000FFF744FE06460028EDD1AB68A34210D2D6
:1076700013B12868FFF724FE6B7B20462BB1FFF780
:1076800017FE286020B9A860E5E7FFF7DDFDF8E701
:10769000AC60396819B122462868FAF727FB2868D8
:1076A00004F11F01012621F01F013860FFF756FF8A
:1076B0002E73D0E720B103688B4204BF002303730D
:1076C00070470000034B1A681AB9034AD2F8D02455
:1076D0001A607047386500200040025808B5FFF76F
:1076E000F1FF024B1868C0F3806008BD38650020C8
:1076F000EFF30983054968334A6B22F001024A63BC
:1077000083F30988002383F31188704700EF00E0BA
:10771000302080F3118862B60D4B0E4AD96821F4EF
:10772000E0610904090C0A430B49DA60D3F8FC2034
:1077300042F08072C3F8FC20084AC2F8B01F1168FA
:1077400041F0010111602022DA7783F822007047AE
:1077500000ED00E00003FA0555CEACC5001000E0D6
:10776000302310B583F311880E4B5B6813F400636C
:1077700014D0F1EE103AEFF309844FF08073683CB7
:10778000E361094BDB6B236684F30988FEF7B8FEDF
:1077900010B1064BA36110BD054BFBE783F31188C5
:1077A000F9E700BF00ED00E000EF00E02F04000863
:1077B0003204000870B5BFF34F8FBFF36F8F1A4AC2
:1077C0000021C2F85012BFF34F8FBFF36F8F536980
:1077D00043F400335361BFF34F8FBFF36F8FC2F891
:1077E0008410BFF34F8FD2F8803043F6E074C3F3B8
:1077F000C900C3F34E335B0103EA0406014646EABF
:1078000081750139C2F86052F9D2203B13F1200F83
:10781000F2D1BFF34F8F536943F480335361BFF309
:107820004F8FBFF36F8F70BD00ED00E0FEE70000EB
:10783000214B2248224A70B5904237D3214BC11EBA
:10784000DA1C121A22F003028B4238BF00220021F8
:10785000FAF772FA1C4A0023C2F88430BFF34F8F44
:10786000D2F8803043F6E074C3F3C900C3F34E335B
:107870005B0103EA0406014646EA81750139C2F854
:107880006C52F9D2203B13F1200FF2D1BFF34F8F8E
:10789000BFF36F8FBFF34F8FBFF36F8F0023C2F81B
:1078A0005032BFF34F8FBFF36F8F70BD53F8041B7F
:1078B00040F8041BC0E700BF0C9D0008346700209F
:1078C000346700203467002000ED00E0074BD3F858
:1078D000D81021EA0001C3F8D810D3F8002122EA19
:1078E0000002C3F80021D3F8003170470044025869
:1078F00070B5D0E9244300224FF0FF359E6804EBB9
:1079000042135101D3F80009002805DAD3F8000921
:1079100040F08040C3F80009D3F8000B002805DAD6
:10792000D3F8000B40F08040C3F8000B013263181D
:107930009642C3F80859C3F8085BE0D24FF0011330
:10794000C4F81C3870BD0000890141F020010161BC
:1079500003699B06FCD41220FEF71CBE10B50A4C2E
:107960002046FEF7B7FA094BC4F89030084BC4F82C
:107970009430084C2046FEF7ADFA074BC4F890301F
:10798000064BC4F8943010BD3C6500200000084050
:10799000449C0008D865002000000440509C00086A
:1079A00070B503780546012B5CD1434BD0F890406D
:1079B000984258D1414B0E216520D3F8D82042F08F
:1079C0000062C3F8D820D3F8002142F00062C3F867
:1079D0000021D3F80021D3F8802042F00062C3F8E0
:1079E0008020D3F8802022F00062C3F88020D3F8F2
:1079F0008030FDF7B3FC324BE360324BC4F8003803
:107A00000023D5F89060C4F8003EC02323604FF4F3
:107A10000413A3633369002BFCDA01230C203361C8
:107A2000FEF7B8FD3369DB07FCD41220FEF7B2FD88
:107A30003369002BFCDA00262846A660FFF758FFC2
:107A40006B68C4F81068DB68C4F81468C4F81C6874
:107A500083BB1D4BA3614FF0FF336361A36843F009
:107A60000103A36070BD194B9842C9D1134B4FF06D
:107A70008060D3F8D82042F00072C3F8D820D3F841
:107A8000002142F00072C3F80021D3F80021D3F89E
:107A9000802042F00072C3F88020D3F8802022F0CA
:107AA0000072C3F88020D3F88030FFF70FFF0E215B
:107AB0004D209EE7064BCDE73C6500200044025870
:107AC0004014004003002002003C30C0D865002074
:107AD000083C30C0F8B5D0F89040054600214FF082
:107AE00000662046FFF730FFD5F8941000234FF0D2
:107AF00001128F684FF0FF30C4F83438C4F81C28E6
:107B000004EB431201339F42C2F80069C2F8006BD4
:107B1000C2F80809C2F8080BF2D20B68D5F8902019
:107B2000C5F89830636210231361166916F01006C9
:107B3000FBD11220FEF72EFDD4F8003823F4FE63AB
:107B4000C4F80038A36943F4402343F01003A36151
:107B50000923C4F81038C4F814380B4BEB604FF00D
:107B6000C043C4F8103B094BC4F8003BC4F810698B
:107B7000C4F80039D5F8983003F1100243F48013AB
:107B8000C5F89820A362F8BD209C00084080001032
:107B9000D0F8902090F88A10D2F8003823F4FE63D1
:107BA00043EA0113C2F80038704700002DE9F8439A
:107BB00000EB8103D0F890500C468046DA680FFA4B
:107BC00081F94801166806F00306731E022B05EBC7
:107BD00041134FF0000194BFB604384EC3F8101B98
:107BE0004FF0010104F1100398BF06F1805601FA2D
:107BF00003F3916998BF06F5004600293AD0578AE9
:107C000004F15801374349016F50D5F81C180B4354
:107C10000021C5F81C382B180127C3F81019A740FC
:107C20005369611E9BB3138A928B9B08012A88BFFC
:107C30005343D8F89820981842EA034301F14002D0
:107C40002146C8F89800284605EB82025360FFF7EA
:107C50007BFE08EB8900C3681B8A43EA84534834DF
:107C60001E4364012E51D5F81C381F43C5F81C78FB
:107C7000BDE8F88305EB4917D7F8001B21F4004154
:107C8000C7F8001BD5F81C1821EA0303C0E704F16C
:107C90003F030B4A2846214605EB83035A60FFF752
:107CA00053FE05EB4910D0F8003923F40043C0F827
:107CB0000039D5F81C3823EA0707D7E70080001001
:107CC00000040002D0F894201268C0F89820FFF752
:107CD0000FBE00005831D0F8903049015B5813F4C2
:107CE000004004D013F4001F0CBF02200120704795
:107CF0004831D0F8903049015B5813F4004004D06B
:107D000013F4001F0CBF02200120704700EB81011B
:107D1000CB68196A0B6813604B68536070470000AA
:107D200000EB810330B5DD68AA691368D36019B927
:107D3000402B84BF402313606B8A1468D0F89020D6
:107D40001C4402EB4110013C09B2B4FBF3F4634361
:107D5000033323F0030343EAC44343F0C043C0F8B2
:107D6000103B2B6803F00303012B0ED1D2F8083827
:107D700002EB411013F4807FD0F8003B14BF43F0B6
:107D8000805343F00053C0F8003B02EB4112D2F89D
:107D9000003B43F00443C2F8003B30BD2DE9F04105
:107DA000D0F8906005460C4606EB4113D3F8087BEB
:107DB0003A07C3F8087B08D5D6F814381B0704D552
:107DC00000EB8103DB685B689847FA071FD5D6F89C
:107DD0001438DB071BD505EB8403D968CCB98B6954
:107DE000488A5A68B2FBF0F600FB16228AB9186876
:107DF000DA6890420DD2121AC3E90024302383F3CB
:107E0000118821462846FFF78BFF84F31188BDE8CF
:107E1000F081012303FA04F26B8923EA02036B81E8
:107E2000CB68002BF3D021462846BDE8F041184727
:107E300000EB81034A0170B5DD68D0F890306C69C1
:107E40002668E66056BB1A444FF40020C2F81009B9
:107E50002A6802F00302012A0AB20ED1D3F80808F8
:107E600003EB421410F4807FD4F8000914BF40F0F3
:107E7000805040F00050C4F8000903EB4212D2F8E1
:107E8000000940F00440C2F800090122D3F8340888
:107E900002FA01F10143C3F8341870BD19B9402E3C
:107EA00084BF4020206020681A442E8A8419013C37
:107EB000B4FBF6F440EAC44040F00050C6E70000CE
:107EC0002DE9F843D0F8906005460C464F0106EBCB
:107ED0004113D3F8088918F0010FC3F808891CD0A2
:107EE000D6F81038DB0718D500EB8103D3F80CC0A7
:107EF000DCF81430D3F800E0DA68964530D2A2EB13
:107F00000E024FF000091A60C3F80490302383F387
:107F10001188FFF78DFF89F3118818F0800F1DD0AD
:107F2000D6F834380126A640334217D005EB840337
:107F30000134D5F89050D3F80CC0E4B22F44DCF8EB
:107F4000142005EB0434D2F800E05168714514D3D5
:107F5000D5F8343823EA0606C5F83468BDE8F88356
:107F6000012303FA01F2038923EA02030381DCF807
:107F70000830002BD1D09847CFE7AEEB0103BCF817
:107F80001000834228BF0346D7F8180980B2B3EB2C
:107F9000800FE3D89068A0F1040959F8048FC4F861
:107FA0000080A0EB09089844B8F1040FF5D81844F4
:107FB0000B4490605360C8E72DE9F84FD0F890501B
:107FC00004466E69AB691E4016F480586E6103D09A
:107FD000BDE8F84FFDF7EEBF002E12DAD5F8003EEF
:107FE0009B0705D0D5F8003E23F00303C5F8003EFB
:107FF000D5F80438204623F00103C5F80438FEF70D
:1080000007F8370505D52046FFF772FC2046FDF737
:10801000EDFFB0040CD5D5F8083813F0060FEB6867
:1080200023F470530CBF43F4105343F4A053EB609C
:1080300031071BD56368DB681BB9AB6923F0080304
:10804000AB612378052B0CD1D5F8003E9A0705D0FB
:10805000D5F8003E23F00303C5F8003E2046FDF7A7
:10806000D7FF6368DB680BB120469847F30200F145
:10807000BA80B70226D5D4F8909000274FF0010AB5
:1080800009EB4712D2F8003B03F44023B3F5802FED
:1080900011D1D2F8003B002B0DDA62890AFA07F3FE
:1080A00022EA0303638104EB8703DB68DB6813B117
:1080B0003946204698470137D4F89430FFB29B6880
:1080C0009F42DDD9F00619D5D4F89000026AC2F3B8
:1080D0000A1702F00F0302F4F012B2F5802F00F03D
:1080E000CA80B2F5402F09D104EB8303002200F5CA
:1080F0008050DB681B6A974240F0B0803003D5F8AF
:10810000185835D5E90303D500212046FFF746FE70
:10811000AA0303D501212046FFF740FE6B0303D5D8
:1081200002212046FFF73AFE2F0303D50321204604
:10813000FFF734FEE80203D504212046FFF72EFEA8
:10814000A90203D505212046FFF728FE6A0203D5C0
:1081500006212046FFF722FE2B0203D507212046E9
:10816000FFF71CFEEF0103D508212046FFF716FE9E
:10817000700340F1A780E90703D500212046FFF7EF
:108180009FFEAA0703D501212046FFF799FE6B0742
:1081900003D502212046FFF793FE2F0703D50321C5
:1081A0002046FFF78DFEEE0603D504212046FFF79B
:1081B00087FEA80603D505212046FFF781FE690644
:1081C00003D506212046FFF77BFE2A0603D50721AB
:1081D0002046FFF775FEEB0574D520460821BDE863
:1081E000F84FFFF76DBED4F890904FF0000B4FF0B2
:1081F000010AD4F894305FFA8BF79B689F423FF6F0
:1082000038AF09EB4713D3F8002902F44022B2F546
:10821000802F20D1D3F80029002A1CDAD3F80029B6
:1082200042F09042C3F80029D3F80029002AFBDB72
:108230003946D4F89000FFF787FB22890AFA07F342
:1082400022EA0303238104EB8703DB689B6813B1F5
:108250003946204698470BF1010BCAE7910701D137
:10826000D0F80080072A02F101029CBF03F8018BBD
:108270004FEA18283FE704EB830300F58050DA68E3
:10828000D2F818C0DCF80820DCE9001CA1EB0C0CCB
:1082900000218F4208D1DB689B699A683A449A6052
:1082A0005A683A445A6029E711F0030F01D1D0F817
:1082B00000808C4501F1010184BF02F8018B4FEA77
:1082C0001828E6E7BDE8F88F08B50348FFF774FE05
:1082D000BDE80840FFF744BA3C65002008B50348F4
:1082E000FFF76AFEBDE80840FFF73ABAD8650020FC
:1082F000D0F8903003EB4111D1F8003B43F4001368
:10830000C1F8003B70470000D0F8903003EB4111FA
:10831000D1F8003943F40013C1F800397047000068
:10832000D0F8903003EB4111D1F8003B23F4001357
:10833000C1F8003B70470000D0F8903003EB4111CA
:10834000D1F8003923F40013C1F800397047000058
:10835000064BD3F8DC200243C3F8DC20D3F8042119
:108360001043C3F80401D3F80431704700440258A5
:1083700008B53C4B4FF0FF31D3F8802062F000424B
:10838000C3F88020D3F8802002F00042C3F8802098
:10839000D3F88020D3F88420C3F88410D3F8842045
:1083A0000022C3F88420D3F88400D86F40F0FF4047
:1083B00040F4FF0040F4DF4040F07F00D867D86F02
:1083C00020F0FF4020F4FF0020F4DF4020F07F0089
:1083D000D867D86FD3F888006FEA40506FEA5050E2
:1083E000C3F88800D3F88800C0F30A00C3F88800F7
:1083F000D3F88800D3F89000C3F89010D3F8900019
:10840000C3F89020D3F89000D3F89400C3F89410E8
:10841000D3F89400C3F89420D3F89400D3F89800CC
:10842000C3F89810D3F89800C3F89820D3F89800B0
:10843000D3F88C00C3F88C10D3F88C00C3F88C20D0
:10844000D3F88C00D3F89C00C3F89C10D3F89C1090
:10845000C3F89C20D3F89C30FCF72EFABDE8084006
:1084600000F0D6B90044025808B50122534BC3F8B6
:108470000821534BD3F8F42042F00202C3F8F42051
:10848000D3F81C2142F00202C3F81C210222D3F8C7
:108490001C314C4BDA605A689104FCD54A4A1A6088
:1084A00001229A60494ADA6000221A614FF4404280
:1084B0009A61444B9A699204FCD51A6842F480721E
:1084C0001A603F4B1A6F12F4407F04D04FF4803291
:1084D0001A6700221A671A6842F001021A60384BC4
:1084E0001A685007FCD500221A611A6912F0380286
:1084F000FBD1012119604FF0804159605A67344A1D
:10850000DA62344A1A611A6842F480321A602C4BDB
:108510001A689103FCD51A6842F480521A601A68EE
:108520009204FCD52C4A2D499A6200225A631963A1
:1085300001F57C01DA6301F5E77199635A64284A11
:108540001A64284ADA621A6842F0A8521A601C4B70
:108550001A6802F02852B2F1285FF9D148229A61D4
:108560004FF48862DA6140221A621F4ADA641F4AB5
:108570001A651F4A5A651F4A9A6532231E4A1360BC
:10858000136803F00F03022BFAD10D4A136943F06D
:1085900003031361136903F03803182BFAD14FF06A
:1085A0000050FFF7D5FE4FF08040FFF7D1FE4FF0AF
:1085B0000040BDE80840FFF7CBBE00BF008000517F
:1085C000004402580048025800C000F002000001B8
:1085D0000000FF010088900832206000630209015A
:1085E000470E0508DD0BBF01200000200000011030
:1085F0000910E00000010110002000524FF0B042CD
:1086000008B5D2F8883003F00103C2F8883023B1EE
:10861000044A13680BB150689847BDE80840FFF75B
:108620009FB800BFB46600204FF0B04208B5D2F842
:10863000883003F00203C2F8883023B1044A9368FB
:108640000BB1D0689847BDE80840FFF789B800BF74
:10865000B46600204FF0B04208B5D2F8883003F07D
:108660000403C2F8883023B1044A13690BB150697E
:108670009847BDE80840FFF773B800BFB466002014
:108680004FF0B04208B5D2F8883003F00803C2F8C2
:10869000883023B1044A93690BB1D0699847BDE88B
:1086A0000840FFF75DB800BFB46600204FF0B0424D
:1086B00008B5D2F8883003F01003C2F8883023B12F
:1086C000044A136A0BB1506A9847BDE80840FFF7A7
:1086D00047B800BFB46600204FF0B04310B5D3F8E0
:1086E000884004F47872C3F88820A30604D5124A9F
:1086F000936A0BB1D06A9847600604D50E4A136B93
:108700000BB1506B9847210604D50B4A936B0BB104
:10871000D06B9847E20504D5074A136C0BB1506C37
:108720009847A30504D5044A936C0BB1D06C9847C5
:10873000BDE81040FFF714B8B46600204FF0B04316
:1087400010B5D3F8884004F47C42C3F88820620551
:1087500004D5164A136D0BB1506D9847230504D507
:10876000124A936D0BB1D06D9847E00404D50F4ABF
:10877000136E0BB1506E9847A10404D50B4A936E4B
:108780000BB1D06E9847620404D5084A136F0BB141
:10879000506F9847230404D5044A936F0BB1D06FF0
:1087A0009847BDE81040FEF7DBBF00BFB46600206D
:1087B00008B50348FCF748FCBDE80840FEF7D0BF09
:1087C000C836002008B50348FCF742FDBDE8084064
:1087D000FEF7C6BF2039002008B50348FCF738FD76
:1087E000BDE80840FEF7BCBF8C39002008B503483F
:1087F000FCF72EFDBDE80840FEF7B2BFF8390020B7
:1088000008B500F0BDFCBDE80840FEF7A9BF0000B8
:10881000062108B50846FCF7A1FD06210720FCF754
:108820009DFD06210820FCF799FD06210920FCF793
:1088300095FD06210A20FCF791FD06211720FCF783
:108840008DFD06212820FCF789FD09217A20FCF7FF
:1088500085FD09213120FCF781FD07213220FCF73D
:108860007DFD0C212620FCF779FD0C212720FCF74B
:1088700075FD0C215220BDE80840FCF76FBD0000DB
:1088800008B5FFF775FD00F043FCFDF747F9FDF76C
:10889000E5F8FDF71DFBFDF7EFF9FEF7B1F9BDE8CF
:1088A000084000F029BA000030B50433039C01727F
:1088B000002104FB0325C160C0E90653049B036348
:1088C000059BC0E90000C0E90422C0E90842C0E9F4
:1088D0000A11436330BD00000022416AC260C0E952
:1088E0000411C0E90A226FF00101FDF7FFBE00008C
:1088F000D0E90432934201D1C2680AB9181D704709
:1089000000207047036919600021C2680132C2600B
:10891000C269134482699342036124BF436A0361BD
:10892000FDF7D8BE38B504460D46E3683BB1626931
:108930000020131D1268A3621344E36207E0237A48
:1089400033B929462046FDF7B5FE0028EDDA38BDDB
:108950006FF00100FBE70000C368C269013BC36020
:108960004369134482699342436124BF436A43616C
:1089700000238362036B03B11847704770B530233F
:10898000044683F31188866A3EB9FFF7CBFF05469C
:1089900018B186F31188284670BDA36AE26A13F8FD
:1089A000015B9342A36202D32046FFF7D5FF002369
:1089B00083F31188EFE700002DE9F84F04460E46D7
:1089C000174698464FF0300989F311880025AA46CA
:1089D000D4F828B0BBF1000F09D141462046FFF77B
:1089E000A1FF20B18BF311882846BDE8F88FD4E9A8
:1089F0000A12A7EB050B521A934528BF9346BBF109
:108A0000400F1BD9334601F1400251F8040B91424B
:108A100043F8040BF9D1A36A403640354033A362D2
:108A2000D4E90A239A4202D32046FFF795FF8AF33E
:108A30001188BD42D8D289F31188C9E730465A4619
:108A4000F9F754F9A36A5E445D445B44A362E7E727
:108A500010B5029C0433017203FB0421C460C0E919
:108A600006130023C0E90A33039B0363049BC0E998
:108A70000000C0E90422C0E90842436310BD0000C1
:108A8000026A6FF00101C260426AC0E9042200225A
:108A9000C0E90A22FDF72ABED0E904239A4201D197
:108AA000C26822B9184650F8043B0B607047002397
:108AB0001846FAE7C3680021C2690133C3604369FD
:108AC000134482699342436124BF436A4361FDF7C3
:108AD00001BE000038B504460D46E3683BB123698A
:108AE00000201A1DA262E2691344E36207E0237AC0
:108AF00033B929462046FDF7DDFD0028EDDA38BD03
:108B00006FF00100FBE7000003691960C268013AD9
:108B1000C260C269134482699342036124BF436AFD
:108B2000036100238362036B03B1184770470000A1
:108B300070B530230D460446114683F31188866ACA
:108B40002EB9FFF7C7FF10B186F3118870BDA36A75
:108B50001D70A36AE26A01339342A36204D3E16900
:108B600020460439FFF7D0FF002080F31188EDE79D
:108B70002DE9F84F04460D46904699464FF0300ACD
:108B80008AF311880026B346A76A4FB949462046A2
:108B9000FFF7A0FF20B187F311883046BDE8F88FBA
:108BA000D4E90A073A1AA8EB0607974228BF1746E6
:108BB000402F1BD905F1400355F8042B9D4240F886
:108BC000042BF9D1A36A40364033A362D4E90A23C7
:108BD0009A4204D3E16920460439FFF795FF8BF3ED
:108BE00011884645D9D28AF31188CDE729463A46FD
:108BF000F9F77CF8A36A3D443E443B44A362E5E7B1
:108C0000D0E904239A4217D1C3689BB1836A8BB120
:108C1000043B9B1A0ED01360C368013BC360C36959
:108C20001A4483699A42026124BF436A03610023A4
:108C300083620123184670470023FBE701F01F03FE
:108C4000F0B502F01F0456095A1C0123B6EB511F60
:108C500050F8265003FA02F34FEA511703F1FF339D
:108C60003DBF50F82720C4F12000134003EA05005F
:108C70003BBF03FA00F225FA04F0E0401043F0BDD8
:108C800070B57E227F210546FFF7D8FF18B1012875
:108C900019D0002070BD3E2249212846FFF7CEFFA3
:108CA0002F22044631212846FFF7C8FF064601342B
:108CB0005022023653212846B440FFF7BFFF09383F
:108CC00004FA00F0E6E7302245212846FFF7B6FF18
:108CD00001308002DEE7000090F8D63090F8D7200F
:108CE0001B0403EB026390F8D42090F8D5001344E2
:108CF00003EB00207047000000F018BA014B586ADF
:108D0000704700BF000C0040034B002258631A61FB
:108D10000222DA60704700BF000C0040014B0022C5
:108D2000DA607047000C0040014B5863704700BF89
:108D3000000C0040024B034A1A60034A5A60704715
:108D40008C6600203867002000000220074B494253
:108D500010B55C68201A08401968821A8A4203D349
:108D6000A24201D85A6010BD0020FCE78C660020AA
:108D700008B5302383F31188FFF7E8FF002383F35E
:108D8000118808BD0448054B03600023C0E9013386
:108D90000C3000F017B900BF94660020718D0008F8
:108DA000CB1D083A23F00703591A521A10B4D208FF
:108DB0000024C0E9004384600C301C605A605DF8F8
:108DC000044B00F0FFB800002DE9F74F364FCD1DE2
:108DD0008846002818BF0746082A4FEAD50538BF3D
:108DE000082207F10C003C1D9146019000F02CF97F
:108DF000019809F10701C9F1000E2246246864B9FF
:108E000000F02CF93B68CBB308224946E8009847AC
:108E1000044698B340E9027830E004EB010CD4F842
:108E200004A00CEA0E0C0AF10106ACF1080304EBF5
:108E3000C6069E42E1D9A6EB0C0CB5EBEC0F4FEA4F
:108E4000EC0BDAD89C421DD204F10802AB45A3EB2F
:108E500002024FEAE202626009D9691CED4303EBAA
:108E6000C1025D445560256843F8315022601C46BC
:108E7000C3F8048044F8087B00F0F0F8204603B003
:108E8000BDE8F08FAA45216802D111602346EEE7C4
:108E9000013504EBC50344F8351003F10801761AD7
:108EA000F6105E601360F1E79466002073B5044627
:108EB000A0F1080550F8080C54F8043C061D0C30CD
:108EC00007330190DB0844F8043C00F0BDF833465A
:108ED00001989E421A6801D0AB4228D20AB195424D
:108EE00025D244F8082C54F8042C1D60013254F8A3
:108EF000081C05EBC206B14206D14E68324444F864
:108F0000042C0A6844F8082C5E68711C03EBC1014C
:108F10008D4207D154F8042C013232445A6054F87F
:108F2000082C1A6002B0BDE8704000F097B81346F4
:108F3000CFE70000FEE7000070B51E4B0025044699
:108F400086B058600E4605638163FEF7E1FB04F1CD
:108F50002803A5606563C4E90A3304F11003C4E97A
:108F600004334FF0FF33C4E90044C4E90635FFF78A
:108F7000C5FE2B46024604F13C012046C4E9082305
:108F800080230D4A6567FDF70FFB7368E0600B4AAD
:108F900003620123009280F824306846F26801924F
:108FA0003269CDE90223064BCDE90435FDF730FBEC
:108FB00006B070BD10490020649C00085C9C00084D
:108FC000358F00080023C0E900008360036170470B
:108FD00070B51C4B05468468DE685CB3B44213D19F
:108FE00003690133036170BDA36094F8243083B139
:108FF000062B15D1A06A2146D4E9003213605A60CD
:10900000FDF73EFAA36A9C68B368A2689A42EBD364
:1090100006E0D4E90032204613605A60FDF740FABA
:1090200028463146FDF72CFAB5620620BDE87040AF
:10903000FDF738BA0369866001330361336BC3609F
:109040003063D0E76846002008B5302383F31188E9
:10905000FFF7BEFF002383F3118808BD194BD968C1
:1090600083688B4210B520D1302383F311880269C5
:10907000013A0261B2B90468C368A0420B631ED012
:109080004A6B9BB901238A60036103681A68026016
:1090900050601A6B8360C26018631846FDF700FACF
:1090A000FDF750FA002383F3118810BD1C68A3421A
:1090B00003D0A468A24238BF2246DB68E1E78260A1
:1090C000F0E700BF68460020024A536B1843506324
:1090D000704700BF6846002038B5EFF311859DB991
:1090E000EFF30584C4F30804302334B183F311880B
:1090F000FDF734FC85F3118838BD83F31188FDF743
:109100002DFC84F3118838BDBDE83840FDF726BC3E
:109110000023054A19460133102BC2E9001102F160
:109120000802F8D1704700BFB4660020114BD3F895
:10913000E82042F00802C3F8E820D3F8102142F0FA
:109140000802C3F810210C4AD3F81031D36B43F056
:109150000803D363C722094B9A624FF0FF32DA62E9
:1091600000229A615A63DA605A6001225A611A60D9
:10917000704700BF004402580010005C000C004023
:10918000094A08B51169D3680B40D9B29B076FEA49
:109190000101116107D5302383F31188FDF7F8F938
:1091A000002383F3118808BD000C004010B501397D
:1091B0000244904201D1002005E0037811F8014FEC
:1091C000A34201D0181B10BD0130F2E7884210B550
:1091D00001EB020402D98442234607D8431EA14270
:1091E00008D011F8012B03F8012FF8E702440146DB
:1091F0008A4200D110BD13F8014D02F8014DF7E786
:10920000C9B2034610F8012B1AB18A42F9D11846A7
:109210007047002918BF0023F9E70000034611F842
:10922000012B03F8012B002AF9D1704710B5013941
:10923000034632B111F8014F03F8014B013A002CFB
:10924000F7D11A440021934200D110BD03F8011B4D
:10925000F9E700004D4435002D2D0A002F6172649E
:109260007570696C6F742E6162696E002F61726433
:109270007570696C6F742D7665726966792E61629E
:10928000696E002F6172647570696C6F742D666C05
:109290006173682E6162696E002F61726475706916
:1092A0006C6F742D666C61736865642E6162696EA3
:1092B000000000000000000000000000050F000892
:1092C000A10F000851110008D90F0008990F0008DC
:1092D0000000000000000000010F0008AD0F0008B2
:1092E00089110008FD0E0008090F000853544D3382
:1092F0003248373F3F3F0053544D3332483733787D
:109300002F3732780053544D3332483734332F37A8
:1093100035332F373530000001105A000310590043
:1093200001205800032056002F000000537563638E
:1093300065737366756C6C79206D6F756E7465649A
:10934000205344436172642028736C6F77646F7795
:109350006E3D2575290A0000EB769045584641542C
:1093600020202000464154333220202000000000FD
:109370002A3A3C3E7C223F7F002B2C3B3D5B5D002C
:10938000435545414141414345454549494941418D
:109390004592924F4F4F5555594F554F9C4F9E9F59
:1093A00041494F55A5A5A6A7A8A9AAABACADAEAF9C
:1093B000B0B1B2B3B4414141B8B9BABBBCBDBEBF94
:1093C000C0C1C2C3C4C54141C8C9CACBCCCDCECF30
:1093D000D1D145454549494949D9DADBDCDD49DF89
:1093E0004FE14F4F4F4FE6E8E85555555959EEEFCD
:1093F000F0F1F2F3F4F5F6F7F8F9FAFBFCFDFEFFF5
:1094000001030507090E10121416181C1E00000097
:1094100061001A03E0001703F8000703FF000100D2
:1094200078010001300132010601390110014A01C1
:109430002E017901060180014D0043028101820164
:1094400082018401840186018701870189018A01E3
:109450008B018B018D018E018F0190019101910192
:1094600093019401F60196019701980198013D023C
:109470009B019C019D0120029F01A001A001A2016E
:10948000A201A401A401A601A701A701A901AA01A3
:10949000AB01AC01AC01AE01AF01AF01B101B20152
:1094A000B301B301B501B501B701B801B801BA0103
:1094B000BB01BC01BC01BE01F701C001C101C20179
:1094C000C301C401C501C401C701C801C701CA0164
:1094D000CB01CA01CD011001DD0101008E01DE01C9
:1094E0001201F3010300F101F401F401F801280174
:1094F000220212013A020900652C3B023B023D02A6
:10950000662C3F0240024102410246020A01530218
:10951000400081018601550289018A0158028F01AC
:109520005A0290015C025D025E025F0293016102D9
:109530006202940164026502660267029701960165
:109540006A02622C6C026D026E029C017002710252
:109550009D01730274029F017602770278027902FC
:109560007A027B027C02642C7E027F02A6018102C9
:109570008202A9018402850286028702AE014402AA
:10958000B101B20145028D028E028F02900291025A
:10959000B7017B030300FD03FE03FF03AC030400DC
:1095A0008603880389038A03B1031103C2030200FF
:1095B000A303A303C4030803CC0303008C038E039B
:1095C0008F03D8031801F2030A00F903F303F4032D
:1095D000F503F603F703F703F903FA03FA0330047C
:1095E000200350041007600422018A043601C104DC
:1095F0000E01CF040100C004D0044401610526041B
:10960000000000007D1D0100632C001E9601A01EBD
:109610005A01001F0806101F0606201F0806301FEB
:109620000806401F0606511F0700591F521F5B1FE7
:10963000541F5D1F561F5F1F601F0806701F0E001E
:10964000BA1FBB1FC81FC91FCA1FCB1FDA1FDB1FD2
:10965000F81FF91FEA1FEB1FFA1FFB1F801F0806E8
:10966000901F0806A01F0806B01F0400B81FB91FEE
:10967000B21FBC1FCC1F0100C31FD01F0206E01F7A
:109680000206E51F0100EC1FF31F0100FC1F4E2125
:109690000100322170211002842101008321D02495
:1096A0001A05302C2F04602C0201672C0601752C42
:1096B0000201802C6401002D260841FF1A030000DE
:1096C000C700FC00E900E200E400E000E500E7007C
:1096D000EA00EB00E800EF00EE00EC00C400C5007B
:1096E000C900E600C600F400F600F200FB00F90035
:1096F000FF00D600DC00F800A300D800D7009201DC
:10970000E100ED00F300FA00F100D100AA00BA0078
:10971000BF00AE00AC00BD00BC00A100AB00BB00B0
:1097200091259225932502252425C100C200C00061
:10973000A9006325512557255D25A200A500102508
:10974000142534252C251C2500253C25E300C300C9
:109750005A25542569256625602550256C25A400C9
:10976000F000D000CA00CB00C8003101CD00CE000F
:10977000CF0018250C2588258425A600CC0080253F
:10978000D300DF00D400D200F500D500B500FE0004
:10979000DE00DA00DB00D900FD00DD00AF00B40020
:1097A000AD00B1001720BE00B600A700F700B8005A
:1097B000B000A800B700B900B300B200A025A00017
:1097C00010000240080002400008024000000B00A8
:1097D00028000240080002400408024006010C0074
:1097E00040000240080002400808024010020D003C
:1097F00058000240080002400C08024016030E0008
:10980000700002400C0002401008024000040F00EB
:10981000880002400C0002401408024006051000B7
:10982000A00002400C00024018080240100611007F
:10983000B80002400C0002401C08024016072F002E
:1098400010040240080402402008024000083800CA
:109850002804024008040240240802400609390096
:10986000400402400804024028080240100A3A005E
:1098700058040240080402402C080240160B3B002A
:10988000700402400C04024030080240000C3C000E
:10989000880402400C04024034080240060D4400D3
:1098A000A00402400C04024038080240100E45009B
:1098B000B80402400C0402403C080240160F460067
:1098C0000100000000000000009600000000000001
:1098D0000000000000000000000000000000000088
:1098E00000000000F96B0008FD6B0008F15600084D
:1098F000295A000885560008AD560008D5560008BC
:109900006D56000800000000DD5A0008C95A000822
:10991000055B0008F15A0008FD5A0008E95A0008E2
:10992000D55A0008C15A0008115B00080000000069
:10993000F55B0008E15B00081D5C0008095C00089D
:10994000155C0008015C0008ED5B0008D95B0008AD
:10995000295C000800000000010000000000000079
:109960006330000060990008000000000000000063
:10997000E0460020104900200000812A000000007D
:10998000AAAAAAAA00000024FFFE0000000000000E
:1099900000A00A000001000000000000AAAAAAAA74
:1099A00000000000FFFF00000000000000000000B9
:1099B0001400AA5600000000AAAAAAAA140055542E
:1099C000FFFF000000000000CCCC0C0020681A0053
:1099D00000000000AAAA8AAA10541500FFFF000088
:1099E000000C7007770000004081020100100000A9
:1099F000AAAAAAAA00410100F7FF00000000007017
:109A0000070000000000000000000000AAAAAAAAA7
:109A100000000000FFFF0000000000000000000048
:109A20000000000000000000AAAAAAAA000000008E
:109A3000FFFF000000000000000000000000000028
:109A400000000000AAAAAAAA00000000FFFF000070
:109A50000000000000000000000000000000000006
:109A6000AAAAAAAA00000000FFFF00000000000050
:109A7000000000000000000000000000AAAAAAAA3E
:109A800000000000FFFF00000000000000000000D8
:109A90000000000000000000AAAAAAAA000000001E
:109AA000FFFF000000000000000000004865782F64
:109AB00050726F6669434E430025424F4152442520
:109AC0002D424C002553455249414C2500000000D1
:109AD0000200000000000000155E0008855E00081E
:109AE00040004000C0610020D06100200200000062
:109AF000000000000300000000000000CD5E000830
:109B00000000000010000000E061002000000000E4
:109B100001000000000000003C650020010102007F
:109B2000F56C0008056C0008A16C0008856C000845
:109B300043000000389B000809024300020100C0F6
:109B40003209040000010202010005240010010591
:109B500024010001042402020524060001070582F5
:109B6000030800FF09040100020A000000070501C4
:109B700002400000070581024000000012000000C2
:109B8000849B00081201100102000040AE2D161047
:109B900000020102030100000403090425424F41B1
:109BA00052442500437562654F72616E67650030EF
:109BB0003132333435363738394142434445460033
:109BC0000000002000000200020000000000003041
:109BD000000004000800000000000024000008004D
:109BE000040000000004000000FC0000020000006F
:109BF0000000043000800000080000000000003871
:109C000000000100010000001F1C1F1E1F1E1F1F5F
:109C10001E1F1E1F1F1D1F1E1F1E1F1F1E1F1E1F5C
:109C20000000000029600008E16200088D63000860
:109C300040004000746600207466002001000000AF
:109C40008466002080000000400100000800000041
:109C500000010000001000000800000069646C654D
:109C6000000000006D61696E002C0438040438089F
:109C70000C10141C202425260000000000006404A1
:109C80000100040000000000000C00102830340027
:109C9000D867FF7F010000008C000000000000007A
:109CA00000001E0000000000FF0000001849002016
:109CB000203900208C390020F839002000000000F5
:109CC000EC92000883040000F792000850040000A2
:109CD000059300080100000000000000009600004D
:109CE00000000800960000000008000004000000CA
:109CF000989B000800000000000000000000000029
:109D0000000000000000000000000000FFFFFFFF57
:109D1000FFFFFFFFFFFFFFFFFFFFFFFFFFFFFFFF53
:109D2000FFFFFFFFFFFFFFFFFFFFFFFFFFFFFFFF43
:109D3000FFFFFFFFFFFFFFFFFFFFFFFFFFFFFFFF33
:109D4000FFFFFFFFFFFFFFFFFFFFFFFFFFFFFFFF23
:020000040801F1
:020000040802F0
:1000000000060030010E020881DB110871030208AE
:10001000FDDA1108F5DA1108F9DA1108030E020801
:10002000030E0208030E0208030E0208012D180831
:10003000030E0208030E0208030E0208030E020854
:10004000030E0208030E0208030E0208030E020844
:10005000030E0208030E0208F9B0180825B11808AB
:1000600051B118087DB11808A9B118082D3C18081D
:10007000553C1808813C1808AD3C1808D93C1808B4
:10008000013D18082D3D1808153818085DC91108DC
:1000900045CA1108CDC91108B5CA1108D5B118084B
:1000A000030E020839B31808030E02084DB31808EE
:1000B00061B31808030E020875B31808354518080F
:1000C000A94518081D46180891461808DD52180859
:1000D000F1521808030E0208C1B21808D5B2180868
:1000E00039B21808030E0208030E0208030E0208B4
:1000F000030E0208030E0208030E0208593D1808F9
:10010000030E0208ADB2180889B31808030E0208DE
:10011000E9B21808030E0208030E0208030E0208D3
:10012000853D1808AD3D1808D93D1808053E18084A
:10013000313E1808030E0208030E0208030E0208DF
:10014000030E0208030E0208030E0208030E020843
:10015000593E1808853E1808B13E1808FDB2180827
:10016000030E0208030E0208030E0208030E020823
:10017000030E02083DAD1808030E0208030E020824
:10018000030E0208030E020811B3180825B318085D
:1001900005531808030E0208030E0208030E020896
:1001A000030E0208030E0208030E0208030E0208E3
:1001B000030E0208030E0208030E0208030E0208D3
:1001C000030E0208030E0208030E0208030E0208C3
:1001D000030E020829AD1808030E0208030E0208D8
:1001E000030E0208030E0208030E0208030E0208A3
:1001F000030E0208030E0208030E0208030E020893
:10020000030E0208030E0208030E0208030E020882
:10021000030E0208030E0208030E0208030E020872
:10022000030E0208030E0208030E0208030E020862
:10023000030E0208030E0208030E020835381808E0
:10024000030E0208DD391808053A1808313A180873
:100250005D3A1808893A1808B53A1808E13A1808BA
:100260000D3B1808030E0208030E0208030E0208D5
:10027000030E0208030E0208030E0208030E020812
:10028000030E0208030E0208030E0208030E020802
:10029000030E0208030E0208030E0208030E0208F2
:1002A000030E0208030E0208030E0208030E0208E2
:1002B000030E0208030E0208030E0208030E0208D2
:1002C000030E0208030E0208030E0208030E0208C2
:1002D000030E0208030E0208030E0208030E0208B2
:1002E0000585020855EB04088D4E0508D9DF050881
:1002F000E564070821F6090841FD0908F1A80A0884
:100300007D270B0815300B08A1330B0819BE0B080D
:1003100061F30B08A5080C08A5AC0C08A5E10D08B5
:100320001D4D0E08995C0E0831CE11086DD31108D1
:10033000ADF21108AD971308EDE91308F93F140861
:10034000C5901408DD201608655D1608A97A160800
:10035000BDA41608ADD81608750917081116170898
:1003600045521708995D17080000000000000000C2
:10037000EFF30383EFF30982EFF30881DFF814D082
:100380002DE9FE4F684601F011F8BDE8FE4F8D469D
:100390007047000064330030F1EE101AA0EC200A20
:1003A00001607047A0EC108A704700BF81F00041E7
:1003B00002E000BF83F0004330B54FEA41044FEA4A
:1003C000430594EA050F08BF90EA020F1FBF54EAE5
:1003D000000C55EA020C7FEA645C7FEA655C00F081
:1003E000E2804FEA5454D4EB5555B8BF6D420CDD52
:1003F0002C4480EA020281EA030382EA000083EAD5
:10040000010180EA020281EA0303362D88BF30BD74
:1004100011F0004F4FEA01314FF4801C4CEA1131CA
:1004200002D0404261EB410113F0004F4FEA033329
:100430004CEA133302D0524263EB430394EA050FB4
:1004400000F0A780A4F10104D5F1200E0DDB02FA23
:100450000EFC22FA05F2801841F1000103FA0EF2B7
:10046000801843FA05F359410EE0A5F120050EF17D
:10047000200E012A03FA0EFC28BF4CF0020C43FAAE
:1004800005F3C01851EBE37101F0004507D54FF0BB
:10049000000EDCF1000C7EEB00006EEB0101B1F50B
:1004A000801F1BD3B1F5001F0CD349085FEA300051
:1004B0004FEA3C0C04F101044FEA445212F5800F5C
:1004C00080F09A80BCF1004F08BF5FEA500C50F1F9
:1004D000000041EB045141EA050130BD5FEA4C0CDC
:1004E000404141EB0101013C28BFB1F5801FE9D239
:1004F00091F0000F04BF01460020B1FA81F308BF5C
:100500002033A3F10B03B3F120020CDA0C3208DD27
:1005100002F1140CC2F10C0201FA0CF021FA02F102
:100520000CE002F11402D8BFC2F1200C01FA02F172
:1005300020FA0CFCDCBF41EA0C019040E41AA2BF97
:1005400001EB0451294330BD6FEA04041F3C1CDA5F
:100550000C340EDC04F11404C4F1200220FA04F07F
:1005600001FA02F340EA030021FA04F345EA030129
:1005700030BDC4F10C04C4F1200220FA02F001FAEB
:1005800004F340EA0300294630BD21FA04F029466D
:1005900030BD94F0000F83F4801306BF81F4801106
:1005A0000134013D4EE77FEA645C18BF7FEA655C79
:1005B00029D094EA050F08BF90EA020F05D054EA4B
:1005C000000C04BF1946104630BD91EA030F1EBF50
:1005D0000021002030BD5FEA545C05D14000494154
:1005E00028BF41F0004130BD14F580043CBF01F547
:1005F000801130BD01F0004545F0FE4141F470012D
:100600004FF0000030BD7FEA645C1ABF1946104607
:100610007FEA655C1CBF0B46024650EA013406BF08
:1006200052EA033591EA030F41F4002130BD00BFC7
:1006300090F0000F04BF0021704730B54FF4806484
:1006400004F132044FF000054FF0000150E700BF05
:1006500090F0000F04BF0021704730B54FF4806464
:1006600004F1320410F0004548BF40424FF0000151
:100670003EE700BF42004FEAE2014FEA31014FEA94
:1006800002701FBF12F07F4393F07F4F81F06051E3
:10069000704732F07F4208BF704793F07F4F04BF2E
:1006A00041F40021704730B54FF4607401F000450B
:1006B00021F000411CE700BF50EA010208BF70476B
:1006C00030B54FF000050AE050EA010208BF70475C
:1006D00030B511F0004502D5404261EB41014FF4C5
:1006E000806404F132045FEA915C3FF4D8AE4FF0CD
:1006F00003025FEADC0C18BF03325FEADC0C18BFB0
:10070000033202EBDC02C2F1200300FA03FC20FA00
:1007100002F001FA03FE40EA0E0021FA02F114444D
:10072000BDE600BF80F0004002E000BF81F0004164
:1007300042001FBF5FEA410392EA030F7FEA226C87
:100740007FEA236C6AD04FEA1262D2EB1363C1BF17
:10075000D218414048404140B8BF5B42192B88BF86
:10076000704710F0004F40F4000020F07F4018BFA9
:10077000404211F0004F41F4000121F07F4118BFC9
:10078000494292EA030F3FD0A2F1010241FA03FC71
:1007900010EB0C00C3F1200301FA03F100F0004359
:1007A00002D5494260EB4000B0F5000F13D3B0F121
:1007B000807F06D340084FEA310102F10102FE2A90
:1007C00051D2B1F1004F40EBC25008BF20F0010000
:1007D00040EA03007047490040EB0000013A28BF9F
:1007E000B0F5000FEDD2B0FA80FCACF1080CB2EB22
:1007F0000C0200FA0CF0AABF00EBC25052421843A0
:10080000BCBFD0401843704792F0000F81F4000144
:1008100006BF80F400000132013BB5E74FEA410317
:100820007FEA226C18BF7FEA236C21D092EA030F83
:1008300004D092F0000F08BF0846704790EA010FFD
:100840001CBF0020704712F07F4F04D1400028BF2A
:1008500040F00040704712F100723CBF00F500000C
:10086000704700F0004343F0FE4040F40000704742
:100870007FEA226216BF08467FEA236301464202EE
:1008800006BF5FEA412390EA010F40F48000704701
:100890004FF0000304E000BF10F0004348BF4042A7
:1008A0005FEA000C08BF704743F0964301464FF0E3
:1008B00000001CE050EA010208BF70474FF000033F
:1008C0000AE000BF50EA010208BF704711F0004380
:1008D00002D5404261EB41015FEA010C02BF844650
:1008E0000146002043F0B64308BFA3F18053A3F5AF
:1008F0000003BCFA8CF2083AA3EBC25310DB01FAF6
:1009000002FC634400FA02FCC2F12002BCF1004F79
:1009100020FA02F243EB020008BF20F0010070470A
:1009200002F1200201FA02FCC2F1200250EA4C005E
:1009300021FA02F243EB020008BF20EADC707047A4
:100940007BB972B90029BEBF00204FF0004106E01C
:1009500008BF00281CBF6FF000414FF0FF3000F0CF
:100960004DBAADF1080C6DE904CE002909DB002B6E
:100970001ADB00F0DBF8DDF804E0DDE9022304B067
:100980007047404261EB4101002B1BDB00F0CEF8C9
:10099000DDF804E0DDE9022304B0404261EB4101EF
:1009A000524263EB43037047524263EB430300F050
:1009B000BDF8DDF804E0DDE9022304B0404261EB5C
:1009C00041017047524263EB430300F0AFF8DDF89A
:1009D00004E0DDE9022304B0524263EB43037047B5
:1009E00053B94AB9002908BF00281CBF4FF0FF3196
:1009F0004FF0FF3000F002BAADF1080C6DE904CE03
:100A000000F094F8DDF804E0DDE9022304B070475B
:100A100030B1012390FAA0F0B0FA80F0184470478A
:100A200008460029FBD02123F4E700BF430803F068
:100A30005533C01A830803F0333300F033301844C1
:100A400000EB101000F00F3000EB002000EB004036
:100A5000000E704707EE900AF5EEC07AF1EE10FA3C
:100A600001D400F023B8F1EE677A08B517EE900ACA
:100A700000F01CF8404261EB410108BD08B5024698
:100A80000B4643EC172BB5EEC07BF1EE10FA03D406
:100A9000BDE8084000F02AB8B1EE477B51EC170BD7
:100AA00000F024F8404261EB410108BD9FED0B6B63
:100AB00007EE900A9FED0B5BB7EEE77A27EE066B29
:100AC000BCEEC66BB8EE464BA4EE457BFCEEC77B96
:100AD00016EE101A17EE900A704700BF00000000D3
:100AE0000000F03D000000000000F0419FED0B6BA6
:100AF00041EC170B9FED0B5B27EE066BBCEEC66B54
:100B0000B8EE464BA4EE457BFCEEC77B16EE101A02
:100B100017EE900A704700BFAFF30080000000009E
:100B20000000F03D000000000000F0412DE9F0471A
:100B3000089D04468E46002B4DD18A42944669D9C1
:100B4000B2FA82F252B101FA02F3C2F1200120FAA4
:100B500001F10CFA02FC41EA030E94404FEA1C48F2
:100B6000210CBEFBF8F61FFA8CF708FB16E341EAEE
:100B7000034306FB07F199420AD91CEB030306F174
:100B8000FF3080F01F81994240F21C81023E634495
:100B90005B1AA4B2B3FBF8F008FB103344EA034439
:100BA00000FB07F7A7420AD91CEB040400F1FF334E
:100BB00080F00A81A74240F207816444023840EA8B
:100BC0000640E41B00261DB1D4400023C5E90043C4
:100BD0003146BDE8F0878B4209D9002D00F0EF8047
:100BE0000026C5E9000130463146BDE8F087B3FA7A
:100BF00083F6002E4AD18B4202D3824200F2F98062
:100C0000841A61EB030301209E46002DE0D0C5E964
:100C1000004EDDE702B9FFDEB2FA82F2002A40F0B0
:100C20009280A1EB0C014FEA1C471FFA8CFE0126B3
:100C3000200CB1FBF7F307FB131140EA01410EFB57
:100C400003F0884208D91CEB010103F1FF3802D2FE
:100C5000884200F2CB804346091AA4B2B1FBF7F0F8
:100C600007FB101144EA01440EFB00FEA64508D91B
:100C70001CEB040400F1FF3102D2A64500F2BB8058
:100C80000846A4EB0E0440EA03409CE7C6F12007A7
:100C9000B34022FA07FC4CEA030C20FA07F401FAED
:100CA00006F31C43F9404FEA1C4900FA06F3B1FB76
:100CB000F9F8200C1FFA8CFE09FB181140EA0141DB
:100CC00008FB0EF0884202FA06F20BD91CEB010178
:100CD00008F1FF3A80F08880884240F28580A8F1D0
:100CE00002086144091AA4B2B1FBF9F009FB101122
:100CF00044EA014100FB0EFE8E4508D91CEB0101C0
:100D000000F1FF346CD28E456AD90238614440EA62
:100D10000840A0FB0294A1EB0E01A142C846A646E2
:100D200056D353D05DB1B3EB080261EB0E0101FA6B
:100D300007F722FA06F3F1401F43C5E900710026C8
:100D40003146BDE8F087C2F12003D8400CFA02FC1E
:100D500021FA03F3914001434FEA1C471FFA8CFE2E
:100D6000B3FBF7F007FB10360B0C43EA064300FB1E
:100D70000EF69E4204FA02F408D91CEB030300F1BC
:100D8000FF382FD29E422DD9023863449B1B89B273
:100D9000B3FBF7F607FB163341EA034106FB0EF3FC
:100DA0008B4208D91CEB010106F1FF3816D28B42A9
:100DB00014D9023E6144C91A46EA004638E72E4675
:100DC000284605E70646E3E61846F8E64B45A9D26D
:100DD000B9EB020864EB0C0E0138A3E74646EAE7DC
:100DE000204694E74046D1E7D0467BE7023B61448A
:100DF00032E7304609E76444023842E7704700BFF3
:100E000002E000F000F8FEE772B6374880F3088889
:100E1000364880F3098836483649086040F20000B9
:100E2000CCF200004EF63471CEF200010860BFF340
:100E30004F8FBFF36F8F40F20000C0F2F0004EF60C
:100E40008851CEF200010860BFF34F8FBFF36F8F60
:100E50004FF00000E1EE100A4EF63C71CEF20001B8
:100E60000860062080F31488BFF36F8F69F146F99C
:100E700067F172FE4FF055301F491B4A91423CBF4B
:100E800041F8040BFAE71D49184A91423CBF41F86A
:100E9000040BFAE71A491B4A1B4B9A423EBF51F812
:100EA000040B42F8040BF8E700201849184A914255
:100EB0003CBF41F8040BFAE769F162F967F184FF7E
:100EC000144C154DAC4203DA54F8041B8847F9E77B
:100ED00002F0A6FC114C124DAC4203DA54F8041B8C
:100EE0008847F9E769F14AB900060030002200306E
:100EF0000000020808ED00E00000003000060030AD
:100F0000285A1E0800220030703100307031003045
:100F100064420230E0020208680302086803020823
:100F2000680302082DE9F04F2DED108AC1F80CD0AE
:100F3000D0F80CD0BDEC108ABDE8F08F002383F30D
:100F400011882846A047002067F134FBFEE767F1CF
:100F500033F900DFFEE7000070B54FF0FF0C4CF4F2
:100F6000E06C1CEA11541DBF1CEA135594EA0C0FE7
:100F700095EA0C0F00F0DEF82C4481EA030621EA22
:100F80004C5123EA4C5350EA013518BF52EA03355D
:100F900041F4801143F4801338D0A0FB02CE4FF00F
:100FA0000005E1FB02E506F00042E0FB03E54FF03F
:100FB0000006E1FB03569CF0000F18BF4EF0010E37
:100FC000A4F1FF04B6F5007F64F5407404D25FEA33
:100FD0004E0E6D4146EB060642EAC62141EA5551E6
:100FE0004FEAC52040EA5E504FEACE2EB4F1FD0C28
:100FF00088BFBCF5E06F1ED8BEF1004F08BF5FEAA6
:10100000500E50F1000041EB045170BD06F0004657
:1010100046EA010140EA020081EA0301B4EB5C0404
:10102000C2BFD4EB0C0541EA045170BD41F48011FC
:101030004FF0000E013C00F3AB8014F1360FDEBF21
:10104000002001F0004170BDC4F10004203C35DAFD
:101050000C341BDC04F11404C4F1200500FA05F380
:1010600020FA04F001FA05F240EA020001F0004221
:1010700021F0004110EBD37021FA04F642EB060197
:101080005EEA430E08BF20EAD37070BDC4F10C04C1
:10109000C4F1200500FA04F320FA05F001FA04F285
:1010A00040EA020001F0004110EBD37041F1000171
:1010B0005EEA430E08BF20EAD37070BDC4F120057C
:1010C00000FA05F24EEA020E20FA04F301FA05F2E4
:1010D00043EA020321FA04F001F0004121FA04F28C
:1010E00020EA020000EBD3705EEA430E08BF20EA5C
:1010F000D37070BD94F0000F0FD101F00046400096
:1011000041EB010111F4801F08BF013CF7D041EA17
:10111000060195F0000F18BF704703F0004652001B
:1011200043EB030313F4801F08BF013DF7D043EAEC
:101130000603704794EA0C0F0CEA135518BF95EAA2
:101140000C0F0CD050EA410618BF52EA4306D1D129
:1011500081EA030101F000414FF0000070BD50EA48
:10116000410606BF1046194652EA430619D094EAD2
:101170000C0F02D150EA013613D195EA0C0F05D1BC
:1011800052EA03361CBF104619460AD181EA030110
:1011900001F0004141F0FE4141F470014FF00000C8
:1011A00070BD41F0FE4141F4780170BD4FEA41024B
:1011B00012F5001215D211D56FF47873B3EB6252A9
:1011C00012D94FEAC12343F0004343EA505311F0D0
:1011D000004F23FA02F018BF404270474FF0000062
:1011E000704750EA013005D111F0004008BF6FF0A0
:1011F000004070474FF00000704700BF4FEA4102C7
:10120000B2F1E04324BFB3F5001CDCF1FE5C0DD964
:1012100001F0004C4FEAC0024CEA5070B2F1004FAE
:1012200040EB830008BF20F00100704711F0804FB1
:1012300021D113F13872BCBF01F00040704741F476
:1012400080114FEA5252C2F11802C2F1200C10FA7A
:101250000CF320FA02F018BF40F001004FEAC1235E
:101260004FEAD32303FA0CFC40EA0C0023FA02F302
:101270004FEA4303CCE77FEA625307D150EA0133D8
:101280001EBF4FF0FE4040F44000704701F00040A8
:1012900040F0FE4040F40000704700BF01F0FF0145
:1012A000102A2BDB10F0070F08D010F8013B013A91
:1012B0008B422DD010F0070F42B3F6D1F0B441EAC3
:1012C000012141EA014122F007047FF000070023D9
:1012D000F0E80256083C85EA010586EA010685FA2F
:1012E00047F5A3FA87F586FA47F6A5FA87F68EB989
:1012F000EED1F0BC01F0FF0102F0070232B110F8AC
:10130000013B013A83EA010313B1F8D10020704791
:1013100001387047002D06BF35460338073815F0F1
:10132000010F07D1013015F4807F02BF013015F4A1
:10133000C03F0130F0BC0138704700BFEC46A0E868
:10134000F05F4FF000007047B0E8F05FE54608003E
:1013500008BF0120704700BF10F8012B11F8013BB6
:10136000012A28BF9A42F7D0D01A7047034613F8D3
:10137000012B002AFBD1181A01387047A8B110B50B
:1013800004460AE000F096FA14F8041C54E903033A
:101390001B1AB3FBF1F200F08DFA204654F80C3B17
:1013A000082201210133EDD110BD70472DE9F04F26
:1013B0000023A7B00293C36A009013F0040FD0E992
:1013C000002118BF0A46D9064FF0E021D3694CBF6F
:1013D00002F1200002F168000192DB0903F004032E
:1013E00003430393D1F8883D03F4A003B3F5A00FA2
:1013F00001D10123029393694FF004094F4D4FF03F
:1014000001081B884E4C03F47F43A3F53E43B3FA17
:1014100083F35B09049329E000F040F9FFF7AEFF86
:101420004FF0E023D3F8003D03F47023B3F5402FD1
:101430000ED0444A4FF0FF3305A88DF81C9005925A
:1014400014328DF828800692CDE90833FFF796FF15
:101450002B68A34206D03C4B0422012105A805932A
:1014600000F028FA00F070FB00285ED103A82C6081
:1014700000F00CFC04220121344800F01BFA042285
:10148000012102A800F016FA10220121019800F0B3
:1014900011FA0098202201210C3000F00BFA01987B
:1014A00004220121103000F005FA0422012103A8D2
:1014B00000F000FA01980C220121143000F0FAF932
:1014C0000C220121009800F0F5F9029BDA07A3D560
:1014D000009BDB6ADB0622D415A80DF1140AFEF787
:1014E00061FFDDF804E0D4460EF120060EF1600B3A
:1014F0003068103656F80C1C674656F8082C0CF16C
:10150000100C56F8043C5E450FC7F1D1DEF8603090
:10151000259384225046012100F0CCF97CE70DF19F
:10152000140A5046FEF738FFF3E7049B1BB1019AFB
:1015300093690233936127B0BDE8F08F70310030BA
:10154000ED55CEAC28ED00E0ACCE55ED3443190896
:1015500038B527206D2564F1A9FE144B144A4FF0CD
:10156000FF34D3F890100D2041F48021C3F890107F
:10157000D3F8901021F48021C3F89010D3F8901084
:10158000D3F8E81041F48021C3F8E810D3F8101123
:1015900041F48021C3F810110121D3F81031054B1B
:1015A000D56014621060197038BD00BF0044025845
:1015B000004800409C330030002953D02DE9F84FFB
:1015C000074689460026284DDFF8A480274C17F8E7
:1015D00001AB2B784FEA1A1218F802B0002B3CD05E
:1015E000C4F828B0E369580604D468F14DFDE369F6
:1015F0005906FAD50AF00F0A2B7818F80AA04BB34F
:10160000C4F828A0E3695A0604D468F13DFDE369F3
:101610005B06FAD50136B14522D03107D7D12B78F8
:101620004FF00D0BDFF84CA08BB1C4F828B0E36984
:101630005A0604D468F128FDE3695B06FAD51AF866
:1016400001BFBBF1000FC2D02B78002BEDD1FFF70B
:101650007FFFEAE7FFF77CFFD2E7FFF779FFBFE7FD
:10166000BDE8F88F704700BF9C3300300048004051
:10167000BC4319087C9A1A08014B1868704700BFD0
:10168000FCFF1F08014B0248C01A7047A0691E08E2
:101690000000200800487047A0691E08774943F6FB
:1016A0009822774B09682DE9F04F0A441B7883B0E4
:1016B000744F02EB030966F17DFC734B044600286E
:1016C00000F0C8800225FF1ADFF8E0810126DFF86C
:1016D000CCB130E01846019168F1C6F801990028B4
:1016E00036D1206AAA460AF101030AEB4A0E04F138
:1016F0003C058944DBB201440BEB8E0CB94503EB8E
:1017000043034BF82E40CCF804500AF102058CF844
:1017100008600BEB830CEDB24BF823008CF80860EB
:10172000CCF8041023D2204666F154FC044600286D
:1017300035D04E2D33D8206A404505D0211AE369B3
:10174000002BC7D1AA46CEE7504BA3EB0801F6E722
:1017500005EB450C01350BEB8C005FFA85FA067240
:10176000E3694BF82C300D334360206ABBE74F2D03
:1017700063D94FF0FF330122CBF8B4338BF8BC238D
:10178000CBF8B833424B1B782BB1424A424B12681C
:101790001B68CBE90023414803B0BDE8F08FB7EBED
:1017A0000900E4D44E2DE2D80AF1030A3C4EDFF8DA
:1017B00000C15FFA8AFAA6EB0C03BAF14E0F51464C
:1017C00094BF0024012483422BDC05EB450503EB89
:1017D000090201200BEB85034BF825C05E601872EF
:1017E000BA1A12D48CB92F4801EB41052E4BC41AFA
:1017F000944224DD1A440AF101014BF825300BEB29
:101800008503C9B25A6001221A7201EB41054FF0FB
:10181000FF3201210BEB85034BF8252019725A602A
:10182000B0E705EB4505012260440BEB85034BF85F
:1018300025C01A723A465860D2E72946E5E70AF110
:10184000010101224BF825300BEB8503C9B258602A
:101850001A72DAE7FF1AB7EB09000BD4104E4FF0FB
:10186000030ADFF84CC00225DFF830B05146A6EB82
:101870000C03A8E70221DFF824B0C6E78C33003060
:101880006433003000002008A0691E0800220030E8
:1018900000220030903300308833003004220030C2
:1018A000644202300000043068420230000600301A
:1018B000703100309A4B1B782DE9F04F824685B08D
:1018C0000E4693462BB9974B1B782BBB05B0BDE852
:1018D000F08F022900F0EE80042900F0B580012984
:1018E00000F0AE80904D2B780D27DFF858828F4C9A
:1018F0007BB1A762E3695A0604D468F1C5FBE369CA
:101900005B06FAD518F8017F002FDCD02B78002B6E
:10191000EFD1FFF71DFEECE7854B4FF00009854A3C
:101920009B1A0093CB45D1D0834F844C38682578DF
:10193000031D009A2B44934279D2202D51D0022EC0
:1019400024D0042E0DD0012EECD12378DFF8F081C5
:101950005A1C22701AF8092009F1010908F803201D
:10196000E0E7DFF8DC810025434620789AF8001094
:10197000421CE9400835D2B208F80010202A227033
:1019800018D0202DF1D109F10109CBE725789AF87B
:101990000030DFF8AC8108F805300135EDB2202DBC
:1019A000257030D06B1C09F101092370002308F861
:1019B0000530B7E738685F4901920844194667F176
:1019C000F3FC39684FF00003019A203123705C4B1F
:1019D0003960002118466EF12BF868F155FB584B21
:1019E000CFE7544B2A465649184467F1DDFC3B6863
:1019F00000212A462033524821703B606EF118F8CE
:101A000068F142FB9BE74B4B2A4638684146184435
:101A100067F1CAFC3B6800212A462033404621700A
:101A20003B606EF105F868F12FFB2578BAE7444A70
:101A30004FF0FF312023D161237005B0BDE8F08F56
:101A40001146FFF7B9FD4DE7002A3FF44BAF0246C0
:101A50000027354D0DF10C0852F8043B334C009231
:101A600003930191013704214046FFF7A5FDBB45D3
:101A70001ED0009ABE0752F8043B00920393F1D1A6
:101A80002A780D26DFF8BC907AB1A662E369580681
:101A900004D468F1F9FAE3695906FAD519F8016F27
:101AA000002EDFD02A78002AEFD1FFF751FDECE7B6
:101AB000019E18E7002A3FF415AF024600271A4D91
:101AC0000DF10C0832F8023B184C0092ADF80C30C6
:101AD0000191013702214046FFF76EFDBB45E7D07B
:101AE000009A790732F8023B0092ADF80C30F0D141
:101AF0002A780D26DFF84C907AB1A662E3695A067F
:101B000004D468F1C1FAE3695B06FAD519F8016FEC
:101B1000002EDED02A78002AEFD1FFF719FDECE77E
:101B200065330030002200309C3300300048004014
:101B300000002008A0691E088C3300306433003098
:101B4000683300307C9A1A08F8B5324B1A782AB9F3
:101B5000314A1078F0B901221A70F8BD2F4E0D25C8
:101B60002F4F304C3B7893B1A562E3695A0604D4F9
:101B700068F18AFAE3695B06FAD516F8015F002D71
:101B8000F0D1294B5868003818BF0120F8BDFFF785
:101B9000DFFCE9E7254D264E2B68264C26481A1D0A
:101BA0003178241A0A44A24206D239BB9C421CD87E
:101BB000002067F1AFFCE4E7204A4FF0FF31D1612C
:101BC00020223270184420221C4967F1EDFB2A685C
:101BD0003378002119481344202231702B606DF1B5
:101BE00027FF68F151FA2B68E0E7144920221448D6
:101BF000CB6167F1D9FB68F147FAD9E703F120021D
:101C00009442DFD81F29DDD80C4AD36120223270DC
:101C1000D8E700BF65330030002200303843190890
:101C20009C33003000480040943300308C33003047
:101C30006433003000002008A0691E0868330030BB
:101C4000E0FF1F080E4B1B7810B5B3B164210020D4
:101C50000C4A0D4CD3699B06FCD5536ADBB28B4210
:101C60004FF0640101D00020F4E70130C0B20E282B
:101C700001D0015DEEE7002010BDFFF769FCE5E74C
:101C80009C33003000480040484319082DE9F041DA
:101C900002680646EFF30581D9205369C9B2FBF00B
:101CA0002FFF674B1B782BB9664C2378002B37D15D
:101CB000BDE8F081644B0D27DFF8B081634D644CC3
:101CC00096E8030083E803002B7833B3A762E36947
:101CD0005F0604D468F1D8F9E3695806FAD518F814
:101CE000017F002FF0D173680BB32B784227DFF808
:101CF0008081574C73B1A762E369590604D468F137
:101D0000C3F9E3695A06FAD518F8017F1FB32B7897
:101D1000002BF0D1FFF71CFCEDE7FFF719FCD5E72E
:101D20003568002D47D100232370BDE8F081DFF82E
:101D300044814327464C2B78002B6AD0A762E36985
:101D40005B0604D468F1A0F9E3695F06FAD518F8D8
:101D5000017F002FEFD1DFF8208120273C4C2B782A
:101D6000002B53D0A762E369580604D468F18CF9BC
:101D7000E3695906FAD518F8017F002FEFD1FFF774
:101D800061FF2B78DFF8F4800D27314C83B1A76217
:101D9000E3695A0604D468F177F9E3695B06FAD57A
:101DA00018F8017F002F3FF47FAF2B78002BEED186
:101DB000FFF7CEFBEBE7284667F156FD0028B2D0CF
:101DC000284667F179FD00F21450854231D3214B4A
:101DD000A5F214521A60284667F184FD05F5E05318
:101DE000834220D81C4A136000231C481C4A03600D
:101DF0001C481D49801A0B7002D10DE083420BD2A2
:101E000052F8041B04330131F8D08CE7FFF7A0FB34
:101E1000A8E7FFF79DFB91E768F136F90120BDE8DF
:101E2000F04167F177BB284667F15CFD0A4B18600B
:101E3000DAE7284667F140FD064B1860CBE700BFA4
:101E40006533003000220030943300309C33003082
:101E50000048004090330030883300308C3300302D
:101E6000A0691E0800002008643300305843190898
:101E700060431908B44319086C4319087C9A1A087E
:101E800000207047036800221B681847614AF0B5BC
:101E9000B2F9DC3291B005460E4623B9B2F8DA1237
:101EA0000BB2A2F8DC129BB2632B40F28D800127AB
:101EB0000021594C2E2204A803916DF1B9FDD4F8EC
:101EC0000C03322103AA03681B689847002873D0CB
:101ED000B4F8E83241F65832A3F57A739BB29342D4
:101EE00006D94E4B3246202128460027DDF05AFE07
:101EF00094F92C35002B0DDD94F9E434002B53DCE0
:101F000094F89035A3B91F463246454B2021284608
:101F1000DDF048FE94F9E434002B09DD94F8153522
:101F200033B91F4632463F4B20212846DDF03AFEAA
:101F3000322303AA3C49D4F81803F0F08BF80028A8
:101F400053D0322303AA3949D4F81403EDF024FF07
:101F5000002840D020212846DDF01CFE50B1D4EDF1
:101F6000DA7A9FED337AF0EEE77AF4EEC77AF1EEA3
:101F700010FA0AD494F92C35002B03DD94F9D933E7
:101F8000002B3CD1384611B0F0BD94F92C35002B14
:101F900003DD94F89035002BF0D1264A31462846CF
:101FA0000027DEF065FAE5E7234B3246202128467C
:101FB0000027DDF0F7FDBBE7074603AB1F4A3146BC
:101FC0002846DEF055FA83E71D4A314628460027A9
:101FD000DEF04EFA6CE703AB074632462021009351
:101FE0002846184BDDF0DEFDB4E703AB074632466A
:101FF000202100932846134BDDF0D4FDA1E70027F4
:102000002846114B32462021DDF0CCFD384611B078
:10201000F0BD00BFB0330030B0C300300444190835
:10202000404419086844190890441908A84419083C
:1020300000000034AC44190818441908F843190882
:10204000D043190894441908C844190838B50446FF
:10205000DDF078FD114A124B156893F8C814002979
:1020600008BF0146E86A03681B6898478BF044F88C
:10207000EB6A93F89C1089F0FBFE94F8603003B98A
:1020800038BDFBF0B5FDEB6AD3F8A030C01AB0F54F
:10209000FA6FF5D3002384F8603038BDAC330030DC
:1020A000B0C3003070B50E4605469AF0C9F99AF0F3
:1020B000EBF820B10B4B93F91233012B02D0012422
:1020C000204670BD9AF0BCF9437A002BF7D19AF004
:1020D000B7F9847A002CF2D1034A31462846DEF063
:1020E000C7F9EDE7B073003004451908034BD3F886
:1020F0007C330BB101207047DDF0F6BCB0730030CB
:1021000070B50E460546FFF7CDFF0446314628461A
:10211000DEF028FB2040C0B270BD00BF2DE9F043C7
:10212000C57F91B005BB90F90430044603B39A4BC8
:102130000E461F68B86A03685B6B9847002800F07A
:10214000BC80A368CBB923683146944A20469B6B78
:10215000934240F0B880FFF7A5FF05463146204680
:10216000DEF000FB2840C5B2284611B0BDE8F08380
:102170000125284611B0BDE8F083FD6A884A2B6826
:102180005B68934240F0F6803146864F2046DFF090
:1021900003FB314605462046DEF00AFB97EDC97A7F
:1021A000D7EDC87A0540B4EEE77AEDB2F1EE10FA59
:1021B00004D597F91C33032B40F0D580F0EE087A54
:1021C00097EDB17AB4EEE77AF1EE10FA00F1C08043
:1021D000F0EE087A97EDB27AB4EEE77AF1EE10FA03
:1021E00000F1AB80F8EE087A97EDB37AB4EEE77AB7
:1021F000F1EE10FA00F38F80B7F9B032042B40F300
:102200008180DFF8E091D9F830079AF049F980B180
:1022100097F912336BB1D9F83037B7F91423B3F902
:102220000E309A4205DA604A314620460025DEF03B
:102230001FF931462046FFF735FF5C4B00EA0507E2
:1022400093F9AC234AB193F8F433002B00F09D804E
:1022500031462046FFF71AFE0740DFF88C8198F8D8
:10226000513B002B62D14FF48061514801F0CEFA0E
:1022700078B1D9F83037B3F90C30A3F2E24292B218
:10228000B2F5FA7F05D94B4A314620460027DEF0E9
:10229000EFF8494890F874323BBB00212E2204A885
:1022A00003916DF1C5FB03AA3221D8F83C0B0CF069
:1022B000D3FC054658B13D4656E7404A31462046D4
:1022C000DEF0D6F850E711B0BDE8F0431847D8F873
:1022D0003C0B03689B68984703AA0346314600926B
:1022E0002046374ADEF0C4F83EE700F51B7052F096
:1022F00079FC0028D1D10746324A31462046DEF02B
:10230000B7F8CAE7052231462046002500922E4A3A
:10231000DEF0AEF875E7B7EEC77A2C4A31462046B4
:1023200000258DED007BDEF0A3F865E7284A3146F5
:1023300020460027DEF09CF895E7B7EEC77A254ADD
:102340003146204600258DED007BDEF091F849E70F
:10235000B7EEC77A204A3146204600258DED007B36
:10236000DEF086F834E71D4A314620460025DEF0CF
:102370007FF823E72846984700283FF405AF95F8F3
:102380004D50002D7FF4F0AEFEE6154A3146204652
:102390001F46DEF06DF860E7AC3300300121020823
:1023A000811E0208B0730030D8451908B0C3003050
:1023B000B033003018461908B0B30030144519087E
:1023C0008C411A0840461908B8451908944519085F
:1023D0000046190870451908504519082C45190878
:1023E000E0441908B0830030B0A3003070B590B05D
:1023F00005460E46DEF09EFA044610B9204610B09F
:1024000070BD10212846DDF0C5FB0028F6D0002164
:102410002E2204A803916DF10BFB22F057FD32230D
:1024200003AA012121F01EFF04460028E6D103A9DA
:10243000034B3246284600911021DDF0B3FBDDE767
:102440005446190870B504460D4681B990F91060DC
:102450000EB9304670BD1B4818F0BAFFB0EEC00A86
:10246000DFED197AB4EEE70AF1EE10FA22D5A3688F
:1024700013B90126304670BD144B154A1B68DE6A3D
:1024800033685B68934205D129462046BDE8704019
:10249000DDF018BD304698470028F5D096F84D601D
:1024A000002EF1D098F074FB0A4A04218EF01EFD34
:1024B000304670BD084A012120462E46DDF0D8FF87
:1024C000C7E700BFB033003000000034AC33003049
:1024D000811E0208744619086046190838B5054679
:1024E000DFF08AFA044608B9204638BD104808F0E3
:1024F00099FC98B92846FFF7A9FD0E4B0E481B68BA
:10250000DB6A93F89C1012F035FD012328460B4935
:1025100085F86030DEF0E2FF204638BD0849094802
:1025200022F096F80028E5D0014801F04FF9E1E7E4
:10253000B0330030AC33003090C6003098461908F4
:102540000CC5003030580030F8B505460E46174629
:102550001AB1232937D0012935D93A4631462846C0
:10256000DFF0D2FA0446002840D0274FD7F83C0BC2
:1025700007F50863984205D003F6EC1050F060FBB5
:10258000D7F83C0B0368214E9B6B984786F84002B6
:1025900006F58056D6F83033012B2AD02846FFF7AF
:1025A00055FD1B4B1B481B68DB6A93F89C1012F00F
:1025B000E1FC4FF0FF3328461749C7F8743BDEF0C3
:1025C0008DFF2046F8BD15480BF0D4FC044668B9D1
:1025D000002EC2D195F91030022BBED098F0D8FA57
:1025E0000F4A06218EF082FC2046F8BD00242046CA
:1025F000F8BD99F025FF54219BF0D2F90028CDD1E8
:10260000C6F83003CAE700BFB0A30030B0B3003053
:10261000AC33003090C60030C0461908B0330030EB
:10262000A84619082DE9F047DFF864910746884667
:102630002DED028B90B0DDF0E3FC99F9E742054601
:102640004CB14B4C94F8F433F3B9284610B0BDECC0
:10265000028BBDE8F087BD21464853F041FB0028BE
:102660007CD1BC21434853F03BFB0028E9D0404CCF
:102670004246414B4FF4804138460025DDF092FA46
:1026800094F8F433002BE0D0A4F5805304A8B3F8F9
:10269000A0620023CDE90233CDE90433CDE906334E
:1026A00008932BF04DFA012ECFD9DFF8E8A0DFED2B
:1026B000338AA244012411E001340DF1240E0DF1FE
:1026C000080CA4B2BEE80F00A642ACE80F009EE8DA
:1026D0000700ACE803008CF80020B6D00BA82BF064
:1026E0002FFA09AA2146234850F05AFC03462448F1
:1026F000002BAAD0BDF826100AF06AFC0028DBD017
:10270000BDF80A30102BD7D104A90BA82BF004FC7C
:10271000B7EEC08B9AED000A1A48B4EEE80AF1EE63
:1027200010FAB8BF99EDAD0A20EE000A13F034FE9E
:10273000B6EE087A20EE077AB4EEC78AF1EE10FA08
:10274000BAD5B7EEC77A104B42464FF480413846AF
:1027500000258DED007BDDF025FAADE70B4B424601
:102760004FF4804138462546DDF01CFA79E700BF7A
:10277000B0C300301CB60030004719080000003418
:10278000B033003090C6003034471908D4461908D9
:10279000B073003058C8FFFF00207047014800F0B8
:1027A000DBBE00BFB033003090ED080A704700BFB9
:1027B00003685B68184700BF1CF058BFABF0D8BF78
:1027C00099F0C0BC08F02CB946F0DABC89F00CBD19
:1027D0000BF03EBD86F074BF11F07AB81AF062BA01
:1027E00004F05ABB85F0BEB827F0F4BF9EF02CBCB5
:1027F0009DF074BE1AF0DABB77F06EBBACF0C0B9D6
:1028000018F078BE26F01ABEAFF0B8B896F0E0BD6A
:1028100097F04ABC0AF0DEBD06F0F2BD10F088BAAF
:1028200010F0FEB91AF02CB81AF09EBC18F098BC43
:102830001AF066B901F060BE00F63C102DF034B815
:10284000034649F2C00003F5E0421844D2F8601B89
:10285000E4F00EBE0BF0C6B970B50C46A1F1040150
:1028600048F6805682B0B1FA81F10546064449091E
:1028700030460191F3F042FD01993046F3F03EFD00
:10288000042C11D005F50046D6F84832012B01D1B1
:10289000032C1FD0072C0DD02846C6F8484202B0A2
:1028A000BDE8704004F05ABC134805F50046BCF082
:1028B000DDF9F1E7D6F8682145F61C700F4B284486
:1028C00083FB0213D2170521C2EB63130C4A8EF06F
:1028D0000DFBE1E749F26C202844DDF03DF90028CA
:1028E000DAD028460BF046FB0028D5D045F25C40F4
:1028F0002844BCF0B5F9CFE70C8800301F85EB51B8
:10290000C8471908034645F27C40DFED087A03F515
:10291000A042184402F26C7392F8501793ED000A2B
:1029200001F0010120EE270AF8F0A6B80000C84225
:1029300000F5E04310B50446D3F83C0B03689B6DEB
:102940009847014647F67C202044BDE81040F8F047
:1029500029BD00BF38B50F4D044600F5567038F05C
:10296000FBFD29460C4822F03DFA04F5E0430246FF
:1029700004F5125004F5104405F13C0183F86D2B69
:1029800021F00AFED4ED667AF1EE677AC4ED667A3C
:1029900038BD00BF0CC500303058003010B50446BB
:1029A0002DF0BCFA90F925305BB190F8443343B177
:1029B00094F964392BB1064B1B68DB6A93F89C30A1
:1029C00003B110BD04F63C10BDE810402CF006BE6B
:1029D000AC33003010B4044C31200C60082110706E
:1029E0005DF8044B19607047D04C1908F8B50446DF
:1029F00049F26C2004F512552044FFF727FB002113
:102A0000284622F039F9802120461AF075FD002869
:102A10005FD104F580439FED347A04F5A04649F276
:102A20002850D3EDB17A06F24477204467EE877AD6
:102A3000FDEEE77A17EE902AC6F84027D3F8CC329D
:102A40003B601BF019FAC8B9D6F8403795ED937A78
:102A500007EE903AF8EEE77A67EE877AFDEEE77ACE
:102A600017EE903AC6F84037D5ED927A97ED007A96
:102A7000F0EEE77A67EE877AC7ED007A42F2B87136
:102A800004F5004605F5457021444FF0DDF994ED5D
:102A9000D47AD6ED587AE7EE007AB7EEE70AC6EDBB
:102AA000587A49F015FBB7EEC00B49F2E02086EDED
:102AB000580A204411F05EFF49F2EC200021204426
:102AC000E8F07CFB4FF4001120461AF015FD28B900
:102AD000F8BD48F0C9FD45F0DDFA9AE72846BDE8A3
:102AE000F8401FF059BE00BF0000C842FFF77EBF8C
:102AF00070B500F5E04349F2E02504460544D3F8FB
:102B00003C0B03689B6B98470646284617F0D4FC9D
:102B100030B904F5004393F89F31012B00D08EB9F2
:102B2000284614F0B7FA38B904F5104494F8F43391
:102B30003BB194F8213423B12846BDE8704014F02D
:102B4000C1BA70BD45F2E8702044E6F0F7FBE7E754
:102B5000FFF7CEBF10B54FF4801104461AF0CCFC3D
:102B600070B1022120461AF0C7FC04F512501FF084
:102B70000BFD4FF4805120461AF0BEFCD0B910BDB9
:102B8000012120461AF0B8FC0028EAD10221204693
:102B90001AF0B2FC0028ECD0204604F077F804F5D7
:102BA00012501FF0F1FC4FF4805120461AF0A4FCA3
:102BB0000028E4D049F2E8102044BDE810409EF01F
:102BC00007BE00BFFFF7C6BF38B504464FF48011FB
:102BD0001AF092FC0121054620461AF08DFC80F087
:102BE0000103DBB203B9A5B3102120461AF084FC1F
:102BF00008BB202120461AF07FFCA8B94FF40051F1
:102C000020461AF079FC58B9802120461AF074FC4D
:102C100000B938BD48F028FDBDE8384045F060BA3D
:102C2000204604F041FBEFE7204604F01BFA204663
:102C300004F058FBE2E7204604F04CF94FF4800121
:102C400020461AF059FC40B104F5E650CCF03CFDAA
:102C5000CFE7204604F01AF8C6E748F005FD45F036
:102C600049FBF1E7FFF7B0BF484B1B68DB6A93F8FD
:102C70009C30002B00F089802DE9F04100F50055D3
:102C8000044695F889370BB9BDE8F0810BF072F96D
:102C90000028F9D043F6E40604F54057264497F897
:102CA0003A1A30461FF022FA0028EDD094F8F9269F
:102CB00094F86436002AE7D14FF0B00808FB0343CC
:102CC00093F84124022ADFD903F25C43F1EE007A43
:102CD00093ED007AB4EEE77AF1EE10FAD4D497F8D7
:102CE0003A1A30461FF068FB04F58042B2F9B03260
:102CF00007EE903AB8EEE77AB4EEC07AF1EE10FA49
:102D00000EDD94F86436F8EE677A08FB034303F2AD
:102D10005C4393ED007AF4EEC77AF1EE10FAB3DC7F
:102D2000D5F8783604F5A041002BD1F84007B8BF9C
:102D30005B428342A8DC05F27C6392EDB27ADFED60
:102D4000146AD3ED007A27EE267AF8EEE77AF4EEED
:102D5000C77AF1EE10FA97DC01F2447191ED007A36
:102D600067EE266AF4EEE67AF1EE10FA8CD494F867
:102D70006416B0233046B2F9B22203FB0141BDE82C
:102D8000F04101F274411EF01BBC7047AC330030BF
:102D90000000C842FFF768BF70B504463B4A94F88C
:102DA0006436106804EB0311D1F8141488422AD059
:102DB00094F8F90660B104F5E04393F86C2B12B176
:102DC000052283F86C2B2046BDE8704010F0C0BA95
:102DD000B02000FB034090F841040228EBD904F531
:102DE000E045116095F86C2B012A1CD9013A85F851
:102DF0006C2B42F6BC00204424F0BEF82046BDE80F
:102E0000704010F0A5BA94F8F926002AD3D1B02268
:102E100002FB034393F84134022BCCD92046BDE892
:102E2000704010F095BAE4D104F51046D6F864214C
:102E300032B9D6F868211AB9052385F86C3BD8E772
:102E4000134A14491268D06A026852688A4217D13C
:102E5000B022204602FB034303F24C4108F05EF827
:102E6000D6F8483106F5A67C4FF0000E06F5B6768A
:102E70000FCB8CE80F0086E80F0085F86CEBB8E705
:102E800090470028B5D194F86436E1E7A0330030CC
:102E9000AC330030811E0208FFF77EBF38B500F565
:102EA0001045044695F8F43373B904F5004393F8DC
:102EB0009F21F2B9D3F84832042B20D004F50054F6
:102EC000012384F8893738BD49F2285020441BF08B
:102ED000A5F80028F2D149F2E020204414F0DAF8F5
:102EE00038B995F8F433002BDFD095F82134002B56
:102EF000DBD004F50054002384F8893738BD48F648
:102F00008050204404F50054F3F05CFA84F88907FB
:102F100038BD00BF10B500F5E04400F5F143D4F82A
:102F20003C2B9A4219D047F6242303449A4200F5D9
:102F300000431CBF4FF0FF32C3F858210849094A2B
:102F4000C3F84811C3F84C21FFF7A8FFD4F83C0B95
:102F50000368BDE810401B69184700F50043EDE722
:102F60000000C8420000C8C200F50043D3F8483250
:102F70008B4201D0FFF770BC704700BFF8B500F579
:102F8000E0460446D6F83C0B04F5004503689B6B0D
:102F90009847B8B195F84032A3B9D6F83C2B04F560
:102FA000F1439A4236D047F6242323449A4230D044
:102FB000D5F84832032B2CD020460321BDE8F84039
:102FC000FFF74ABC49F2E020204414F063F848B906
:102FD00004F5104393F8F423002AE9D093F8213440
:102FE000002BE5D0D5F84832022B12D048F6805697
:102FF000002126443046F3F081F930460021F3F0F9
:103000007DF902232046C5F84832BDE8F84004F0B7
:10301000A5B8F8BD49F2E020204413F0C5F8002817
:10302000E0D195F8986146B3B5F8AA32152BCFD107
:1030300095F8843D13F00101D5F8483243D1072BB0
:10304000E7D095F9262F002A45D1042BE1D048F688
:103050008056012126443046F3F050F930460121D4
:10306000F3F04CF92248BBF001FE04232046C5F8DA
:103070004832BDE8F84004F071B8D5F84832012B69
:10308000C7D048F68057314627443846F3F036F922
:1030900038463146F3F032F901232046C5F848326C
:1030A000BDE8F84004F05AB848F680502044F3F0E8
:1030B000FFF8D0B145F61C700E4A062120448DF071
:1030C00015FFD5F84832072BA3D020460721BDE8CD
:1030D000F840FFF7C1BB204618F07AF9DFED067A19
:1030E000B4EEE70AF1EE10FADEDAD5F84832ACE7D2
:1030F0000C880030EC4719080000B44238B5304C59
:1031000004F50863D4F83C2B9A422DED028B03D0D2
:103110000020BDEC028B38BD05462A48B0EE408A3F
:1031200013F042F870BB04F58055D5F84832042BF3
:1031300007D0B5F8AA12A4F5E04009F049FF00282D
:10314000E6D094F86D3B33BB1F4C94F8F43353BB7B
:10315000F0EEC87A9FED1D7AF4EEC77AF1EE10FA20
:1031600007D49FED1B0A28EE000ABDEEC00A85EDCC
:103170005A0A1848F3F09CF80028C9D0002385F8B3
:103180009B31C6E749F2E020BDEC028B2844BDE844
:10319000384017F041B91049A1F56F6053F048F875
:1031A0000028D1D0B5E704F5387012F0FDFF0028F3
:1031B000AED104F5387015F07DFE0028A8D1C7E720
:1031C000B0A3003090C60030B0C30030000000341F
:1031D0000000C84230C100300CC5003000F500438B
:1031E00010B5D3F8483282B00446042B05D000F560
:1031F000104494ED660A02B010BD01A907F0F6FA7A
:1032000018B19DED010A02B010BD204606F0EAFC9F
:1032100020468DED010A06F05DFEDDED017A37EE08
:10322000C00AE8E72DE9F04100F5F46504462DED0C
:10323000028B284688B024F085FF002305A904F5F9
:10324000125005930693079321F010FE002871D0C9
:103250009DED070A9FED607A04F50045DFED5F7A8A
:1032600048F2B84020EE070A95ED5E7A2044A7EEBA
:10327000270A85ED5E0AB0F083FF2046FFF77EFE49
:10328000204609F04DFD00284FD104F5E047D7F85E
:103290003C0B03689B6B9847064649F2E0202044AC
:1032A00017F00AF9002840D195F89F31012B3CD046
:1032B000DEB395F84032C3BBD5F84832042B6ED04C
:1032C0009FED478A204606F029FE04F5104247F696
:1032D000AC030646C2F854062344D7F83C1B994277
:1032E00042D0D7F8702B2046D5F84832039202938B
:1032F0001CF05AF9B7F97E8B07462046FFF76EFFA0
:1033000045F2E87095ED991AF0EE400A204404F574
:103310008044CDF80480B0EE480A00973146D4EDE1
:10332000D31ADDE90232E7F047FD08B0BDEC028BAD
:10333000BDE8F08194F8F92694F8643672B9B022A9
:1033400002FB034393F84124022A07D993F89024FF
:1033500022B103F27C4393ED000A7BE7284624F078
:1033600083FBB1EE400A75E792F8E031002BB8D14B
:1033700004F5A043B3F90C37002B26DDD2F8481131
:103380000A334868D2F85011091A642000FB03F38D
:10339000B142ACBF5E189E19C2F85466A1E749F26B
:1033A0005C1649F26C1849F24C112644A0442144A1
:1033B000424630462BF092FB002881D041463046F1
:1033C0002AF0AAFDB7EEC08B7CE70649D1F8541469
:1033D000C90686D5D2E700BFCDCC4C3ECDCC4C3F04
:1033E00000000000B0830030FFF71CBFF8B500F507
:1033F000E04247F63C13D2F83C2B03449A4210D0EB
:1034000049F2E02704460E46381813F043FE0546FD
:1034100050B904F500440125D4F8803128463360C2
:10342000F8BD00252846F8BD381912F059FE70B1D4
:1034300004F51044D4F81C0303689B689847DFED3B
:10344000057A20EE270A284686ED000AF8BD9FED92
:10345000020AF8E70AD7233C00000000F8B500F59F
:10346000E04247F63C13D2F83C2B03449A421CD06E
:1034700049F2E02704460E46381813F00BFE0546C5
:10348000B0B904F5C0440125D4F8840103681B6970
:10349000984707EE900A9FED107AF8EEE77A67EE0C
:1034A000877A2846C6ED007AF8BD00252846F8BD83
:1034B000381912F015FE58B104F51044D4F81C0365
:1034C0000368DB68984707EE900AF8EEE77AE8E7CA
:1034D000DFED027AE5E700BF0AD7233C00000000D9
:1034E000F8B500F5E04247F63C13D2F83C2B034414
:1034F0009A4218D049F2E02704460E46381813F0D5
:10350000C9FD0546A0B904F5C044114AD4F88401A8
:1035100003685B69934209D190ED080A01252846AA
:1035200086ED000AF8BD00252846F8BD9847F5E766
:10353000381912F0D5FD10B99FED060AEFE704F532
:103540001044D4F81C331869EDF05CFEE7E700BFC7
:10355000A92702080000000010B584B084466C461C
:103560000FC984E80F0040F279322146604607F027
:103570009FF90D4B03F51062D3F83C3B934202D008
:10358000002004B010BD9DF8001011F0040106D019
:103590002146064807F002FC012004B010BD204679
:1035A0002AF0D8FBF4E700BFB0A30030B0330030FE
:1035B00038B500F5E04305460C46D3F83C0B0368EC
:1035C0005B6898470F2803D8092806D8002038BD23
:1035D000A0F11303DBB2022BF8D849F26C132B4491
:1035E0000FCB84E80F00012038BD00BF2DE9F84360
:1035F00049F26C160C4605461746064420463146ED
:103600002BF0D8F920B94FF000084046BDE8F88308
:10361000314620462BF0DCF980460028F3D02046C6
:103620002AF0E4FA044638462AF0E0FA8442EAD165
:1036300049F26C1405F5E04997E80F002C4484E842
:103640000F0040F2B1323146284607F031F947F613
:10365000B013D9F83C2B2B449A4204D047F6901370
:103660002B449A42D1D1FAF0C3FAC9F8AC09CCE79D
:1036700070B549F2E02504460E460544284613F08D
:1036800009FD30B9284613F0EFFC034608B9184687
:1036900070BD04F5104496E8030004F5936383E8D5
:1036A0000300FAF0A5FA0123C4F8A004184670BD7F
:1036B00010B5044649F2E0202DED028B2044B0EE17
:1036C000408A13F0EBFA68B904F5E04147F6B0120E
:1036D0000346D1F83C1B2244914203D01846BDEC6E
:1036E000028B10BD04F5104404F2B44383ED008A4C
:1036F000FAF07EFA0123C4F8B8041846BDEC028B38
:1037000010BD00BF00B549F24C1E00F5004C8644C8
:103710000FC98EE80F0001208CF89C015DF804FBB6
:1037200010B50446064813F0B9FA40B904F5E04371
:10373000D3F83C0B0368BDE810409B6C184710BDE4
:1037400090C6003010B50446064815F00DFB40B990
:1037500004F5E043D3F83C0B0368BDE81040DB6C94
:10376000184710BD90C6003070B5044649F2E020FD
:103770000E461546204415F0AFF9D0B904F51252A3
:10378000D2F808322B6004F5A043D2F8042232604C
:10379000D3F854349B050BD404F58044D5ED007A5E
:1037A0009FED097AD4EDD36AE6EEC77AC5ED007ACB
:1037B00070BD04F51044D4F8A4359B682B60D4F890
:1037C000A4355B68336070BD35FA8E3C38B50D4D5D
:1037D00004460D48294621F005FB04F5E043024666
:1037E00004F5125004F5104405F13C0183F86D2BEB
:1037F00020F0D2FED4ED667AF1EE677AC4ED667AF7
:1038000038BD00BF0CC500303058003000F5A04076
:10381000D0F85434194214BF01200020704700BF73
:1038200038B5054C0A46054B0146246825682046F4
:103830002C68A047002038BDAC330030B0330030D6
:103840002DE9F0412DED028B0368044600F580451B
:1038500000F5A048D3F8BC3004F51046984745F26F
:10386000207195F98A2304F50047B8F84C342144B7
:1038700095EDCF0A8648AFF015FB96F82130B5F9E3
:10388000B022002B40F0DB8002EB82039FED817AB7
:1038900007F6387103EB83039B007382B5F9B232EC
:1038A00007EE903AF8EEE77A67EE877AC1ED397A5B
:1038B000D8F85414090600F1C980B5F8E22249F29B
:1038C0006C25754B2544DFF8D8811A709BF042FDBA
:1038D0009AF070FC00212846FEF720FC012388F8AE
:1038E0000600284688F80730DCF02CF9002800F0A4
:1038F000C88088F804000421204619F0FDFD002846
:1039000040F0B9802846DCF01DF960B994F86426CF
:1039100041F2883004EB0213D3F81414D6F8E431E2
:10392000CB1A834275D8B4F9DC3223B9B4F8DA2261
:1039300013B2A4F8DC22D4EDB90A9BB2DFED576ACA
:10394000B7EE007AB0EEE06A07EE903AF8EEE77A6A
:10395000B4EEE66A87EE270AF1EE10FA09D5B4F95B
:10396000DA3207EE903AF8EEE77AC7EE270AC4EDAE
:10397000B90A48F02FFA002842D0D4EDB90ADFED99
:10398000477AB0EEE07A94EDD40AB4EEE77AF1EE3D
:1039900010FA0BD5B4F9DA32B7EE007A07EE903AA6
:1039A000F8EEE77AC7EE270AC4EDB90A48F012FA32
:1039B00030B384F095F883F019FD96F8F433B0EE47
:1039C000408A23B1D6F8140303681B6F984745F665
:1039D000A420B0EE480A2044C7F014F945F60C4084
:1039E000B0EE480A2044C7F00DF9B0EE480A45F69B
:1039F0004C50BDEC028B2044BDE8F041C7F002B949
:103A000087F024FA40F27D124FF4801187F0D0F94C
:103A1000CFE794F8F936002B85D1B02303FB02429F
:103A200092F84134022B7FF67EAF2046C6F8E411AF
:103A300007F0F8F907F5586700233B6073E7D8F8FB
:103A40005414B5F9B23209067FF537AF991A04F567
:103A5000125048BF0131D31848BF013349105B10E1
:103A600007EE901A00EE103AF8EEE70AB8EEC00A38
:103A700020F02AFA21E748F2D840204485F0BCFF24
:103A800040E72846DDF03CFDB0FA80F0400930E721
:103A9000F4760130E5CFF83FDC2700300000003439
:103AA000B8CB0030FFF7CCBE70B500F5004595F9F6
:103AB000243F002B00DC70BD04460AF05BFA0028AE
:103AC000F9D149F26C263019DDF01AFD0028F2D048
:103AD0003019DCF037F80028EDD0FAF089F8D5F885
:103AE000882195F9243F801A4FF47A7202FB03F380
:103AF0009842E0D301221C213019FEF725FD002851
:103B0000D9D045F61C70034A06212044BDE8704018
:103B10008DF0ECB90C4819080020704700F5AC7026
:103B2000704700BF00F51370704700BF704700BFBB
:103B30000020704770B504460AF042F847F6CC13EF
:103B4000064604F5E0452344D5F83C2B9A4224D0A0
:103B500049F2E020204414F0A9FF20BBD5F83C0B2B
:103B600003689B6B984720B995F8503BEBB901204F
:103B700070BD124BD3F83C0B03685B6B9847002871
:103B8000F2D004F5804494F95903002818BF0328A3
:103B900014BF01200020304070BD04F5104393F89D
:103BA000C034022BD4D9002070BD04F5804494F9B0
:103BB0001C03023818BF012070BD00BFB0A3003045
:103BC00070B52DED028B82B0044600F5125001A9AC
:103BD00021F014F9002800F0C68004F50045DDED61
:103BE000016AD5ED5C7AF4EEE67AF1EE10FA00F1B6
:103BF000AD8004F580459FED817AB6EE005ADFED89
:103C0000804AB5F9B232F0EE005A95EDC16A18203B
:103C100007EE903AB5F9B032052BF8EEE77AB8BF67
:103C2000052377EEA77A04EE103AF8EEC48AC6EEC2
:103C3000270A28EE877A86EE071AF4EE450AF1EE97
:103C400010FA75FE200AB4EE651AF1EE10FAF4EEE1
:103C5000E46A48BFB0EE651AF1EE10FACCBF86EE0A
:103C6000260AB0EE410A48F073FA49F2E020B0EEBD
:103C7000408A204413F00EFA90B904F5104393F8EB
:103C8000F42312B193F8213453B95E481FF0FAFBC4
:103C9000002875D0B0EE480A02B0BDEC028B70BDB2
:103CA00049F26C202044DBF057FF0028EDD0B6EE3F
:103CB000002A9DED011A28EE822AB4EEC21AF1EE16
:103CC00010FAE2D5D5EDC10A04F5A045DFED4E1A94
:103CD00045F6A426C0EE820A9FED4C0A48F006F98C
:103CE00005F66C23DFED4A8A2644D3ED517A30463F
:103CF000B4EEC08A67EEA87AF1EE10FAC3ED517AFD
:103D000058BFB0EE408AC7F0B7F9304620EE280A17
:103D1000C7F0C8F905F53D6345F60C4605F6345580
:103D2000D3ED527A264467EEA87A3046C3ED527A34
:103D3000C7F0A2F9304620EE280AC7F0B3F9D5ED56
:103D4000597A67EEA88AC5ED598A9EE749F26C2038
:103D50002044DBF001FFDDED016A00283FF449AFAC
:103D6000C5ED5C6A45E749F26C202044DBF0F4FEC7
:103D7000E0B92448B7EE008A1FF084FB002889D1FF
:103D800040212448FFF742FD002883D0224BD3F87E
:103D90004832012B7FF47EAFF7EE007AB4EEE78A6B
:103DA000F1EE10FA58BFB0EE678A73E746209AF03A
:103DB00073FDF7EE007AB4EEE70AF1EE10FA14DDC7
:103DC0009FED167AC7EE007AF5EE407AF1EE10FA22
:103DD0000ED4B1EEE70A2F209FED111ADFED110A84
:103DE00048F0B6F9B0EE408A4FE7DFED0C7AF0E725
:103DF000B0EE670A68F1A0FFEDE700BF3333333F51
:103E000017B7D13830580030000000006F12833AE5
:103E100052B87E3FB0330030B0B3003000003442BF
:103E20008FC2D53F9A99193F10B5044698F008FB08
:103E30000368074ADB68934201D1002010BD984710
:103E40000028FAD02046BDE81040FFF773BE00BF3F
:103E5000193B020830B5044649F2E02004F5E0457C
:103E6000204405F68C332DED028B83B093ED008A50
:103E700014F064FE10B347F29073D5F83C2B234442
:103E80009A425BD0002204F5004304F5005145F648
:103E90006C25D1F878162544D3F85C4293F8583253
:103EA000641A002B3FD1B0EE480A2146284603B0E1
:103EB000BDEC028BBDE83040E2F066BB04F5104576
:103EC0003A4AD5F8140303689B6893426BD100F516
:103ED000AC73D5F8B42552023AD5D5F8142304F5BD
:103EE000A0459FED337AD2ED097AD2ED436A67EEB1
:103EF000A67AF4EEC77AF1EE10FA2BDB05F527620D
:103F0000F7EE006A92ED007A05F66C2267EE877A8A
:103F100086EEA77AB4EE667AF1EE10FA36FE877A6C
:103F200082ED4C7A16E04FF4006122480192FFF7CF
:103F30006DFC80F00100019AC3B2B4E704F5A04320
:103F4000D3F82837B3F90820003A18BF01229AE7BE
:103F500004F5A04545F66C2093ED280ADFED167AAE
:103F6000F0EE480A2044DFED158A20EE270A00F122
:103F70003804E2F005FB05F66C23B0EE408A2046DB
:103F8000D3ED517A67EEA87AC3ED517AC7F074F891
:103F9000204620EE280AC7F085F8B0EE480A03B0A4
:103FA000BDEC028B30BD9847034692E71D3B0208EB
:103FB00000000034B0330030E02E654252B87E3F3E
:103FC00038B5044609F05EF970B104F5004244F2D8
:103FD000506004F50053D2F85C120D18C2F85C5220
:103FE000D3F87836002B07DB2046FFF733FF042099
:103FF000BDE838409AF038BC091AC2F85C12F3E701
:104000002DE9F04349F2E02500F5E0460446054479
:1040100006F68C332DED028B284683B0D3ED008A53
:1040200014F08CFD00283ED104F51045724AD5F8F5
:1040300014030368DB68934240F0B28000F5137309
:10404000D5F8B425520200F1848004F5A04545F668
:10405000D03093ED280ADFED697AF0EE680A20444B
:10406000DFED678A20EE270A00F13C04E1F0A4FEB0
:1040700005F53D63B0EE408A2046D3ED527A67EEF7
:10408000A87AC3ED527AC6F0F7FF204620EE280A40
:10409000C7F008F8BDEEC80AB8EEC00A03B0BDEC20
:1040A000028BBDE8F08304F58049284612F06AF9D6
:1040B000DFED547A99EDD38A04F50048074646208F
:1040C00028EE278AD8F86032BDEEC88A18EE102A8A
:1040D0001A4408EE102A9AF0DFFBD9EDBD7A47F2B8
:1040E0009073B8EEC88AD6F83C0B2344A0EE278A1A
:1040F0009842FDEEC87A17EE905A5FD0002297B929
:10410000036801925B699847019A60B9D6F83C0B45
:1041100003689B6B9847019A28B904F51043D3F8BC
:104120004C36022B54D045F6D03698F858322644F7
:1041300004F50054D4F87C166D1AA3BBB0EE680ADF
:104140002946304603B0BDEC028BBDE8F043E1F0F8
:1041500029BFD5F8142304F5A0459FED2B7AD2EDA5
:104160000B7AD2ED446A67EEA67AF4EEC77AF1EEE6
:1041700010FAFFF66CAF05F6D431F7EE006A05F5DC
:104180003D6291ED007A67EE877A86EEA77AB4EE0B
:10419000667AF1EE10FA36FE877A82ED4D7A56E7AE
:1041A000984703464CE74FF4006118480192FFF727
:1041B0002DFB80F00100019AC3B2BFE704F5A043D4
:1041C000D3F82C37B3F90820003A18BF012296E73C
:1041D000204616F04DFF019A0028A4D008F604737B
:1041E0009FED087AD3ED007A67EE877AFDEEE77AE5
:1041F00017EE903A1DB296E7253B0208E02E654285
:1042000052B87E3F0000C84200000034B033003096
:1042100010B504461BF0D4F938B92046FFF7F0FE7C
:104220001320BDE810409AF01FBB03B2132003EB2C
:104230004303C3EB031300EE103ABDE81040B8EEA1
:10424000C00A9AF011BB00BF10B598F0F9F80368E6
:10425000144ADB68934200D110BD98470028FBD078
:104260001148FFF767FC0028F6D0104816F01AF93D
:104270000028F1D00E4C04209AF00EFBD4F8280749
:1042800098F048FB04209AF0EFFA13209AF004FB10
:10429000D4F82C0798F03EFB1320BDE810409AF0AC
:1042A000E3BA00BF193B0208B033003090C60030BB
:1042B000B0830030F8B52DED028B044698F0C0F8BD
:1042C00003688A4ADB68934202D1BDEC028BF8BDD9
:1042D00098470028F9D02046FFF72CFC0028F4D09E
:1042E00004F5E04547F2C872D5F83C3B22449342BE
:1042F000EBD047F6040222449342E6D047F664022C
:1043000022449342E1D047F6200222449342DCD07B
:1043100047F63C0222449342D7D047F65812224433
:104320009342D2D047F6741222449342CDD047F63E
:10433000901222449342C8D047F6B01222449342CE
:10434000C3D047F6EC1222449342BED049F2E0209B
:10435000204416F0A7F80028B7D047F2AC73D5F880
:104360003C2B23449A42B0D004F5A047D7F8280745
:1043700098F078F9F6EE007AB4EEE70AF1EE10FA6A
:1043800073DDB0EE087AFFEE007AE0EE077AB0EE69
:10439000670AD7F8402704F5004607EE902A5142F5
:1043A000B8EEE77AD6ED977AF8EEE77AE7EE007A9C
:1043B000FDEEE77A17EE900AC6ED977A47F0B8FF60
:1043C00047F6C803C6F85C022344D5F83C2B9A4252
:1043D00000F08280D7F82C0798F044F9F6EE007AC6
:1043E000B0EE408AB4EEE70AF1EE10FA4DDDB0EE21
:1043F000087AFFEE007AE0EE077AB0EE678A204690
:1044000008F040FF08B1B1EE488AB5EEC08AF1EE7F
:1044100010FA4ADD04F58044D6ED987A9FED346AAF
:1044200007F2447794EDB27AF8EEE77AD7ED006AB6
:1044300027EE088AE8EE067AFDEEE77A17EE900A94
:10444000DFED2B7AC6F8600227EE277A66EEA76AC0
:10445000FDEEC77A17EE902AFDEEE67A17EE901A77
:1044600047F066FFC6F860022FE7FEEE007AB4EE72
:10447000E70AF1EE10FA8CD5B0EE087AF7EE007A82
:10448000E0EE077AB0EE670A83E7FEEE007AB4EE5C
:10449000E70AF1EE10FAB2D5B0EE087AF7EE007A3C
:1044A000E0EE077AB0EE678AA9E707F24477D6ED27
:1044B000987A9FED0F6A04F58044D7ED006AF8EE14
:1044C000E77A94EDB27A28EE668AE8EE067AFDEE97
:1044D000E77A17EE900AB3E74FF480510548FFF7EB
:1044E00095F900283FF476AFEFE600BF193B0208CC
:1044F0000000C842B0330030F8B5044604F5104758
:104500002DED048BF9F074FB97F8F43305463BB1BD
:10451000D7F81C04714A03681B6A934240F0BC80C0
:1045200004F5E046D6F84C3BEB1AB3F5FA6F33D8F6
:1045300047F2AC73D6F83C2BC6F84C5B23449A4246
:1045400009D047F63C1323449A4204D0204608F091
:10455000E7FB00285FD1624BD3F83C0B03681B6874
:1045600098470021204616F033FFB0EEC00ADFED79
:104570005D7AB4EEE70AF1EE10FA0AD5D7ED667A65
:10458000B1EE047AF0EEE77AF4EEC77AF1EE10FAC3
:1045900007D4BDEC048BF8BDD6F83C0B0AF078FBD1
:1045A000C6E704F5F46023F05FFAF6EE007AB0EEA9
:1045B000C00AB4EEE70AF1EE10FAEAD542F6840535
:1045C000F0EE087A254495ED007AB4EEE77AF1EE44
:1045D00010FADED545F66C202044E2F051F845F69D
:1045E000D0302044E1F092FD45F634502044E2F012
:1045F0005BFDF7EE007A95ED007AB4EEE77AF1EE26
:1046000010FAC6D545F6B460BDEC048B2044BDE875
:10461000F840E2F05FBA06F68C3604F5004545F640
:104620006C2096ED009A204495ED6D0AF0EE490A53
:10463000E1F0A6FF45F6D030F0EE490AF0EE408AF0
:10464000204495ED6E0AE1F0B7FBB0EE408A0420FD
:10465000B0EE680A9AF008F91320B0EE480A9AF012
:1046600003F904F5A04393F94A3DEBB195ED738A44
:10467000DFED1D7A95F8D03128EE278A3BB345F659
:104680003450F0EE490A95ED6F0A00212044E2F023
:10469000E9FB38EE008A09E048F25C2248F260212A
:1046A0002244214498473BE79FED108AB0EE480A28
:1046B00015209AF0D9F8B0EE480A1A209AF0D4F8EA
:1046C0000B4B462093ED700A9AF0CEF849E745F679
:1046D00034502044E2F0E8FCE8E700BF2D3B02083C
:1046E000B0A300300000003400003442000000009D
:1046F000B0B3003000F58042034692F9A722012AA8
:104700000BDD45F2E872DFED077A46201A4492EDA0
:10471000290A20EE270A9AF0A7B89FED030A46203F
:104720009AF0A2B80000C842000000002DE9F04154
:1047300000F5E048054608F68C332DED028B93ED2D
:10474000008A16F053FA0646D8F83C0B03681B6A39
:10475000984728B1524CD4F8E831002B00F39080F0
:1047600005F5104305F5804493F84136ABBB47F29D
:104770009073D8F83C1B45F63457002E2B44B0EE0E
:10478000480A2F44A1EB03013846B1FA81F14FEA00
:10479000511108BF0021E2F0EBF9054604209AF020
:1047A0007BF894EDBB7A2BB207EE903AF8EEE77AFD
:1047B000E0EE077AFDEEE77A17EE904A344424B231
:1047C0003846E2F07DFC204641F294123549BDECBA
:1047D000028BBDE8F04147F0BBBDB4F93833002B84
:1047E000C5DD05F5A04393F94A3D002BBFD001215B
:1047F000284616F033FCDFED2C7A05F50046B4F9B7
:10480000383380EE277ADFED296AD6ED977A08EE05
:10481000903A9FED270AF8EEE77AF8EEE88A67EE1D
:10482000A67A27EE800A68EE878A67F1FDFFB4F961
:10483000B03245F6345096ED9A7AF0EE480A07EE1B
:10484000903A9FED1C6ADFED1C6A0021F8EEE77AD2
:10485000284420EE060AB4EEE77AF1EE10FA58BFCB
:10486000F0EE477A80EE277AB0EE680AA7EE260AC5
:10487000E2F0F8FABDEEC00A10EE103A1CB2A2E760
:10488000F9F0B6F9D4F8E831C01A40F6B7339842D7
:104890003FF666AF45F63457B4F9DC412F448FE755
:1048A000B0B300306CEEFFFF00A08C450AD7233C6C
:1048B00035FA8E3C0AE81C41E02E654238B500F519
:1048C000C0430446D3F884010368DB689847014677
:1048D00045F6B4602044E2F0DFF805B297F0B0FD91
:1048E0000368124ADB68934207D1284641F29412CA
:1048F0000F49BDE8384047F02BBD98470028F4D059
:104900002046FFF717F90028EFD007EE905A04F57C
:10491000A044B8EEE70AD4F8340797F0FBFFBDEEE9
:10492000C00A10EE103A1DB2DFE700BF193B0208C3
:104930006CEEFFFF30B5B02290F86436F7EE007AE7
:1049400083B002FB0303044603F25C4393ED007A59
:10495000B4EEE77AF1EE10FA6DD400F50045F9F007
:1049600047F9D5F864210346821AB2F57A7F3AD81E
:10497000C5F86431204616F039F9D5F8483201906F
:10498000012B34D0A3F10702B2FA82F2520972BBB2
:1049900007EE900A9FED3C6A04F58043DFED3B6A29
:1049A000F8EEE77AB3F9FC3287EE867A00EE103A39
:1049B000B8EEC00A27EE000AF0EEC07AF4EEE67A0E
:1049C000F1EE10FA58D445F6B46085F85C21204425
:1049D000E1F02AFF00B241F294122D4903B0BDE884
:1049E000304047F0B5BC002285F85C21C0E795F85F
:1049F0005C215AB90122934285F85C2106D0072B2D
:104A000004D000230021C5F860310DE0D5ED586ACF
:104A1000DFED207A9FED207A67EEE67A67EE877AFF
:104A2000FDEEE77A17EE901A45F6B4602044E2F006
:104A300033F800B2CFE7002104F5004516F0C8FCBA
:104A4000B0EEC00ADFED117AB4EEE70AF1EE10FA2B
:104A500085D5D5F84832072B81D0012B3FF47FAFA5
:104A600000220023204685F85C21C5F8603103B0A0
:104A7000BDE8304016F0BAB895F85C31002BC5D1CE
:104A8000012385F85C31BCE700A08C4500000034B0
:104A90006CEEFFFFE02E65420000C84270B548F69C
:104AA0008055044605442DED028B284682B0F1F076
:104AB00053FB58BB04F5A0430646D3F82837B3F997
:104AC0000830002B56D02846F1F060FB002867D054
:104AD0002846F1F041FB00286BD104F50043D3F8E0
:104AE0005831013377D0DEB92046FFF71FFE07EEBD
:104AF000900AB8EEE70A15208DED010A99F0B4FE90
:104B00009DED010A1A2099F0AFFE29E02846F1F048
:104B100023FB28B904F50043D3F8583101335CD0A6
:104B20002046FFF7CBFE08EE100A2046FFF7FEFDF9
:104B300007EE900AB8EEC88AB8EEE70A1A208DEDA3
:104B4000010A99F06FFC9DED010A08B9B0EE480A20
:104B5000152099F089FEB0EE480A1A2099F084FEDB
:104B600049F26830204402B0BDEC028BBDE87040D1
:104B700004F00EBB04F5104204F580432846D2ED44
:104B8000667A93EDBE7AF0EEE77AF4EEC77AF1EE4C
:104B900010FA4CBF01260026F1F0F8FA002897D150
:104BA0002846F1F0D9FA00289ED02046FFF786FE6D
:104BB0009AE72046FFF782FE05462046FFF7B6FD3E
:104BC00007EE900AB8EEE70A002E94D007EE905A4E
:104BD000B8EEE78AB2E7002E86D02046FFF7AAFE9D
:104BE000A1E700BF00F5A04300F580419FED146AE6
:104BF00003F2447203F5FD63DFED125A10B5D1EDF7
:104C0000B26A044692ED007AD3ED2A7A66EE866A9D
:104C100027EE067A04F5004467EEA57AFDEEE66A13
:104C2000BDEEC77AFDEEE77A16EE902A17EE101A5F
:104C300017EE900A47F07CFBC4F8600210BD00BF7D
:104C40000000C842A00CB34510B5044618F05AFC49
:104C5000031E28DB04F5804191F9A7229A4222DD48
:104C600004F50044D4F8480202281CD007EE902A2C
:104C7000D01AD1EDC05AB8EEE77A07EE900A9FED50
:104C80000A6AF8EEE77AD4ED986A26EE656AF8EEDD
:104C9000E66AC7EE875AF0EE667AE6EE257AFDEE12
:104CA000E77AC4ED987A10BD0000C84270B500F5EF
:104CB00000469FED560A9FED567A0446D6ED977A48
:104CC000F8EEE77A67EE807AF0EEE76AF4EEC76A0C
:104CD000F1EE10FA1FDC9FED4F0A27EE800A66F115
:104CE00031FF47F0E5F8B7EE007A04F51043C7EE60
:104CF000007AC6ED997A93F8F42332B1D3F81C0404
:104D0000454A03685B6A934258D104F5804595F99A
:104D1000D8321BB970BD9FED410AE2E7204608F08A
:104D2000B1FA0028F6D149F22850204419F0A4F82D
:104D30000028EFD1B5F9B032F7EE006A96ED9A6A25
:104D4000012BB8BF012307EE903AF8EEE77A86EE22
:104D5000277AB4EEE67AF1EE10FA41D9D6ED997AD7
:104D6000F4EEC77AF1EE10FAD4DD86EE870A04F588
:104D7000A04420EE000A67F115FF9FED297ADFEDD0
:104D8000297A40F6C41320EE070AD6F85C0260EEDA
:104D9000277AFDEEE77A17EE905A9D42B8BF1D467E
:104DA0002A46694247F0C4FAC6F85C02D4F8403794
:104DB000AB42A8BF2B46C4F8403770BD45F24071E6
:104DC000214498470028A0D004F5A044D6F85C02FE
:104DD000D4F84027514247F0ABFAC6F85C0270BDE8
:104DE00004F5A04440F6C4120F49D6F85C0247F01F
:104DF0009FFA40F6C412C6F85C02D4F840379342DA
:104E0000A8BF1346C4F8403770BD00BF0AD7233C83
:104E10000000AA4235FA8E3C313B0208BE7EB23D0C
:104E2000E02E65420000C8423CF6FFFF00F5C0439B
:104E300010B50446D3F8840103681B68984704F54D
:104E4000A043D3F84027514247F072FA04F50043DB
:104E500002462046C3F85C22BDE81040FFF726BF9B
:104E6000704700BF704700BF0120704700F55070C9
:104E7000704700BF0820704701207047014B93F82E
:104E8000E4027047B0730030034B93F94C020038D2
:104E900018BF0120704700BFB0830030014B93F969
:104EA000E6027047B0730030064B083110B5D3F8F6
:104EB0003C0B82B0CA68036800925C6C0EC9A047C4
:104EC00002B010BDB0A30030094B82B09FED097A4B
:104ED00003F53763D3ED007AF8EEE77A67EE877A69
:104EE000FCEEE77ACDED017A9DF8040002B0704740
:104EF000B0A30030CDCC4C3D704700BF38B52A4D33
:104F0000D5F83C0B03685B689847192849D8DFE857
:104F100000F0460D36464636363636480D0D0D0D38
:104F20000D0D48363636360D48460D0D18241F4BEC
:104F300093F8152F12B193F8143F0BB944F01004F5
:104F4000D5F83C3B1A4A93421BD002F11C018B421C
:104F500017D0184A44F0100492F9591331B10329BB
:104F600002D1154A934201D144F040041348DAF0CB
:104F7000E9FD08B144F0800444F0010038BD10247C
:104F8000D5E70C4991F9591321B19342E7D144F087
:104F9000010038BD9342E9D144F0010038BD4024FE
:104FA000C5E70124C3E700BFB0A30030B0830030E1
:104FB000D0AC0030B073003030AC00301CC60030D4
:104FC00008B5044808F0D6FF00280CBF01200220D5
:104FD00008BD00BFB0330030F0B52DED028B8BB0B3
:104FE00005461FF073FF04464FF480712248D4F841
:104FF000047294ED828AD4F80C62FEF707FC60B963
:105000001E4BB7EEC87A93EDD36A9FED195BB7EEEE
:10501000C66AA6EE457BB7EEC78B194813F05CFD58
:1050200030B1184BD3F8A4355F6893ED028ADE687F
:105030002D7CF8F0DDFDD4F8141327221C230390F7
:1050400007912846D4F8181304970891D4F81C1334
:10505000019203AA09911E2100938DED058A0696FF
:105060008DF0CCF90BB0BDEC028BF0BDAFF300803E
:10507000000000A046DF913FB0330030B073003035
:1050800090C60030B0C3003010B5134C82B094F815
:105090003A1A04F6E4001DF029F830B194F83A1AEF
:1050A00004F6E4001DF030F868B91FF00FFF01A905
:1050B0001FF0A4FE18B99FED090A02B010BD9DEDC6
:1050C000010A02B010BD94F83A1A04F6E40002B0E6
:1050D000BDE810401DF070B9B06300300000000062
:1050E00008B5024818F00EFA00B208BDB03300301F
:1050F00000B5002387B00393049305931FF0E6FEE9
:1051000000F55A7003AB07C883E8070018464DF056
:1051100027FBB1EE047ADFED0B7A20EE070AB4EE3E
:10512000E70AF1EE10FA08D5FCEEC07ACDED017A6F
:105130009DF8040007B05DF804FBFF2007B05DF8A0
:1051400004FB00BF00007F4330B50C4683B040F243
:10515000EF22164805F0ACFB217811F004050AD0C7
:1051600003226168124828F023FD104803B0BDE80F
:10517000304004F06BBB01AA2946204628F014FEFB
:105180000028F2D0DDED017A2A469FED0A7A084820
:1051900067EE877AFDEEE77A17EE901A28F008FDA1
:1051A000024803B0BDE8304004F050BBB0330030DB
:1051B0001CC500300000C8420148F4F055BF00BFD4
:1051C0002C880030012310B5044C84F8173F8EF072
:1051D000F1FE002384F8173F10BD00BFB0830030FC
:1051E00070B5144605460E4607481146E2F02EFFFC
:1051F00021460648F4F084FB224631462846BDE8A5
:10520000704094F0B5BD00BF18C40030288A00304B
:105210002DE9F041224F4FF000080D4614464FF49F
:105220007A7306462DED028B9FED1E8A82B0B0EE9A
:10523000480A0092CDF80480B1F90220D7F8281767
:1052400095F072F80123B0EE480AD7F82C170193B5
:10525000304600944FF47A73B5F9002095F064F865
:105260004346D7F8301730469FED0F0ACDE9004886
:10527000B5F9042095F058F8B0EE480ACDF804804E
:105280004FF47A73B5F906203046D7F834170094F6
:1052900095F04AF802B0BDEC028BBDE8F08100BF8A
:1052A000B08300300000FA4400007A44074A40F21C
:1052B0004D1310B540F24D3492F9D824002A08BF9E
:1052C0001C468EF0E9FC204310BD00BFB0B3003097
:1052D00010B584B01FF0FAFD0446684628F030FC93
:1052E000694620461FF07EFD1C4813F0F5FB00B315
:1052F0001B4B03F65812D3F83C1B914216D003F512
:105300000053DDED017A9FED177AD3F81833F8EEEC
:10531000E77AD3ED0F6A77EEA67A67EE877AFDEE2D
:10532000E77A17EE903A18B204B010BD002004B02E
:1053300010BD019C0C4804F01DF923189FED097A5B
:1053400007EE903AF8EEE77A67EE877AFDEEE77AB5
:1053500017EE903A18B204B010BD00BF90C60030EE
:10536000B0A300300AD7233CB033003000B583B07F
:105370001FF0ACFDD0EDDA0A90EDDB0AF1EE600A29
:10538000B1EE400A67F176FCDFED097A20EE270ADC
:1053900046F04EFEF6EE007A20EE270AFCEEC07ACA
:1053A000CDED017A9DF8040003B05DF804FB00BF69
:1053B000E02E654210B5044629F0E2FB204610BD00
:1053C00008B51B4813F088FBB0B91A4BDFED1A7A09
:1053D00093ED607AB4EEE77AF1EE10FA09D5F2EEC9
:1053E000046AC7EE267AFCEEE77A17EE903A98B296
:1053F00008BD41F6991008BD0D4810F071FE002857
:10540000F6D00E4BD3F81C0303689B689847DFED7A
:105410000A7AB4EEE70AF1EE10FAEAD5B2EE047AAF
:10542000C0EE077AFCEEE77A17EE903A98B208BD24
:1054300090C60030B0B3003000FF7F47B0C30030EB
:1054400010B58EF09FFE044650B90B48A0F580526F
:10545000A0F5F06380F89B41D2F83C2B9A4201D032
:10546000204610BD90F87032002BF9D100F51B706A
:1054700050F022FEF4E700BFB0B3003000B516488C
:1054800085B013F029FB88B9144BD3F88401036865
:105490001B69984746F00AFE114B83FB0023C01797
:1054A000C0EBA310C0B205B05DF804FB0D4B9FED3F
:1054B0000E0AD3F814036C304CF04AFCDFED0B7A83
:1054C00021EE271AFCEEC17A17EE900AC0F34700CE
:1054D00005B05DF804FB00BF90C60030B09300300B
:1054E0001F85EB51B0C300309F0CB3450AD7233C56
:1054F000044B93F8F40320B1D3F81C0403681B6B2E
:1055000018477047B0C3003008B5084BD3F83824AB
:10551000002A06DD03F556708AF09AFE90ED000A27
:1055200008BDBDE808408EF08BBB00BFB0830030E3
:105530002DE9F04F2DED028B89B005461CF08AFF56
:1055400038B307464FF00008F8F052FB9FED2A8A67
:10555000814604AE4FF0140A95F80F4303AB05AA39
:10556000384644440096013404F0010421461CF0FE
:105570004DFF28B1059BA9EB0303B3F5FA6F0DD9D5
:10558000B8F1000F05D14FF00108E5E7287C8BF05A
:1055900085FF09B0BDEC028BBDE8F08F287C8CF054
:1055A000ADFE8346287C8DF0D9FE431D9B45EDD38F
:1055B0009DED047A0523DDED037A43F2782127EE91
:1055C000087ACDF804A067EE887A0093287CBCEEB8
:1055D000C77A8DF81C40FDEEE77A17EE102AADF879
:1055E0001A2017EE902AADF8182006AA8CF006FFB4
:1055F00085F80F43C4E700BF0000C84230B585B04E
:1056000005460C46684628F09BFA6A46214628461D
:1056100093F090F800283FD040F24F326946364868
:1056200005F046F9D4ED037AF4EE677AF1EE10FA5C
:1056300052D6F0EEE77A9FED317AF4EEC77AF1EECA
:1056400010FA54BF012200229DF8003068462C4910
:1056500062F341038DF8003029F0E6F8E0B96946BD
:105660002848B6F081FF88B1D4ED017AFDEEE77AE3
:1056700017EE903ADB0712D4234B03F51062D3F8F0
:105680003C3B93420BD0042005B030BD87F034FD85
:105690000522162187F052FA022005B030BD1B49C1
:1056A0000222A1F5F24017F05BFB9DF8001011F00B
:1056B00004011CD06946104805F070FB94ED020A05
:1056C000B4EE400AF1EE10FA04D6B5EEC00AF1EEDF
:1056D00010FA03DC0020E0E70022B5E79DF8001097
:1056E0000A48C1F340010AF073FD0020D5E768467F
:1056F00028F030FBDEE700BFB0330030000000349C
:105700000CC50030CC710030B0A30030B0AC00301C
:10571000B1F81CC0BCF1160F17D170B514460D4678
:105720002422002120466AF183F9AB7F0722A37768
:10573000EB7F84F82020E377AB8BA383D5ED067A4B
:10574000F1EE677AC4ED067A70BD8EF0F3BF00BF4C
:10575000F0B50446272200212DED028BE57891B0AB
:10576000954206A828BF15466AF162F904F10C01BA
:1057700006A82A466AF112F99DF83E400798E443CC
:105780000899099AE4B20A9B0290039104F08707F2
:10579000049205938DF83E40F8F02AFA14F0810F38
:1057A000054618D1802F16D014F0820F62D114F064
:1057B000840F5CD163060AD5DDED0E7A9FED397A50
:1057C000394B67EE877AC3F8F051C3ED7B7A11B09D
:1057D000BDEC028BF0BD02A8DFED348A9FED318A6B
:1057E00001904AF083FF20EE280A2F4E14F0820F1A
:1057F0000198C6F8E05120EE080ABDEEC00A86ED19
:10580000750A20D1802FD2D101904AF089FF20EE75
:10581000280A0198C6F8E45120EE080ABDEEC00A35
:1058200086ED760A4AF08CFF9FED207ADFED1D7A37
:1058300020EE070AC6F8E85120EE270ABDEEC00A9E
:1058400086ED770AB6E701904AF06AFF20EE280A53
:1058500014F0840F0198C6F8E45120EE080ABDEE5A
:10586000C00A86ED760ADDD1802FDBD0A2E702A840
:105870000D4ED7E702A80C4E01904AF051FF9FED64
:105880000B7A14F0840FDFED077A20EE070A0198F7
:10589000C6F8E45120EE270ABDEEC00A86ED760A6E
:1058A00088D0BFE70000C842B0B30030E02E6542A8
:1058B000124808B500F51263D0F83C2B9A421AD072
:1058C000B0F9543B3BB900F5805393F8252112B948
:1058D00090F8512B0AB1052008BD93F831320BB175
:1058E000062008BDA0F5E04008F044FB00280CBFEE
:1058F0000320042008BD022008BD00BFB0A3003073
:10590000234B03F63C12D3F83C3B93423FD0002399
:1059100030B591B004461F48029328F017F90028CB
:105920002FD0257CF8F064F9DDED027A96221A4931
:105930003323F8EEE77A9FED197A01920022D1F82D
:105940007841039067EE877AD1F874014FF6F851E9
:1059500005940024049028460792089209920A921E
:105960000B920C920D920E9203AAADF83C105721A7
:105970000093CDED067A8DF83E408CF03FFD11B0DE
:1059800030BD014602AA034828F03CF9C9E7704738
:10599000B0A300301CC50030B0C300300AD7233C90
:1059A00030B58DB00446F8F023F9174AD2F8183410
:1059B000C31A642B26D8D2F8142325231625029067
:1059C000D2F88410207C0391D2F888100491D2F888
:1059D0008C100591D2F890100691D2F8DC100A9143
:1059E000D2F894100791D2F898100891D2F89C1030
:1059F00002AA01950991002100938DF82C105321E2
:105A00008CF0FCFC0DB030BDB0C300302DE9F0438C
:105A1000994E2DED048B06F63C13D6F83C2B91B035
:105A20009A4277D00446954813F056F800287DD165
:105A3000934B94F8109003F50054D3F884719FEDC4
:105A4000918AD4ED977A38463B68B8EEE79AD4ED60
:105A5000987A9B68F8EEE78A984707EE900A3846EE
:105A600029EE089AB8EEE77A68EE888A27EE087A77
:105A7000BDEEC77A17EE103A1DB23B681B69984716
:105A800007EE900A94ED607AF8EEE77ADFED7E6A31
:105A9000B4EEE67A67EE887AF1EE10FAFDEEE77A78
:105AA00017EE903A1CB23AD44FF6FF78774806F6D4
:105AB000783603F05FFD3B6807EE900A744A5B6935
:105AC000B8EEE78AD6ED009A9FED6E7A9342DFED4D
:105AD000717A28EE078A69EEA79A40F0C38097EDA5
:105AE000080AB7221A2348463E21019209AA0093C8
:105AF0008DED099ACDED0A8A8DED0B8ACDED0C9ACC
:105B00008DED0D0AADF83850ADF83A40ADF83C8057
:105B10008CF074FC11B0BDEC048BBDE8F083BCEEDE
:105B2000C77A17EE103A1FFA83F8BFE7534810F010
:105B3000D7FA00283FF47CAF06F500589FED560ACF
:105B4000DFED508AD8F814036C304CF001F908F5F9
:105B50003B70B0EE609ACDED070AB0EE418A8DED54
:105B6000081AF0EE409A8DED060AE5F07BFBD8F8B6
:105B70001833014604A893EDDE6B93EDDC7BB7EEA2
:105B8000C66BB7EEC77B8DED056A8DED047A4BF0E1
:105B9000CFFD09A88DED090AB0EE680ACDED0A0A1D
:105BA0004BF0D6FD28EE288A02A894F81090CDED8F
:105BB000030A69EEA89ABDEEC88A8DED020A69EE65
:105BC000288A18EE103A1CB24BF036FEDFED337A1D
:105BD00002A820EE270AFDEEC07A17EE903A1DB219
:105BE0004BF074FEDFED287AB4EEE70AF1EE10FA1E
:105BF0003BD5BCEEC00A10EE103A9FB2284BD6F847
:105C00003C2B9A4234D0D8F81833DFED1E7A93ED4E
:105C10000F9A29EE279A06F67836D8F81C33DFED6E
:105C20001D7A96ED008A186928EE278AEBF0EAFAC9
:105C30001A23B72248463E21019209AA0093ADF8E3
:105C400038408DED0D0ACDED099ACDED0A8A8DED26
:105C50000B9A8DED0C8AADF83A50ADF83C708CF093
:105C6000CDFB57E7384698473BE74FF6FF77C5E748
:105C70009FED0C9ACFE700BFB0A3003090C6003074
:105C8000B09300300AD7233C00FF7F47B033003089
:105C9000A92702080000C8429F0CB345E02E6542C8
:105CA00008AD003000000000002310B50B4C84F854
:105CB0009B318FF021FCA4F58052A4F5F063D2F85B
:105CC0003C2B9A4200D010BD94F87032002BFAD1D0
:105CD00004F51B70BDE8104050F0EEB9B0B30030D1
:105CE000014810F00DBA00BF90C6003008B5034B54
:105CF000D3F83C0B03685B68984708BDB0A300303D
:105D000030B5044687B01FF0E1F8257C0446F7F073
:105D100063FF1023D4F88412CD22D4F88842029075
:105D20002846049142F60C3105940024CDE9003256
:105D300002AA03948CF062FB07B030BD30B52DEDA4
:105D4000028B89B005461FF0C1F800F55A7002AC0D
:105D50002D7C07C884E80700DDED020A9DED030AEB
:105D6000F1EE600AB1EE400A66F184FF2046B0EE23
:105D7000408A4CF0F5FCDFED0B7A0C2304990122EC
:105D800028EE278A28460791A8218DED060A8DED79
:105D9000058ACDE9003205AA8CF030FB09B0BDECD4
:105DA000028B30BDE02E6542A1F11B0370B50446A5
:105DB000382B1ED8DFE803F0711D1D1D1D1D1D1D94
:105DC0001D211D1D2C371D1D1D1D1D1D1D1D1D1DD6
:105DD0001D1D1D1D1D1D1D1D1D1D1D1D1D411D4BA1
:105DE000541D1D1D1D1D1D1D1D1D1D1D1D1D1D1DAC
:105DF0005B00BDE8704095F07DB80C218BF060FB36
:105E00000546002846D02046FFF798FF284670BD7B
:105E100012218BF055FB054600283BD0217C2248FF
:105E200082F004FCF2E716218BF04AFB054688B3AA
:105E3000217C1D4882F012FDE8E726218BF040FB13
:105E4000054638B3217C1948C2F0ECF8DEE7102192
:105E50008BF036FB0546E8B12046FFF751FFD5E74A
:105E60000125017C1248F0F06BF9284670BD052130
:105E70008BF026FB054668B1207C8CF03FFA064685
:105E8000207C8DF06BFA431D9E4208D32046FFF71D
:105E90004FFBBBE70025284670BD0125B6E7207CF7
:105EA0008BF0FCFAB2E700BF88B80030E8C20030DF
:105EB00030C1003000293DD0F0B505460C461646ED
:105EC0002DED028B8DB0007CB0EE408A8CF016FA7E
:105ED0000746287C8DF042FA00F121039F4221D32E
:105EE0006221A26921238DF824600191216A287C16
:105EF0000592CDF82910626A00931923E168CDF864
:105F0000252003AA069121698DED048A0791616914
:105F1000089121680391C2218CF070FA0DB0BDEC9C
:105F2000028BF0BD287C0DB0BDEC028BBDE8F040CB
:105F30008BF0B4BA704700BF70B5564C04F63C13F2
:105F4000D4F83C2B9A4215D0A4F540560546B6F934
:105F50008C33DA072DD49C074ED458073BD419074D
:105F60001BD4DA0604D54C4CD4F84822042A73D04A
:105F70009B0600D470BD494811F08CF80028F9D078
:105F8000474B28460422D3F81813BDE8704091ED22
:105F9000AE0A01F52D71FFF78DBF42490522284653
:105FA0000B46043993ED000AFFF784FFB6F98C33F2
:105FB000D7E73A4811F06EF8002842D004F50054B3
:105FC000394AD4F8140303689B6893425CD100F506
:105FD000AC71A03137E0314811F05CF838B3304B88
:105FE000324AD3F8140303681B6993424FD100F57A
:105FF000507000F1A0011BE0284811F04BF860B18F
:10600000274B2B4AD3F814030368DB68934239D13A
:1060100000F5137000F1A00100E0264991ED010A9E
:1060200002222846FFF746FFB6F98C3395E722494E
:1060300091ED010A03222846FFF73CFFB6F98C33A5
:106040008DE7A4F5A35191ED010A01222846FFF73F
:1060500031FFB6F98C337EE71EF038FF034604F5B6
:1060600058601C46F0F0B6F8DFED147A014694ED66
:10607000C70A0622284620EE270AFFF71BFFB6F9BB
:106080008C3375E79847C5E798470146A1E79847DD
:10609000AFE700BFB0A30030B0B3003090C600300F
:1060A000B0C30030989200301D3B02086D4E0208CC
:1060B000253B0208B890003038920030E02E65424F
:1060C00070B50E46044635F06FFB0346B0222046FD
:1060D00093F80C1302FB0131F43104F01FFF054665
:1060E00070B17EB904F5E04247F6AC03D2F83C0B40
:1060F000234498420FD047F6CC13234498420AD049
:10610000284670BD1EF0E2FE90F87C3243F0020398
:1061100080F87C32E6E708F0AFFC284670BD00BF8F
:1061200070B582B01546064601911EF0CFFE01996A
:106130001EF08EFA044670B185B906F5E04247F6C6
:10614000AC03D2F83C0B3344984210D047F6CC1342
:10615000334498420BD0204602B070BD1EF0B6FE0C
:1061600090F87C3243F0020380F87C32E5E708F0D7
:1061700083FC204602B070BD10B52DED028BD1ED31
:10618000017A8AB091ED008A0446FCEEE77A05AA0E
:10619000CDED037A9DF80C1094F0AEF8C8B1DFEDA8
:1061A0000F7A0022059B06A828EE278A1146009345
:1061B000FDEEC87A17EE903A27F0DAFC2368204605
:1061C00006A9D3F8E830984700200AB0BDEC028B4E
:1061D00010BD02200AB0BDEC028B10BD0000C84209
:1061E000F0B54AF2F9720C462DED028B8B8B83B021
:1061F00093420CD04AF2FA7293424ED04AF2F872AD
:10620000934210D0032003B0BDEC028BF0BD854F4C
:1062100007F51063D7F83C2B9A427FD0042003B0D7
:10622000BDEC028BF0BD7F4D05F51063D5F83C2B1E
:106230009A42F3D1D1ED007AFDEEE77A17EE903A6B
:10624000002B73D1A5F5405391ED010AB3F9B222A9
:1062500007EE902AF8EEE77AB4EEE70AF1EE10FACC
:1062600064DCB3F9B03207EE903AF8EEE77AB4EEB8
:10627000E70AF1EE10FA59D49FED6B8A05F58056C6
:1062800020EE088AD6ED7D0AB0EE480A45F0A2FD60
:10629000002800F099800020B5E7624E06F51063F3
:1062A000D6F83C2B9A42B9D191ED010AB5EEC00A5D
:1062B000F1EE10FA3AD4DFED5D7AB4EEE70AF1EED2
:1062C00010FA33DA45F04AFED4ED007A9FED588A91
:1062D000FDEEE77A20EE088A17EE903A5BB3012BC9
:1062E00024D106F58056022386F828325148C4F09E
:1062F000CFFE9FED517A86ED878AD4ED027AF4EED7
:10630000C77AF1EE10FA77FE877AC6ED887AF7F051
:106310006FFC03460020C6F8243274E7FFEE000A43
:1063200091ED060A054645F055FD98B1022003B0EF
:10633000BDEC028BF0BD06F50053012106F5805639
:1063400003F5AE7203F5A67586F828120FCA85E824
:106350000F00CBE7DFED390A94ED060A45F03AFD70
:1063600006460028E2D101AA284694F8201093F0AE
:10637000C3FF0028DAD094F8203007F580559FED50
:106380002A7A07F5905085F81832D4ED067A019AEA
:1063900067EE877AFDEEE77A17EE901A27F008FC91
:1063A000F7F026FCC5F81402D4ED027A9FED247AAA
:1063B000F0EEE77AF4EEC77AF1EE10FA2DD5214B24
:1063C0003046C5F810321EE786ED7D8AF7F010FCE6
:1063D000C6F8FC0105F53763D4ED027A9FED187A13
:1063E000F0EEE77AD6ED7D6AF4EEC77A93ED007AA7
:1063F000B8EEC77AF1EE10FAF4EEC76A48BFDFEDE7
:10640000127AF1EE10FAC6ED7E7A7FF544AFF1EE26
:10641000677A0020C6ED7E7AF5E63046C5ED847ACF
:10642000F1E600BFB0A300300000C8420000B44352
:1064300035FA8E3C34890030CDCC4C3D0000000054
:106440000000003400007A4400007A4430B5124D58
:1064500083B00C46D5F83C0B03681B6A984728B9F3
:1064600005F50863D5F83C2B9A420FD1D4ED007A9C
:10647000D4ED020AFCEEE77A94ED010A0748CDED6F
:10648000017A9DF8041005F06FFB10B9042003B0E9
:1064900030BD002003B030BDB0A30030B0330030B9
:1064A00010B5D1ED007AFCEEE77A17EE903A9CB287
:1064B000012C04D0022C08D00CB1042010BD2146C0
:1064C0001248ADF0EBFD002010BD114890F8CC341F
:1064D0005B0713D490F9B83443B1A0F500400DF038
:1064E00029FA002814BF0020042010BD94F050FBAE
:1064F000084A05218AF0FAFC042010BD94F048FBFC
:10650000054A05218AF0F2FC042010BD68B800306D
:10651000B0B30030C8501908AC50190830B58B8B97
:1065200085B00C460546DF2B34D8B12B52D9B23B8F
:106530002D2B68D8DFE813F0E300670067006700E1
:106540006700670067006700E9006700EF00FE0072
:10655000670034012001670067006700670067007B
:1065600067006700670067006700670067006700F3
:10657000670067002E019E0067006700BF0067008C
:1065800067006700670067006700670067006700D3
:106590006700D1004AF2FA7C63452BD84AF2F77CB7
:1065A000634500F20681B3F5967F00F0078140F65F
:1065B000B8318B4227D1D4ED007A9848FCEEE77AC7
:1065C000CDED027A9DF808100EF0ACFE70BB0420F1
:1065D00005B030BD113B99B20F2914D80F2B12D83A
:1065E000DFE803F01811111F1127111111111111FA
:1065F0001111112F4AF2FD70834204D1884804F032
:10660000D9F80020E4E72146284605B0BDE830402F
:1066100095F04CB802228349814816F0A1FB002076
:10662000D6E7022280497E4816F09AFB002005B08A
:1066300030BD94F82030072B00F0DE80022005B03A
:1066400030BDD4ED007AF5EEC07AF1EE10FAF5DD4A
:106650009FED767AF4EEC77AF1EE10FAEED8FCEE02
:10666000E77A734A0020CDED027A9DF80830A2F84F
:106670007A36ADE7D4ED027AD4ED016AFCEEE77A22
:1066800094ED007AFCEEE66A227CBCEEC77A94EDCB
:10669000030A17EE903A017CCDED026A9CB28DEDB3
:1066A000037A01929DF808309DF80C2000945B4815
:1066B0000CF060F98CE7D4ED007A9FED5E7AF0EE95
:1066C000E77A5748F4EEC77AF1EE10FA54BF012189
:1066D000002106F0AFFD00207AE7D4ED037A94EDB7
:1066E000021AFCEEE77AD4ED010A94ED000A524852
:1066F00017EE901AA8F00EFE002897D167E7214602
:1067000005B0BDE83040FFF7A1BE214605B0BDE8A9
:106710003040FFF731BD494C94F86D3B002B3FF4FE
:1067200056AF4749A1F56F604FF000FE00283FF4D7
:106730004EAF0DE0414C94F86D3B002B3FF447AF5A
:106740003F49A1F56F604FF04DFD00283FF43FAF8A
:1067500004F580550123022204F50861A4F5E04008
:1067600085F8A53216F0FCFA00287FF45FAF00230D
:10677000042085F8A5322BE7D4E9040147F01CF981
:1067800000283FF45BAF2146284605B0BDE8304005
:10679000FEF734BF214605B0BDE83040FFF780BEAC
:1067A00094ED000A1E48FCF7A9FC00287FF43EAFD8
:1067B0000DE705B0BDE83040FFF712BDD1ED007A1E
:1067C0009FED1C7AF0EEE77AF4EEC77AF1EE10FA5C
:1067D0007FF534AFD1ED017AF0EEE77AF4EEC77AC7
:1067E000F1EE10FA7FF52AAF16490222A1F5F14029
:1067F00016F0B6FA0020EBE6134890F8F433002BBD
:106800003FF4E5AE94ED060A00F53870B1EE400AAB
:1068100010F0CCF900287FF409AFD8E690C600301C
:10682000B033003078AC00305CAC003000007F4307
:10683000B08300300000003444770030B0A3003053
:106840000CC5003030AC0030B0C3003030B50C4661
:10685000352291B00021E57802A8954228BF15465F
:1068600069F1E6F804F10C011D4C2A4602A869F111
:1068700095F804F51062D4F83C1B914201D011B098
:1068800030BD9DF83C20072AF9D104F50054DDED18
:10689000056A9FED147AD4ED5C7AF8EEE77AE6EEBD
:1068A000C77AFDEEE77AC4ED5C7A94F071F9D4F81A
:1068B0004811D4F870314C680621DFED0B7A1B1BB0
:1068C0000A4A07EE103AB8EEC77A27EE277AB7EEF3
:1068D000C77A8DED007B8AF009FB11B030BD00BF97
:1068E000B0A300300000C8420AD7233CE05019088A
:1068F000244B03F51062D3F83C3B934200D0704721
:1069000070B53522CE7896B00C46964205464FF0CB
:10691000000108A828BF164669F18AF804F10C01A5
:1069200008A8324669F13AF803AA9DF8541028469F
:1069300093F0E2FCF8B1BDF8503023F004039BB2B1
:106940000BB916B070BDDDED0B7A00229FED0E7A0B
:1069500004A8039B114667EE877A0093FDEEE77A61
:1069600017EE903A27F004F92B6804A92846D3F8CB
:10697000E8309847E5E794F00BF9044A04218AF0DF
:10698000B5FADEE7B0A300300000C842F4501908A1
:1069900000B591F80AE04B7A43EA0E2391F80BE038
:1069A00043EA0E43562B16D00A46844607D8522B8C
:1069B0001BD0542B13D15DF804EBFFF747BF1249EE
:1069C000194421F07F41012909D8017C5DF804EBCD
:1069D0000E4882F003B85DF804EBFFF789BF11465B
:1069E00060465DF804EB93F011BD094B03F51061AF
:1069F000D3F83C3B8B4201D05DF804FB10465DF8B8
:106A000004EBFEF7A5BE00BF7AFFFF0088B8003098
:106A1000B0A3003000207047C820704701207047A5
:106A2000002070470020704790F8D0308B4204D986
:106A300000EB8100D0F8D40070470020704700BF01
:106A400090F8D0308B4204D900EB8100D0F8D4000C
:106A500070470020704700BF03207047014B93F838
:106A6000E2027047B073003070B50446514814F02C
:106A7000A9FC18B1636A43F4000363624D4814F043
:106A8000A1FC00287DD1636A4B4A43F4F84363625A
:106A9000D2F83C0B03685B689847013818281AD86D
:106AA000DFE800F00D524E5952525252190D0D0DA1
:106AB0000D0D0D19525252520D19590D0D00D4E9F8
:106AC0000A2342F4E84243F4E84342F4006243F408
:106AD0000063C4E90A23394B93F87C3D012B47D06E
:106AE000022B0BD1E36AD4E9091243F4800341F489
:106AF000800142F48002E362C4E90912304B1D6850
:106B0000EDB1304E284696F81A177AF05BF9B0B11D
:106B1000636AA6F5805243F48073636292F9883306
:106B20001BB1A36A43F48073A36296F81A17284630
:106B30007AF09AF918B1E36A43F48073E36270BDA6
:106B4000204B93F8142F82BBD4E90A2342F48062CD
:106B500043F48063B9E7D4E90A2343F4806342F441
:106B60008062C4E90A23154B93F87C3D012BB7D111
:106B7000D4E9092342F4800243F48003C4E90923E1
:106B8000BCE7462097F088FEDFED0F7AB4EEE70A07
:106B9000F1EE10FA3FF677AFD4E90A2342F400028F
:106BA00043F40003C4E90A236DE793F8153F002B73
:106BB00091D1C9E7B0330030B0A30030B0B300309A
:106BC000ACCC0030B0830030000000B470B54FF49E
:106BD00044700D46164627F0C7FF044628B13246DA
:106BE00029468DF0C1FE024B2360204670BD00BFD8
:106BF000105319080020704790ED0D0A704700BF30
:106C00000020704700207047002070470020704728
:106C10000020704700207047002070470020704718
:106C20000020704700207047002070470020704708
:106C300000207047002070470020704700207047F8
:106C4000002070470020704700207047034644F240
:106C500044301844704700BF00487047F883190853
:106C600000F5E040D0F83C0B03685B68184700BFB4
:106C700000F5E04300F5F140D3F83C3B181AB0FAB8
:106C800080F04009704700BFB32070472DE9F04104
:106C9000002390B0DFED7B6A49F2E027039300F513
:106CA00000430744044693ED977AD3ED987A38462B
:106CB000B8EEC77A04F51046F8EEE77A27EE267AA2
:106CC00067EEA67A8DED017ACDED027A11F004FF20
:106CD000002800F0BE80D6F814330DF1100E0DF12F
:106CE000300C08AD84330FCB8CE80F008EE80F001A
:106CF00085E80F00704601A903AB02AA49F03AFDEE
:106D0000D6F8A48501A89FED600A4BF021F829462A
:106D100040468DED080ACDED090A8DED0A1A1BF0EB
:106D200099FDF6F065FFD6F81834C01A632839D9F2
:106D300041F698253846254410F0ACF9002873D167
:106D400045F6A03269212846224484F039FF45F6F1
:106D500008526A212846224484F032FF04F5A043F9
:106D600093F94A2D42B903F55463D3ED007AF5EE59
:106D7000C07AF1EE10FA06DD45F688626B212846EE
:106D8000224484F01DFF45F6B46626443046DFF009
:106D9000A5FE002863D11EF099F81EF003F810B08C
:106DA000BDE8F081D6F8140341F69825374A036808
:106DB00025449B68934263D100F5AC7000F1A002BA
:106DC0000421284684F0FCFED6F81403304A0368F8
:106DD000DB68934252D100F5137000F1A002052147
:106DE000284684F0EDFED6F814032A4A03681B698E
:106DF000934241D100F5507000F1A00206212846CF
:106E000084F0DEFED6F818232846072102F52D72FD
:106E100084F0D6FE49F22850204417F099FF3846F6
:106E200010F038F900288BD0D6F81803E9F08CFC64
:106E3000002885D0D6F8182328466E21903284F099
:106E4000BFFED6F818236F212846BC3284F0B8FE66
:106E500076E701A904F512501BF0C0FB61E706F1CB
:106E600030026D21284684F0ABFE1EF02FF81DF095
:106E700099FF10B0BDE8F0819847BDE79847ACE7AF
:106E800098479BE70AD7233CE02E65421D3B02084A
:106E9000253B02086D4E020810B54FF480110446E0
:106EA00016F02AFB30B94FF48001204616F024FB7F
:106EB00050B910BD2046FFF7E9FE4FF4800120468F
:106EC00016F01AFB0028F4D044F0CEFBBDE81040C9
:106ED00041F010BA30B5002591B000230446029568
:106EE00000F5125502A90DF1070228468DF807306A
:106EF0001DF08AFF03A928461CF00AFB08B92F4B96
:106F000003933022002104A868F192FDA322952367
:106F10008DF810208DF81130F6F072FE04F5004265
:106F200004F50053CDF81710D2F85C12D2F86022A5
:106F3000CDF813004620ADF81F20D3F87C26D3F8F7
:106F40007836ADF81B10ADF82120ADF81D3097F064
:106F5000A3FC10EE103A1520CDF8233097F09CFCDE
:106F600045F2E8729FED167A10EE103A029922442B
:106F70002846CDF82730D2ED297A9DF8073067EE04
:106F8000877ACDF82F108DF83330039B17EE902AB7
:106F90000D93CDF82B201DF073FF04F5E04341F66F
:106FA0009820302204A9D3F8803B20448DED0E0AAE
:106FB0000F9384F07DFF11B030BD00BF2292CA7FD5
:106FC0000000C84210B58AB0044625220021684658
:106FD00068F12EFD9523A3218DF801300A238DF849
:106FE00000108DF80230F6F00BFE04F50043DFEDE3
:106FF0001C6ACDF80710D3ED817A93ED7D7AD3F832
:10700000F811F8EEE77A27EE267ACDF80300CDF8EE
:107010000F1004F50240D3F8101267EEA67A17EEAF
:10702000102ACDF8171093F81812CDF80B2017EE90
:10703000902A8DF81B10D3F81C12D3F82032CDF80B
:1070400013200791089326F0D1FD8DF8240041F616
:10705000982025226946204484F02AFF0AB010BDFA
:107060000AD7233C30B58FB004463522002168464C
:1070700004F5C04568F1DCFC95220123A3218DF8BD
:1070800001208DF802308DF80010F6F0B9FD04F5FE
:107090000043CDF80300D5F88401D3F88031CDF852
:1070A0000710CDF80B3003681B699847D5F8843179
:1070B000ADF80F001A6818469368984703462448AD
:1070C000ADF8113002F056FAADF81300D5F884018E
:1070D000204A03685B69934230D1036ACDF81530CA
:1070E00003681D4A9B6993422ED1436B04F5E0422D
:1070F000CDF8193004F51043694602F67830D2F81D
:10710000702B0068CDF831203522CDF81D00D3F862
:107110007401CDF82100D3F87801CDF82500D3F81B
:107120007001D3F85436CDF8290041F69820CDF8F7
:107130002D30204484F0BCFE0FB030BD9847D5F808
:10714000840110EE103AC9E7984710EE103ACDE7E7
:10715000B0330030A9270208F96B020870B59522F8
:1071600086B000240223A32105460494ADF8144000
:1071700005F50046CDE90044CDE902448DF8012033
:107180008DF802308DF80010F6F03AFD03462846DF
:10719000CDF80710CDF8033006F0ECFE184B8DF853
:1071A0000B001B68174AD86AD6F84C32039390F844
:1071B0009C308DF810300368DB6993421DD196F83E
:1071C00031328DF811408DF8123044F04DFA43F011
:1071D000EBFAD6F84832044641F698208DF8143080
:1071E000162296F83232284469468DF813408DF8FD
:1071F000153084F05DFE06B070BD98470446DEE7AA
:10720000AC330030F56B020810B58AB02722044673
:107210000021684668F10CFC9523A3218DF801300C
:1072200009238DF800108DF80230F6F0E9FCCDF856
:1072300003000420CDF8071097F02EFB10EE103A53
:107240001320CDF80B3097F027FB10EE103A4620B4
:10725000CDF80F3097F020FB10EE103A1520CDF846
:10726000133097F019FB10EE103A0320CDF81730C9
:1072700097F022FB10EE103A1A20CDF81B3097F051
:107280000BFB47F68C3310EE101A41F6982027229C
:107290002344CDF81F10204469461B68CDF82330E5
:1072A00084F006FE0AB010BD38B541F698250446B4
:1072B0000544284683F076FF284684F01FF804F53D
:1072C000805393F9C83B23B92046BDE83840FFF707
:1072D0009BBF284684F04AF92046BDE83840FFF7B6
:1072E00093BF00BF00F5E04238B500F5F243D2F895
:1072F0003C2B9A4200D038BD00F500450446D5F835
:1073000024328BB9D5F80432013308D1DFED0B7A82
:1073100095ED7D7AB4EEE77AF1EE10FAEBDB2046DC
:10732000BDE83840FFF74EBE45F2246241F6982092
:1073300008212244204484F043FCE3E700000034A9
:1073400000F5104330B593F8F42389B00446E2B950
:1073500041F69825054404F5E043D3F83C0B036857
:107360005B68984704F580430146284693F8B820A7
:1073700084F07AFF04F512501EF048F804F55670B8
:1073800009B0BDE8304033F061BB41F69825D3F831
:107390000C0369461E222544EBF052FD6A46024961
:1073A000284684F0F5FCD6E7405419080F2904D884
:1073B000302303FB0100B83070470020704700BF46
:1073C000F8B5324B074600F59874314E40F8043B4F
:1073D00007F58665A7F020FB07F1780094F0C2FD61
:1073E0002C4BBB67204695F033F844F8306BAC4229
:1073F000F8D1204641F2CC0497F056FD264A2749A1
:1074000007F56C60F0F020FE07F58055FF233C4443
:10741000234985F8DC30204685F8E43076F0CAF858
:10742000204B1A6872BB41F2EC001C603844F2F049
:1074300013FCF1EE043A9FED1C5A41F2F410F7EE02
:10744000004A9FED1A0AB2EE042A3844B0EE454ACB
:10745000B0EE633AF0EE632AF0EE451AB0EE451A4C
:10746000F0EE450AC3F07EFB41F2E8203844F2F02A
:107470007DF8012338460E4985F8893376F09AF86D
:107480003846F8BD0B48F6F07FFB00BFC84A003015
:1074900090B41908A4B4190854760030988B0030C1
:1074A0006C9F1C08B4D800300000000000409C45D0
:1074B00014A31908EC9F190844F2E0210D222DE9CC
:1074C000F04F01449DB0064682F0BAFB002227210E
:1074D000C84876F037FE0421002097F061FA1321A6
:1074E000012097F05DFA4621022097F059FA152104
:1074F000032097F055FA97F09DFC06F5104393F999
:10750000AC33002B40F06F8177F058FDBA49BB4C8B
:1075100000230A880CAD04F148090DF1200A42F05D
:1075200004021F464FF00108DFF80CB30A803A222C
:1075300004E0A14537D0A2890C34636807A9284626
:107540002F60AF60ADF830200D93EF608DF838807C
:1075500076F0ECFC0028ECD09DF91C30002BE8DD27
:1075600094F06EFF9DF81C100268302301391268F8
:10757000C9B25A4503FB010303F1B80340F0DE80B2
:107580000F29D6D804331846039375F0CBFF039B1D
:107590000028CED11846A3685146ADF8203078F0C7
:1075A00057F9A145C7D100220DF11301944875F098
:1075B00003FC044620B175F0B5FF002800F05A81A5
:1075C00005AC904B0FCB8AE80F002146504676F071
:1075D000ADFC002840F0B88044F27C30B7EE000AE1
:1075E00000220121304476F061FE44F21830B7EEFB
:1075F000000A00220221304476F058FE012243F6B0
:10760000E401002300928E207F4A314476F0B4FDDD
:1076100096F9D4CDBCF1000F00F01081012443F69F
:107620001C610023794A314440F20510009476F041
:10763000A3FD44F24C3000229FED750A0221304434
:1076400076F034FE44F2B42000229FED710A03214B
:10765000304476F02BFE44F2BC2000229FED6C0AF1
:107660000321304476F022FE44F2483000229FEDA0
:10767000680A0321304476F019FE44F250300022AB
:107680009FED630A0221304476F010FE44F2C820D8
:1076900000229FED5F0A0221304476F007FE44F29B
:1076A000CC2000229FED5A0A0221304476F0FEFDE4
:1076B00044F2C420002202219FED550A304476F0A6
:1076C000F5FD48F680503044EEF098FE514B1A68B4
:1076D000D10711D443F63C014F4A43F650201C60B9
:1076E000314441F6AC333044116043F634713344D5
:1076F000D06031445362916144F290300422464993
:107700000124304476F09AFD41F698210023434A43
:107710003144FD20009476F02FFD414B1A68D207CA
:1077200005D442F26C323F491C6032440A600121A8
:107730003C4876F0A1FD1DB0BDE8F08F90470346B0
:1077400000283FF4F6AE1DE7002206A90B9875F05D
:1077500033FB044600283FF43FAF75F0E3FE0746D5
:1077600000287FF439AF9DF81430013BDBB2032BC6
:1077700000F2AA802C4AD356204629468DF8303094
:1077800078F00AF8002207A9284875F015FB04468E
:10779000B5F020FA78B1B5F01BFA90F8283090F8DF
:1077A00030201A4490F84030134490F84820DA42D0
:1077B00014BF01270027002C3FF40EAF20469DF98F
:1077C000148075F0AFFE00287FF406AFB8F1000F0B
:1077D0000CBF002707F00107294620468DF83070BE
:1077E00077F0DAFFF8E69FED120A124877F0EEFB29
:1077F0008AE600BF50A0190874CC0030C0A2190856
:1078000010A01908083C190810EA1908F89A1C0871
:107810000AD7233CA4330030C425003060C31A08C3
:10782000A8330030F42500304CA019081CA019081A
:1078300000009643DCDE1A08AD730208234F2C4685
:107840000FCF0FC40FCF0FC40FCF0FC497E80F0097
:1078500084E80F0062460421284676F073FC9FED11
:107860001C0A1C4877F0B2FBB7EE000A1A4877F002
:10787000ADFBD3E6194B0FCB8AE80F0006A95046A3
:1078800076F054FB88B90427154B0FCB85E80F0021
:1078900007A9284676F04AFB70B9204605AC8DF85A
:1078A0001470214677F078FF8BE606A875F03AFE53
:1078B0000028E8D00C27E7E707A875F033FE00287A
:1078C000EBD047F00107E8E7034655E7183C1908F5
:1078D000000000002CA019083CA01908E83B19087A
:1078E000F83B1908704700BF002070470020704720
:1078F000002070470020704700207047704700BF8D
:10790000002070470020704784B000200DF1040C67
:1079100004B08CE80E0070470020704700207047CC
:10792000704700BF102070470048704740B01908EA
:107930000048704750B0190800207047704700BFDA
:10794000012070470120704700207047027E531CC1
:1079500000EB8202DBB2042B037682ED010A01D92F
:1079600000230376437E042B1FD80133DBB207EEDE
:10797000903A4376B8EEE70AD0ED017A9FED0D7AA2
:10798000D0ED025A77EE877A90ED036AD0ED046A63
:1079900090ED057A77EEA57A77EE867A77EEA67A7D
:1079A00077EE877A87EE800A70470523B1EE040AE6
:1079B0004376E1E70000000000230022436083607B
:1079C000C360036143610283704700BF10B5044682
:1079D00027F0D6F8204610BD05F05CBF04F028BCA7
:1079E00005F084B904F030BC02F0CCBD01F0AABDB2
:1079F00002F094B802F0C4B8FCF756B8FBF7BEBA70
:107A0000F8B54D4A00F510430546026093F85C2036
:107A10003AB99C6D2CB120463FF03CFB204627F044
:107A2000AFF805F5A042454905F5C043C2F81C1F53
:107A3000D3F8180108B127F0A7F8414B43F69C5042
:107A40002B60284426F066F805F5405393F8D827B4
:107A500042B9D3F8D4472CB120463FF01BFB204657
:107A600027F08EF842F2503041F6DC6441F6C466ED
:107A700028442C442E44D6F0F3FC14F8043C083C73
:107A80003BB92768384627B13FF004FB384627F05A
:107A900077F8B442F1D141F6C83041F2847441F232
:107AA000247628442C442E4499F08EF92046183C24
:107AB0003EF086FDA642F9D141F2B01441F26817BA
:107AC000204B2C442F44C5F8883C14F8043C083C57
:107AD0003BB92668304626B13FF0DCFA304627F045
:107AE0004FF8BC42F1D105F64C6088F06DF805F511
:107AF000626088F069F805F6F45088F065F805F6DC
:107B0000485088F061F805F61C5088F05DF805F5DE
:107B10004F6088F059F80C4A95F81032C5F8FC20EF
:107B200043B9D5F80C422CB120463FF0B3FA2046B9
:107B300027F026F82846F8BD18941908DCE01A0842
:107B400048BB1A08145C1A0810041D08F8B56F4BDE
:107B50000546002744F2C80440F8043B44F2482696
:107B6000A7F066FD05F1100022F08EF905F1B000D6
:107B7000DAF026F805F528707FF0D6FC05F556708A
:107B800031F0F0FD05F5F4601FF02EFF05F63C1016
:107B900027F052F805F6884040F0EAFF41F21870ED
:107BA0002C442E442844A6F0B9FC41F2E870284445
:107BB00078F0D0FA41F69820284484F06FF841F626
:107BC000AC302844B3F0A2FB41F6C830284499F009
:107BD000E3F841F60440284425F0A8F805F5E650FE
:107BE000C6F0B6FA42F250302844D6F025FC42F2F4
:107BF0006C30284480F0A6F842F2DC302844A9F02A
:107C000079F905F5005342F23040414A83F8207477
:107C100042F2204328442B4413606DF0D5FD3946D1
:107C200005F512501BF00AF842F678302844AEF001
:107C300069FC42F6A8302844C5F05EFA43F2B4501D
:107C40002844CEF0F7F943F2CC602844CCF0B0FEE3
:107C500043F2F4602844D0F03DFE05F55E50D5F0C7
:107C60006BFB43F2E4702844D6F0EEF843F63C0098
:107C70002844C3F001FB43F6E400284419F01CFE3D
:107C800043F650202844C5F0AFFF43F6A82028440F
:107C9000D7F008FF43F6FC501E49284475F08AFCD3
:107CA00043F614602844DCF0F7F843F61C602844DF
:107CB000B4F09CF943F6DC602844D7F0A3FD43F60A
:107CC00034702844F5F0B4FF05F5804383F8B870AC
:107CD00020460C3488F0B8FAB442F9D144F254206A
:107CE0000D4C2844D7F0E8FD44F27820284487F072
:107CF00065FD236833B92846084975F05BFC2846C2
:107D00002560F8BD0648F5F03FFF00BF48BB1A08E4
:107D100000D8003034A11C08E4CC0030B0B91A08F7
:107D200058B019082DE9F04F2DED028BA5B004468F
:107D3000FFF70CFFE54B44F2903004F5A0452360BB
:107D400044F2A427204404F51259FFF739FB45F209
:107D50002070274445F2E87620444FF0000AD9F01D
:107D600015FF44F22A3304F5AF404FF0000B2344D3
:107D7000264404F5B448C5F84837062385F84C373F
:107D800098F060F948F680534FF4006CD04AE3183D
:107D90004FF07E50C5F804C84FF05A0CC5F80038B3
:107DA000109305F5FD6385F884C8C5F8FC77C5F820
:107DB000F897C849C3F85C0145F6C410C3F86821B8
:107DC000C3F8CC212044C44AC3F86011C3F864212D
:107DD00088F03AFA45F6D010204488F035FABF4AC8
:107DE00005F51E63BE49C5F8E0293046C3F804A076
:107DF000C3F808A0C3F80CA0C3F810A0C3F814A0DF
:107E0000A5F8F8B975F0D6FBB64B45F65820C5F87D
:107E1000049AC5F8003A0123C5F8086A2044C8F856
:107E200034A0C8F83CA045F6EC7A85F8443A25F031
:107E300087FE4046AC49A24485F868BA75F0BAFBA3
:107E400045F66C2039462044DEF034FA45F6D03051
:107E500039462044DDF060FE45F6345039460F9730
:107E60002044DEF047FE59462C2205F6E46067F117
:107E7000DFFD45F61C7345F6B4609C49E31845F6F2
:107E80004C7B20441F46119375F094FB984A07F1F0
:107E90000C00A344C5F81C2FF4F008FF0F9F5846B0
:107EA0000BF1140B8FF0F2FAD345F8D104F5C04A68
